:100000000C9464170C9495170C9495170C949517F1
:100010000C9495170C9495170C9495170C949517B0
:100020000C9495170C9495170C9495170C949517A0
:100030000C9495170C94BD620C9495170C9495171D
:100040000C9495170C944DC50C9495170C9495171A
:100050000C9495170C9495170C942C590C9473626E
:100060000C9495170C94DC3E0C9495170C949517F2
:100070000C9495170C9495170C9495170C94951750
:100080000C9495170C9495170C9495170C94951740
:100090000C9495170C9495170C9495170C94951730
:1000A0000C9495170C9495170C9495170C94951720
:1000B0000C9495170C9495170C9495170C94951710
:1000C0000C9495170C9495170C9495170C94951700
:1000D0000C9495170C9495170C94174C0C94D84BC2
:1000E0000C949517672F842FB52FD22FE72F103040
:1000F0007D30E3308C31253633362C366536693623
:1001000083360F3B9836E4360B3732375B37B137DF
:10011000C237D637E737F83709380F3B1A3A0F3B63
:10012000253A953A9B3ABB3A0F3F153F263F313F60
:10013000393F4E3F3D3F4E3F413F453F4E3F4B3F96
:100140008EB491B480B484B48AB4C8B495B499B46C
:100150009FB4A3B4A7B4ADB4B1B4B5B4C8B4BBB480
:10016000BFB4C3B4A4BAA9BAAEBAB8BAC2BA3BBB98
:10017000CCBAD4BADCBAE6BAF0BAFABA09BB13BB45
:100180003BBB1DBB27BB31BB084AD73B3BCE016EF7
:1001900084BCBFFDC12F3D6C74319ABD56833DDADE
:1001A0003D00C77F11BED9E4BB4C3E916BAAAABEED
:1001B000000000803F05A84CCDB2D44EB93836A916
:1001C000020C50B9918688083CA6AAAA2ABE000053
:1001D00000803F004E414E494E495459494E46CD4C
:1001E000CCCC3D0AD7233C17B7D13877CC2B3295EE
:1001F00095E6241FB14F0A000020410000C84200CC
:10020000401C4620BCBE4CCA1B0E5AAEC59D744352
:100210004F4D4D554E49434154494F4E004452595C
:1002200052554E004552524F525300494E464F00D0
:100230004543484F0047322F4733206261642070A6
:100240006172616D65746572730A00206F662000CB
:100250004D424C2047323920706F696E742000295E
:100260000A0059206F7574206F662072616E676591
:100270002028312D00290A0058206F7574206F66E0
:100280002072616E67652028312D004D65736820EE
:1002900070726F62696E6720646F6E652E0A00531C
:1002A00074617274206D6573682070726F62696E1C
:1002B0006720776974682022473239205331222021
:1002C00066697273742E0A004732380A4732392041
:1002D00053320053746174653A20004D6573682091
:1002E000626564206C6576656C696E672068617311
:1002F000206E6F20646174612E0A0053206F757444
:10030000206F662072616E67652028302D35292E9A
:100310000A004D65736820706F696E742063616EAA
:100320006E6F74206265207265736F6C7665640A07
:1003300000456E642066696C65206C6973740A0000
:10034000426567696E2066696C65206C6973740A22
:10035000004D31323500286E6F2066696C652900CA
:100360005344207072696E74696E67206279746597
:1003700020004E6F74205344207072696E74696E51
:10038000670A0043757272656E742066696C653A1F
:10039000200046696C652064656C657465643A008C
:1003A00044656C6574696F6E206661696C65642C68
:1003B0002046696C653A20005072696E7420746939
:1003C0006D653A20006F6E2E0A006F66662E0A0079
:1003D000473236204465627567200030022B0224C4
:1003E000021D020F026F66660044454255473A00FF
:1003F0004D3131332053006F6B002C20002C200036
:10040000544845524D414C5F50524F544543544916
:100410004F4E004155544F5245504F52545F534434
:100420005F53544154555300454D455247454E4343
:10043000595F50415253455200434153455F4C4927
:100440004748545F4252494748544E45535300541D
:100450004F47474C455F4C494748545300534F461C
:1004600054574152455F504F574552004255494CF1
:10047000445F50455243454E54004C4556454C4907
:100480004E475F44415441005A5F50524F4245002D
:100490004155544F4C4556454C005052494E545FBF
:1004A0004A4F420050524F47524553530041555412
:1004B0004F5245504F52545F54454D5000564F4C8B
:1004C000554D455452494300454550524F4D0053F8
:1004D000455249414C5F584F4E5F584F4646004683
:1004E00049524D574152455F4E414D453A4D61721B
:1004F0006C696E20312E312E392028476974687559
:10050000622C20646176696472616D69726F292062
:10051000534F555243455F434F44455F55524C3A04
:1005200068747470733A2F2F6769746875622E63EC
:100530006F6D2F4D61726C696E4669726D77617275
:10054000652F4D61726C696E2050524F544F434F6E
:100550004C5F56455253494F4E3A312E30204D4153
:100560004348494E455F545950453A416E79637549
:10057000626963206933204D656761204558545294
:10058000554445525F434F554E543A3120555549D5
:10059000443A63656465326132662D343161322DCF
:1005A000343734382D396231322D63353563363284
:1005B0006633363766660A002F2F2000205400204D
:1005C0005200416363656C65726174696F6E3A20B5
:1005D00050005741524E494E4721204C6F77205AC8
:1005E000204A65726B206D6179206C6561642074AE
:1005F0006F20756E77616E746564207061757365C8
:10060000732E0A00546F6F206661722066726F6DE0
:10061000207265666572656E636520706F696E74C1
:100620000A0020466C6F773A200000013637260317
:100630002BFFFFFF3C3D382AFFFFFFFF2E303E120D
:10064000FFFFFFFFFFFFFF0809FF2C071A1C18FF21
:10065000FFFF08440A2C4324221E20643A0020692C
:100660003A0020703A00496E76616C6964206578C2
:100670007472756465720A0043290A0061626C65D0
:100680006420286D696E2074656D702000436F6C66
:1006900064206578747275646573206172652000EA
:1006A00020643A0020693A0020703A004E6F2063BF
:1006B000617365206C696768740A00454550524F44
:1006C0004D204F4B0A00205A004475616C20456E46
:1006D0006473746F702041646A7573746D656E74B1
:1006E00020286D6D293A20003F4B2076616C75659E
:1006F000206F7574206F662072616E6765202830E8
:100700002D3130292E0A00416476616E6365204BDD
:100710003D0041637469766520457874727564653F
:10072000723A2000496E76616C6964206578747253
:10073000756465720A0043616E6E6F7420656E7435
:100740006572207375626469723A20004D313038E9
:10075000005370656369616C204D656E753A204D7C
:1007600031303820526573756D650A004D36303072
:10077000005370656369616C204D656E753A204D5C
:100780003630302050617573650A004739310A47A9
:1007900031205A2D302E310A4739300053706563AD
:1007A00069616C204D656E753A205A20446F776EF2
:1007B00020302E310A004739310A4731205A2D3076
:1007C0002E30320A473930005370656369616C20FE
:1007D0004D656E753A205A20446F776E20302E306A
:1007E000320A004739310A4731205A2B302E303235
:1007F0000A473930005370656369616C204D656E3E
:10080000753A205A20557020302E30320A00473970
:10081000310A4731205A2B302E310A4739300053E4
:1008200070656369616C204D656E753A205A20557C
:100830007020302E310A0047323920533200537075
:10084000656369616C204D656E753A204E657874FC
:10085000204D65736820506F696E740A0047323905
:10086000205331005370656369616C204D656E756E
:100870003A205374617274204D657368204C65761C
:10088000656C696E670A004D313430205336300094
:100890005370656369616C204D656E753A205072C6
:1008A0006568656174204265640A004D3530320028
:1008B0005370656369616C204D656E753A204C6FAD
:1008C00061642046572044656661756C74730A0044
:1008D0004D353030005370656369616C204D656E35
:1008E000753A205361766520454550524F4D0A00B8
:1008F0004D33303320452D312053363020433620C0
:100900005531005370656369616C204D656E753AB1
:10091000204175746F2054756E6520486F74626550
:1009200064205069640A004D31303620533230342F
:100930000A4D333033204530205332313020433696
:10094000205531005370656369616C204D656E758B
:100950003A204175746F2054756E6520486F746538
:100960006E64205049440A003C5370656369616CB1
:100970005F4D656E753E003C5370656369616C5FE9
:100980004D656E753E002F002F002F002F2E2E0A72
:10099000002F2E2E002F2E2E003C537065636961B0
:1009A0006C5F4D656E753E0A003C5370656369610E
:1009B0006C204D656E753E003C5370656369616CDB
:1009C000204D656E753E003C4D31303820526573C8
:1009D000756D653E003C4D31303820526573756D44
:1009E000653E003C4D3630302050617573653E00E9
:1009F0003C4D3630302050617573653E003C4C6F85
:100A000061642046572044656661756C74733E00CE
:100A10003C4C6F61642046572044656661756C7478
:100A2000733E003C4175746F2054756E6520486FAD
:100A300074626564205049443E003C4175746F20E7
:100A400054756E6520486F74626564205049443E59
:100A5000003C4175746F2054756E6520486F746555
:100A60006E64205049443E003C4175746F205475BB
:100A70006E6520486F74656E64205049443E003CAA
:100A8000457869743E003C457869743E003C53618A
:100A9000766520454550524F4D3E003C536176658A
:100AA00020454550524F4D3E003C4E657874204DD8
:100AB00065736820506F696E743E003C4E657874B3
:100AC000204D65736820506F696E743E003C53740E
:100AD000617274204D657368204C6576656C696E33
:100AE000673E003C5374617274204D657368204CFE
:100AF0006576656C696E673E003C5072656865613D
:100B000074206265643E003C5072656865617420C3
:100B10006265643E003C5A20446F776E20302E316F
:100B20003E003C5A20446F776E20302E313E003C10
:100B30005A20446F776E20302E30323E003C5A20CF
:100B4000446F776E20302E30323E003C5A20557074
:100B500020302E30323E003C5A20557020302E304E
:100B6000323E003C5A20557020302E313E003C5A17
:100B700020557020302E313E0056313136004A3338
:100B80003320004D3530300A4D3432302053310A95
:100B90004731205A313020463234300A473120580C
:100BA00030205930204636303030004A3232004A48
:100BB0003232004731205A3520463234300A47312C
:100BC0002058313930205932302046363030300A02
:100BD0004731205A302046323430004731205A35D0
:100BE00020463234300A47312058313930205931CB
:100BF00039302046363030300A4731205A302046CE
:100C0000323430004731205A3520463234300A47DA
:100C1000312058313930205932302046363030308A
:100C20000A4731205A302046323430004739310AE1
:100C30004731205A313020463234300A4739300AA1
:100C40004732380A4732390A473120583230205962
:100C500032302046363030300A4731205A30204674
:100C6000323430004A3032004A3132004731205AA3
:100C70003130004F4B004731205A31300047393076
:100C80000047312045256946353030004731204541
:100C90002D302E314625690047312045302E314612
:100CA0002569004731205A256946256900473120CA
:100CB0005A2D302E31462569004731205A302E31C9
:100CC0004625690047312059256946256900473185
:100CD00020592D302E314625690047312059302EBC
:100CE0003146256900473120582569462569004766
:100CF0003120582D302E314625690047312058309B
:100D00002E314625690047393100473238004732D5
:100D100038205A00473238205900473238205800CE
:100D20004132305620004731205A3130004A3034A9
:100D3000004A3231004A3230004B494C4C45442E77
:100D400020004A303400454E4400464E20004A30D0
:100D500032003939393A393939004D0048004137C4
:100D6000562000413656202D2D2D004A30320041AC
:100D7000365620005A3A2000593A2000583A2000AE
:100D8000413556004134562000413356200041324F
:100D9000562000413156200041305620004D383455
:100DA00000473930004731205A333520463234303D
:100DB0000047393100473930004731205A3130205F
:100DC000463234300047393100473930004731204E
:100DD0005A35204632343000473931004739300027
:100DE0004731205A31204632343000473931004AE9
:100DF0003136004A3138004A3134004A3030004A36
:100E00003031004A313000696E206D6F76655F7455
:100E10006F282920666565645F76616C756520665C
:100E20006F722058593A002C2065793D0029202DF9
:100E30003E202865783D002C2073793D0020436FCB
:100E40006E6E656374696E67207769746820766575
:100E500072746963616C206C696E65202873783DDB
:100E6000002C2065793D0029202D3E202865783D05
:100E7000002C2073793D0020436F6E6E65637469AA
:100E80006E67207769746820686F72697A6F6E7414
:100E9000616C206C696E65202873783D003F53704B
:100EA0006563696669656420582C5920636F6F72A9
:100EB00064696E617465206F7574206F6620626F5F
:100EC000756E64732E0A003F28522965706561743F
:100ED0002076616C7565206E6F7420706C6175731F
:100EE00069626C653B206D75737420626520617466
:100EF000206C6561737420312E0A003F28522965E9
:100F000070656174206D75737420626520737065FF
:100F1000636966696564207768656E206E6F74200A
:100F20007573696E6720616E204C43442E0A003F42
:100F3000537065636966696564206E6F7A7A6C6563
:100F40002074656D7065726174757265206E6F7462
:100F500020706C61757369626C652E0A003F537076
:100F6000656369666965642066696C616D656E7448
:100F70002073697A65206E6F7420706C6175736977
:100F8000626C652E0A003F5370656369666965642B
:100F9000207072696D65206C656E677468206E6F75
:100FA0007420706C61757369626C652E0A003F5025
:100FB00072696D65206C656E677468206D757374F9
:100FC000206265207370656369666965642077686F
:100FD000656E206E6F74207573696E6720616E2078
:100FE0004C43442E0A003F5370656369666965642B
:100FF000206E6F7A7A6C652073697A65206E6F74E3
:1010000020706C61757369626C652E0A003F5370C5
:1010100065636966696564205265747261637469A9
:101020006F6E204D756C7469706C696572206E6F9F
:101030007420706C61757369626C652E0A003F5292
:10104000657472616374696F6E204D756C7469703C
:101050006C696572206D75737420626520737065AC
:101060006369666965642E0A003F5370656369664B
:10107000696564206C617965722068656967687468
:10108000206E6F7420706C61757369626C652E0AD6
:10109000003F53706563696669656420626564201A
:1010A00074656D7065726174757265206E6F742001
:1010B000706C61757369626C65202834302D313431
:1010C0003043292E0A0047323620636F6D6D616E02
:1010D0006420737461727465642E20576169746949
:1010E0006E6720666F722068656174657228732967
:1010F0002E0A0024F4D43050C38E20C2A24017829E
:101100008B7011127A910D816CD90AA861E108C720
:10111000586607615143061E4B5D05C145A7041A79
:10112000411104093D9803713931034036DB0265F2
:10113000339102D4305402802E1D02632CEE0175CF
:101140002AC501B028A001102781018F2564012B39
:10115000244B01E0223401AC211F018D200D0180C0
:101160001FFC00841EED00971DDF00B81CD200E6B6
:101170001BC600201BBC00641AB200B219A8000AEA
:1011800019A0006A189900D117910040178B00B57B
:1011900016840031167E00B31579003A157300C726
:1011A000146F0058146A00EE13660088136300255C
:1011B000135E00C7125B006C12570015125400C179
:1011C00011510070114F0021114B00D61049008DB4
:1011D0001047004610440002104200C00F4000803B
:1011E0000F3E00420F3C00060F3B00CB0E38009331
:1011F0000E37005C0E3500270E3400F30D3200C1AF
:101200000D3100900D3000600D2E00320D2D0005C7
:101210000D2C00D90C2B00AE0C2900850C29005C8C
:101220000C2700350C27000E0C2600E80B2400C408
:101230000B2400A00B23007D0B23005A0B21003947
:101240000B2100180B2000F80A1F00D90A1E00BB52
:101250000A1E009D0A1D00800A1D00630A1C00472B
:101260000A1B002C0A1B00110A1A00F7091A00DDDC
:10127000091900C4091900AB091900920917007B6C
:10128000091800630917004C0916003609160020DA
:101290000916000A091500F5081500E0081400CC2D
:1012A000081400B8081400A4081400900813007D66
:1012B0000812006B08130058081200460812003488
:1012C000081100230811001208110001081100F094
:1012D000071000E0071000D0071000C0071000B092
:1012E000070F00A107100091070E0083070F00747D
:1012F000070F0065070E0057070E0049070E003B59
:10130000070D002E070E0020070D0013070D000625
:10131000070D00F9060C00ED060D00E0060C00D4E8
:10132000060C00C8060C00BC060C00B0060C00A49D
:10133000060B0099060C008D060B0082060B007749
:10134000060B006C060B0061060A0057060B004CEA
:10135000060A0042060A0038060A002E060A002481
:10136000060A001A060A001006090007060A00FD10
:10137000050900F4050900EB050900E2050900D99B
:10138000050900D0050900C7050900BE050900B51B
:10139000050800AD050800A50509009C0508009496
:1013A0000508008C050800840508007C0508007409
:1013B0000508006C050700650508005D0507005677
:1013C0000508004E050700470507004005080038DE
:1013D000050700310507002A050700230507001C43
:1013E000050600160507000F0507000805060002A0
:1013F000050700FB040600F5040700EE040600E8FC
:10140000040600E2040700DB040600D5040600CF52
:10141000040600C9040600C3040600BD040600B7A4
:10142000040600B1040500AC040600A6040600A0F2
:101430000405009B04060095040500900406008A3C
:1014400004050085040500800406007A0405007583
:10145000040500700405006B0405006604050061C6
:101460000405005C04050057040500520405004D06
:1014700004050048040500430405003E0404003A46
:1014800004050035040500300404002C0405002781
:10149000040400230405001E0404001A04040016BA
:1014A000040500110404000D0404000904050004EF
:1014B00004040000040400FC030400F8030400F426
:1014C000030400F0030400EC030400E8030400E458
:1014D000030400E0030400DC030400D8030400D488
:1014E000030400D0030400CC030400C8030300C5B8
:1014F00003030024F404D9201BC40C5C0E9804C41C
:10150000095F0265077101F405F900FB04B30048A7
:10151000048700C10369005803550003034500BE5A
:10152000023A008402310053022A002902250004F5
:10153000022000E4011C00C8011900AF0117009847
:1015400001140084011300710110006101100051A9
:10155000010E0043010D0036010B002B010B002092
:10156000010B00150109000C01090003010800FB33
:10157000000800F3000800EB000700E4000600DEAE
:10158000000600D8000600D2000600CC000500C707
:10159000000500C2000500BD000400B9000400B54C
:1015A000000400B1000400AD000400A9000400A57F
:1015B000000300A20003009F0004009B00030098AA
:1015C0000003009500020093000300900003008DCB
:1015D0000002008B000300880002008600020084E5
:1015E000000300810002007F0002007D0002007BFA
:1015F000000200790002007700010076000200740A
:1016000000020072000100710002006F0002006D14
:101610000001006C0002006A00010069000200671E
:101620000001006600010065000100640002006224
:1016300000010061000100600001005F0002005D28
:101640000001005C0001005B0001005A000100592C
:10165000000100580001005700010056000100552C
:10166000000100540001005300000053000100522B
:1016700000010051000100500001004F0001004E28
:101680000000004E0001004D0001004C0001004B25
:101690000000004B0001004A000100490001004821
:1016A000000000480001004700010046000000461D
:1016B0000001004500000045000100440001004316
:1016C0000000004300010042000000420001004110
:1016D00000000041000100400001003F0000003F09
:1016E0000001003E0000003E0001003D0000003D02
:1016F0000001003C0000003C0000003C0001003BF9
:101700000000003B0001003A0000003A00010039EF
:1017100000000039000100380000003800000038E7
:1017200000010037000000370001003600000036DD
:1017300000000036000100350000003500000035D3
:1017400000010034000000340000003400010033C8
:1017500000000033000000330001003200000032BE
:1017600000000032000100310000003100000031B3
:101770000001003000000030000000300001002FA8
:101780000000002F0000002F0000002F0001002E9D
:101790000000002E0000002E0001002D0000002D92
:1017A0000000002D0000002D0001002C0000002C86
:1017B0000000002C0000002C0001002B0000002B7A
:1017C0000000002B0000002B0001002A0000002A6E
:1017D0000000002A0000002A000100290000002962
:1017E0000000002900000029000000290001002855
:1017F0000000002800000028000000280000002849
:10180000000100270000002700000027000000273B
:10181000000000270001002600000026000000262E
:101820000000002600000026000100250000002521
:101830000000002500000025000000250000002514
:101840000001002400000024000000240000002407
:1018500000000024000100230000002300000023FA
:1018600000000023000000230000002300000023EC
:1018700000010022000000220000002200000022DF
:1018800000000022000000220001002100000021D1
:1018900000000021000000210000002100000021C4
:1018A00000000021000100200000002000000020B6
:1018B00000000020000000200000002000000020A8
:1018C000000000200001001F0000001F0000001F9A
:1018D0000000001F0000001F0000001F0000001F8C
:1018E0000001001E0000001E0000001E0000001E7F
:1018F000000000232C0000B8220000561800003A17
:101900000F0000B8080000B1040000710200003EA2
:101910000100001000C90210012C014001220170D9
:10192000011801B0010E01F00104015002FA00B0EB
:1019300002F0003003E600D003DC009004D2007017
:1019400005C800A006BE000008B400B009AA00D077
:101950000BA000600E960060118C00001582002024
:10196000197800C01D6E00A0226400B0275A0090B4
:101970002C500000314600E0343C0010383200901A
:101980003A2800603C1E00A03D1400803E0A002062
:101990003F00002CFFFFFFFFFF000101010101627A
:1019A00065640A002C2073797374656D2073746FFD
:1019B0007070656421204865617465725F49443ABE
:1019C00020004265642068656174696E6720666105
:1019D000696C65640048656174696E672066616959
:1019E0006C65640045312048656174696E672066E6
:1019F00061696C65640048656174696E6720666141
:101A0000696C6564004B494C4C45442E20007001C4
:101A10002C0190012701B0012201C0011D01F0013C
:101A200018011002130130020E0160020901900238
:101A30000401C002FF000003FA004003F500800328
:101A4000F000D003EB002004E6007004E100E004A5
:101A5000DC004005D700C005D2004006CD00D0060E
:101A6000C8008007C3003008BE00F008B900C009F4
:101A7000B400B00AAF00B00BAA00D00CA500000E55
:101A8000A000500F9B00C01096005012910000144F
:101A90008C00C0158700B0178200B0197D00D01BE4
:101AA0007800001E730040206E0090226900F02430
:101AB000640040275F0090295A00E02B5500102E4B
:101AC000500020304B0010324600E033410090358A
:101AD0003C001037370070383200A0392D00B03A82
:101AE0002800A03B2300603C1E00103D1900903DE3
:101AF0001400103E0F00703E0A00C03E0500003F7B
:101B00000000403FFBFF803FF6FFC03FF1FF453143
:101B100020544845524D414C2052554E4157415951
:101B20000042454420544845524D414C2052554EA8
:101B30004157415900546865726D616C2052756E51
:101B400061776179004531204572723A204D4158E4
:101B500054454D50004572723A204D415854454D00
:101B60005020424544004D415854454D5020747218
:101B700069676765726564004531204572723A2075
:101B80004D494E54454D50004572723A204D494ED4
:101B900054454D5020424544004D494E54454D500A
:101BA00020747269676765726564004D3834205827
:101BB0002059205A204500202F002042403A002082
:101BC000403A00024A3135004A3132004A3137008A
:101BD0002020506C616E6E65724275666665724259
:101BE000797465733A20002046726565204D656DF5
:101BF0006F72793A2000436F6D70696C65643A20AA
:101C000046656220203520323031390A00207C20A0
:101C1000417574686F723A202864617669647261F4
:101C20006D69726F2C20666F7220416E79637562E8
:101C30006963206933204D656761290A00323031BC
:101C4000392D30322D303500204C617374205570A1
:101C500064617465643A2000312E312E390A004DDA
:101C600061726C696E0020536F66747761726520D3
:101C700052657365740A00205761746368646F6706
:101C80002052657365740A002042726F776E206F70
:101C900075742052657365740A0020457874657206
:101CA0006E616C2052657365740A00506F776572BF
:101CB00055700A0073746172740A004D3234004D1D
:101CC0003233202573006175746F25692E670065B6
:101CD00072726F722077726974696E6720746F20F8
:101CE00066696C650A00205A3A0020593A0020586B
:101CF0003A00656E6473746F7073206869743A207B
:101D000000446F6E6520736176696E672066696C4A
:101D1000652E0A004D3239003A004361703A0020C6
:101D20005A00205900580020204D61783A200020A8
:101D30005A00205900580020204D696E3A20004F6B
:101D40006E20004F666600536F667420656E647384
:101D5000746F70733A20004B6420002364656669D9
:101D60006E652044454641554C545F004B69200048
:101D700023646566696E652044454641554C545F51
:101D8000004B70200023646566696E6520444546FB
:101D900041554C545F00504944204175746F74752F
:101DA0006E652066696E697368656421205075747C
:101DB00020746865206C617374204B702C204B6913
:101DC00020616E64204B6420636F6E7374616E7467
:101DD000732066726F6D2062656C6F7720696E7418
:101DE0006F20436F6E66696775726174696F6E2EDE
:101DF000680A00504944204175746F74756E6520FF
:101E00006661696C6564212074696D656F75740A1B
:101E100000453120544845524D414C2052554E41C9
:101E20005741590042454420544845524D414C20A9
:101E300052554E4157415900546865726D616C208E
:101E400052756E617761790045312048656174692A
:101E50006E67206661696C65640042656420686530
:101E60006174696E67206661696C656400486561CC
:101E700074696E67206661696C656400504944202E
:101E80004175746F74756E65206661696C65642157
:101E90002054656D706572617475726520746F6F22
:101EA00020686967680A00204B643A2000204B696B
:101EB0003A2000204B703A20000A20436C61737373
:101EC000696320504944200A002054753A200020BC
:101ED0004B753A2000206D61783A2000206D696EC4
:101EE0003A200020643A200020626961733A2000A1
:101EF000504944204175746F74756E652066616940
:101F00006C6564212054656D7065726174757265CD
:101F100020746F6F20686967680A00504944204147
:101F200075746F74756E652073746172740A0050F5
:101F30004944204175746F74756E65206661696CE3
:101F400065642120426164206578747275646572ED
:101F5000206E756D6265720A004F66660A00466102
:101F60006465204865696768742000426564204C98
:101F70006576656C696E6720004661696C656420F2
:101F8000746F20656E61626C6520426564204C65EB
:101F900076656C696E670A004D65736820426564FA
:101FA000204C6576656C20646174613A0A004D6569
:101FB000736820706F696E742063616E6E6F742039
:101FC0006265207265736F6C7665640A004D343209
:101FD0003120696E636F7272656374207061726123
:101FE0006D657465722075736167650A00496E736B
:101FF0006572742066696C616D656E7420616E64D3
:102000002073656E64204D3130380A0053656E646C
:10201000204D31303820746F2068656174206E6FF8
:102020007A7A6C650A00496E736572742066696C11
:10203000616D656E7420616E6420707265737320CB
:10204000627574746F6E20286F72204D313038299C
:102050000A0020746F6F206C6F6E67206578747251
:102060007573696F6E2070726576656E7465640A4B
:102070000020636F6C6420657874727573696F6E8D
:102080002070726576656E7465640A00486F6D69CC
:102090006E67206661696C656400206E6F742065F0
:1020A0006E74657265642E0A0050726F7465637495
:1020B00065642050696E0A0046696C616D656E74D6
:1020C00020757365643A200053746174733A20007C
:1020D0002C204C6F6E67657374206A6F623A200023
:1020E000546F74616C2074696D653A20005374619B
:1020F00074733A20002C204661696C65643A2000B4
:102100002C2046696E69736865643A2000507269D4
:102110006E74733A200053746174733A20004A302D
:1021200036004A3034004A30370020573A004A30EF
:1021300038004A30390020573A00205A3A002059D6
:102140003A0020436F756E7420583A0020453A00DB
:10215000205A3A0020593A00583A00454550524F0B
:102160004D206461746173697A65206572726F7263
:102170002E0A00290A002062797465733B2063727D
:1021800063200053657474696E67732053746F72B3
:102190006564202800290A002062797465733B2059
:1021A00063726320002073746F72656420736574BA
:1021B00074696E67732072657472696576656420F0
:1021C0002800202863616C63756C61746564292143
:1021D0000A0020213D2000454550524F4D204352DA
:1021E00043206D69736D61746368202D20287374BA
:1021F0006F7265642920002053697A653A2000498E
:102200006E6465783A2000204D61726C696E3D56AF
:102210003535290A0028454550524F4D3D0045456A
:1022200050524F4D2076657273696F6E206D6973E1
:102230006D6174636820002569730025696D202530
:102240006973002569682025696D2025697300255B
:102250006964202569682025696D2025697300253A
:10226000697920256964202569682025696D202504
:10227000697300656E7175657565696E672022000A
:102280005072696E7465722073746F70706564202B
:1022900064756520746F206572726F72732E2046AC
:1022A000697820746865206572726F7220616E644F
:1022B00020757365204D39393920746F207265732C
:1022C000746172742E202854656D70657261747526
:1022D00072652069732072657365742E205365746E
:1022E000206974206166746572207265737461720E
:1022F00074696E67290A004E6F20436865636B73CB
:10230000756D2077697468206C696E65206E756DD7
:102310006265722C204C617374204C696E653A20A2
:10232000004E6F20436865636B73756D2077697429
:1023300068206C696E65206E756D6265722C204C2C
:10234000617374204C696E653A2000636865636B45
:1023500073756D206D69736D617463682C204C61B9
:102360007374204C696E653A20004C696E65204E8E
:10237000756D626572206973206E6F74204C617395
:1023800074204C696E65204E756D6265722B312C20
:10239000204C617374204C696E653A20004D3131D8
:1023A00030004D3331005344207265616420657202
:1023B000726F720A00446F6E65207072696E746984
:1023C0006E672066696C650A0020496E76616C69EB
:1023D0006420657874727564657220000000A0C086
:1023E00000000000000000000000574300005743B9
:1023F00000004D436F70656E206661696C65642CEA
:102400002046696C653A200043616E6E6F74206FE0
:1024100070656E2073756264697220004A30350001
:102420004A32330053442063617264206F6B0A00A8
:102430006F70656E526F6F74206661696C65640AB7
:1024400000766F6C756D652E696E697420666169C2
:102450006C65640A004572726F723A0053442069D9
:102460006E6974206661696C0A006563686F3A0082
:102470007C3C3E5E2B3D3F2F5B5D3B2C2A225C006B
:10248000627573793A2070617573656420666F7246
:1024900020696E7075740A00627573793A207061F4
:1024A0007573656420666F7220757365720A0062C9
:1024B0007573793A2070726F63657373696E670A1A
:1024C000004A3135004B494C4C45442E20004B49C5
:1024D0004C4C20636175736564206279204B494CD4
:1024E0004C20627574746F6E2F70696E0A004B49D0
:1024F0004C4C45442E20004B494C4C206361757375
:10250000656420627920746F6F206D75636820693F
:102510006E6163746976652074696D65202D206332
:10252000757272656E7420636F6D6D616E643A20B2
:10253000004A3131005072696E7465722068616CB6
:102540007465642E206B696C6C28292063616C6C47
:102550006564210A000000A0C00000000000000027
:102560000000004842000048420000804000000097
:10257000005761726E696E673A20486F6D696E67C9
:102580002042756D702044697669736F72203C201B
:10259000310A000202040000A0400000A040000038
:1025A000004000005C430000574300004D43FFFF24
:1025B000FF486F74656E6420746F6F20636F6C6486
:1025C0000A00486F74656E6420746F6F20636F6CCF
:1025D000640A0000002100240027002A002D00309A
:1025E00000330001010000040107010A010000227C
:1025F00000250028002B002E0031003400020100CD
:1026000000050108010B010000200023002600291D
:10261000002C002F00320000010000030106010918
:102620000105050505070508080808020202020A57
:102630000A08080404040401010101010101010365
:1026400003030303030303040707070C0C0C0C0C20
:102650000C0C0C0202020206060606060606060B13
:102660000B0B0B0B0B0B0B0102102020080810208A
:10267000401020408002010201080402010102040E
:1026800008102040808040201008040201800402CD
:102690000180402010080402010804020101020424
:1026A0000810204080010204081020408000000A29
:1026B0000B02090C0D0E08070304010000000000C6
:1026C000000000000000000000000000000000000A
:1026D00000000000000000000012111000000000C7
:1026E00000000000000000000000000000000000EA
:1026F000000000556E6B6E6F776E20636F6D6D61BD
:102700006E643A202200496E736572742066696CAB
:10271000616D656E7420616E6420707265737320E4
:10272000627574746F6E20286F72204D31303829B5
:102730000A002066697273740A005A005900580032
:10274000486F6D652000526573656E643A20006FB6
:102750006B0020746F6F206C6F6E672065787472E9
:102760007573696F6E2070726576656E7465640A44
:102770000020636F6C6420657874727573696F6E86
:102780002070726576656E7465640A00FFFDFCFA60
:10279000F8F6F4F2F0EEECEAE9E7E5E3E1E0DEDC9E
:1027A000DAD9D7D5D4D2D0CFCDCBCAC8C7C5C3C24A
:1027B000C0BFBDBCBAB9B7B6B4B3B2B0AFADACAAC6
:1027C000A9A8A6A5A4A2A1A09E9D9C9A9998979518
:1027D000949392908F8E8D8B8A898887868483824A
:1027E00081807F7E7D7B7A7978777675747372715C
:1027F000706F6E6D6C6B6A69686766656463626151
:10280000605F5E5D5C5B5A59585857565554535239
:102810005150504F4E4D4C4B4A4A49484746464509
:102820004443424241403F3E3E3D3C3B3B3A3938C7
:102830003837363535343332323130302F2E2E2D75
:102840002C2B2B2A29292827272625252423232218
:10285000212120201F1E1E1D1C1C1B1B1A191918AC
:1028600018171616151514131312121111100F0F35
:102870000E0E0D0D0C0C0B0A0A09090808070706B5
:1028800006050504040303020201000054524947EF
:102890004745524544006F70656E003A20007A3219
:1028A0005F6D696E007A5F6D696E00795F6D696E4C
:1028B00000785F6D696E005265706F7274696E6743
:1028C00020656E6473746F70207374617475730A1D
:1028D000000A4D6561737572656420706F696E746E
:1028E000733A0A005A206F66667365743A20004E88
:1028F000756D20582C593A20352C350A00000000FF
:102900000100000001000080005555550000004006
:102910000033333300AAAA2A004992240000002081
:1029200000C7711C0099991900D14517005555151C
:10293000003BB113002449120011111100000010D6
:10294000000F0F0F00E3380E0043790D00CCCC0CC4
:1029500000C3300C00E8A20B0064210B00AAAA0AF5
:1029600000703D0A009DD80900427B0900922409AD
:1029700000DCD30800888808001042080000000826
:1029800000F0C107008787070075500700711C071A
:10299000003EEB0600A1BC060069900600666606D4
:1029A00000703E06006118060017F4050074D1059A
:1029B000005BB00500B29005006272050055550538
:1029C0000078390500B81E0500050505004EEC0429
:1029D0000087D40400A1BD040090A704004992041C
:1029E00000C17D0400EE690400C75604004444049D
:1029F000005C3204000821040041100400000004BF
:102A0000003FF00300F8E0030026D20300C3C30335
:102A100000CCB503003AA803000A9B0300388E03DC
:102A200000C08103009F750300D0690300505E035E
:102A3000001D53030034480300913D03003333036A
:102A40000016290300381F030097150300300C03FC
:102A500000030303000BFA020049F10200BAE80286
:102A6000005CE002002DD802002DD0020059C802FF
:102A700000B0C0020031B90200DAB10200AAAA0215
:102A800000A0A30200BC9C0200FA9502005C8F0229
:102A900000DF88020082820200457C020027760265
:102AA0000027700200436A02007C640200D05E02CC
:102AB000003F590200C853020048617264636F64AA
:102AC00065642044656661756C742053657474692F
:102AD0006E6773204C6F616465640A00B80B000078
:102AE000B00400003C000000102700000000FA4382
:102AF0000000FA430000C040000070420000A04205
:102B00000000A0420000C8433333B94220286D6D55
:102B1000290020204D36303320002055004C00463F
:102B2000696C616D656E74206C6F61642F756E6C7D
:102B30006F6164206C656E677468733A0A002020C8
:102B40004D393030204B004C696E65617220416414
:102B500076616E63653A0A00204400204900202017
:102B60004D33303420500020440020490020204DB7
:102B70003330312050005049442073657474696EBD
:102B800067733A0A00205A0020204D363636004539
:102B90006E6473746F702061646A7573746D656EB2
:102BA000743A0A00205A0020590020204732392068
:102BB0005333205800205A0020204D343230205307
:102BC000004D65736820426564204C6576656C69CC
:102BD0006E673A0A00205A0020590020204D3230FA
:102BE00036205800486F6D65206F66667365743ACD
:102BF0000A00204500205A00205900205800205487
:102C00000020530020204D32303520510020453C1B
:102C10006D61785F655F6A65726B3E0020583C6D40
:102C200061785F785F6A65726B3E20593C6D6178B0
:102C30005F795F6A65726B3E205A3C6D61785F7A9E
:102C40005F6A65726B3E00416476616E6365643AEB
:102C500020513C6D696E5F7365676D656E745F745E
:102C6000696D655F75733E20533C6D696E5F666587
:102C70006564726174653E20543C6D696E5F747268
:102C80006176656C5F66656564726174653E00209F
:102C9000540020520020204D323034205000416337
:102CA00063656C65726174696F6E2028756E6974F6
:102CB000732F7332293A20503C7072696E745F61D1
:102CC0006363656C3E20523C726574726163745F2D
:102CD000616363656C3E20543C74726176656C5F21
:102CE000616363656C3E0A00204500205A0020594C
:102CF0000020204D3230312058004D6178696D75CB
:102D00006D20416363656C65726174696F6E202824
:102D1000756E6974732F7332293A0A0020450020BA
:102D20005A0020590020204D3230332058004D6188
:102D300078696D756D206665656472617465732070
:102D400028756E6974732F73293A0A002045002094
:102D50005A0020590020204D393220580053746504
:102D600070732070657220756E69743A0A002020B5
:102D70004D3230302044300A0020204D3230302097
:102D800044002044697361626C65640A0046696CA2
:102D9000616D656E742073657474696E67733A0053
:102DA0002020473231202020203B004572726F7274
:102DB0002077726974696E6720746F2045455052A0
:102DC0004F4D210A0057726974696E6720746F2035
:102DD00066696C653A20006F70656E206661696C8B
:102DE00065642C2046696C653A20006F70656E2022
:102DF0006661696C65642C2046696C653A20004602
:102E0000696C652073656C65637465640A002053A2
:102E1000697A653A200046696C65206F70656E6559
:102E2000643A20002066696C653A2000646F696E20
:102E300067006672657368004E6F772000454E44E8
:102E400020535542524F5554494E450A0022207096
:102E50006F73002220706172656E743A22005355C0
:102E600042524F5554494E452043414C4C207461C9
:102E7000726765743A22004B494C4C45442E200041
:102E8000747279696E6720746F2063616C6C207353
:102E900075622D67636F64652066696C6573207762
:102EA00069746820746F6F206D616E79206C65762F
:102EB000656C732E204D4158206C6576656C2069D9
:102EC000733A0000D6E88CEA11241FBECFEFD1E29E
:102ED000DEBFCDBF00E00CBF14E0A0E0B2E0EEED3D
:102EE000FEEE01E00BBF02C007900D92A432B107C5
:102EF000D9F729E1A4E2B4E001C01D92A133B207E1
:102F0000E1F717E1C3E6D7E100E006C02197010928
:102F1000802FFE010E94C7F6C236D10780E0080765
:102F2000A9F70E94F7E20C945EF70C9400002F9230
:102F30003F924F925F926F927F928F929F92AF9249
:102F4000BF92CF92DF92EF92FF920F931F93CF9396
:102F5000DF93CDB7DEB7C354D1090FB6F894DEBF07
:102F60000FBECDBF21E02093C510809148118D3454
:102F700009F459C5843511F40C94FB2B873411F0F6
:102F80000C94472C80914611909147118B319105FB
:102F900009F403C2A4F48430910534F4823091051D
:102FA00094F597FF29C03BC58430910509F4BFC152
:102FB0004A9709F034C50E94D1410C94492C8A32B9
:102FC000910509F421C444F48C31910509F415C22A
:102FD0004D9709F417C223C58B35910509F49FC499
:102FE0008C35910509F49FC48A35910509F017C500
:102FF000109235040C94492C8091190281110C9483
:103000004E2C0C94492C20911902222311F40C947B
:10301000492C11E0029709F010E00E949583198273
:103020001A821B821C821D821E821F82188682E5E4
:103030000E943440882309F42AC10E94B43F4B0106
:103040005C0120E030E0A9010E944EEF882309F4E2
:1030500034C140914C0450914D0460914E047091E4
:103060004F0448A759A76AA77BA7609150047091A5
:10307000510480915204909153046CA77DA78EA7B0
:103080009FA78091121190911311A0911411B091EA
:10309000151188AB99ABAAABBBAB409116115091FF
:1030A000171160911811709119114CAB5DAB6EAB9B
:1030B0007FAB9C01AD0168A579A58AA59BA50E945F
:1030C0004EEF81110DC02CA93DA94EA95FA96CA599
:1030D0007DA58EA59FA50E944EEF882309F4EDC023
:1030E00020E030E0A901C501B4010E944EEF881F25
:1030F0008827881F181749F060E070E080E89FEB90
:103100006CAF7DAF8EAF9FAF08C080E090E0A0E8CD
:10311000BFE38CAF9DAFAEAFBFAF28A539A54AA521
:103120005BA568A979A98AA99BA90E94CAF368AF7F
:1031300079AF8AAF9BAF2CA53DA54EA55FA56CA925
:103140007DA98EA99FA90E94CAF36B017C0128ADBD
:1031500039AD4AAD5BADCA01B9010E94B3EF2B0195
:103160003C01A7019601C701B6010E94B3EF9B0184
:10317000AC01C301B2010E94CBF30E9436F62B01D1
:103180003C0120E030E040E05FE30E94B3EF249692
:103190006CAF7DAF8EAF9FAF2497A5019401C501A1
:1031A000B4010E94B3EF4B015C0124962CAD3DAD00
:1031B0004EAD5FAD2497CA01B9010E94B3EF9B01E8
:1031C000AC01C501B4010E94CAF30E9436F62CADD1
:1031D0003DAD4EAD5FAD0E94B3EF4B015C01C70149
:1031E000B6019058A30192010E94A7F4A501940191
:1031F0000E94B3EF6B017C0128A939A94AA95BA9F8
:1032000068A579A58AA59BA50E94CBF320E030E0B4
:1032100040E05FE30E94B3EF9B01AC01C701B60140
:103220000E94CBF328A539A54AA55BA50E94CAF345
:1032300069837A838B839C832CA93DA94EA95FA9BE
:103240006CA57DA58EA59FA50E94CBF320E030E064
:1032500040E05FE30E94B3EF6B017C01A3019201A8
:1032600068AD79AD8AAD9BAD0E94A7F4A50194012C
:103270000E94B3EF9B01AC01C701B6010E94CBF3E2
:103280002CA53DA54EA55FA50E94CAF312C089E4F6
:103290000E943440882331F00E94B43F69837A83CE
:1032A0008B839C838AE40E943440882331F00E94FF
:1032B000B43F6D837E838F83988720E030E0A9013F
:1032C00069817A818B819C810E944EEF81110EC0B1
:1032D00020E030E0A9016D817E818F8198850E9478
:1032E0004EEF811103C0E5E5F4E20DC0412FBE01B0
:1032F0006F5F7F4F82E191E10E947EBB0C94492C6D
:103300000E94679AF80184918F010F5F1F4F81110E
:10331000F7CFE5E3F2E084918F010F5F1F4F882321
:1033200011F40C94492C0E94679AF801F4CF80E5BF
:103330000E943440882329F00E9475996B017C011A
:1033400003C0C12CD12C760183E50E943440882330
:1033500061F00E94B43F20E030E04AE754E40E946C
:10336000B3EF0E9414F56B017C010E94CF7E0E9496
:103370006762C60ED71EE81EF91E0E946762DC0156
:10338000CB018C199D09AE09BF09B7FD02C00C9491
:10339000492C80E00E946EAEF0CF0E9433B78111BD
:1033A0000C94492C80E090E0A0EAB0E489839A83F1
:1033B000AB83BC8380E090E0ADE4B3E48D839E8377
:1033C000AF83B88780E090E0A0EAB1E489879A876C
:1033D000AB87BC8780E50E943440882319F00E94A7
:1033E000843F01C060E068A3BE016F5F7F4FCE01E4
:1033F00080960E9472D00C94492C80E00E94C28674
:103400000C94492C83E50E943440882321F10E94CA
:10341000943F182F863070F0EBEFF2E084918F012B
:103420000F5F1F4F882311F40C94492C0E94679A58
:10343000F801F4CF833009F44AC130F4813091F1BE
:10344000823009F43FC008C0843009F4ABC1853034
:1034500009F4B8C101C010E00E941385811103C0B6
:10346000EBEDF2E013C08091E010882319F063E1E6
:1034700073E002C067E173E083ED92E00E9497C6BB
:103480008AE00E94679A0E9419D1A2C184917F01AB
:103490009FEFE91AF90A882309F49AC10E94679AF2
:1034A000F701F4CF0E94CCD11092010210920002D9
:1034B00088EC92E090934B0480934A040E94CF9A48
:1034C0000C94492C809100029091010297FF0EC04C
:1034D000EFE9F2E084918F010F5F1F4F882311F411
:1034E0000C94492C0E94679AF801F4CF0097A1F43C
:1034F00080913C028093360419821A821B821C82BE
:1035000018A219A21AA21BA2BE016F5F7F4FCE01A3
:1035100080960E94A48627C0815065E00E9493F6A1
:1035200080FF03C024E0291B922FA5E09A02F0013E
:103530001124E80FF11D87FDFA95EE0FFF1FEE0F26
:10354000FF1FED55F74E8091540490915504A091C2
:103550005604B091570480839183A283B3838091F2
:10356000360480933C0280910002909101028931DF
:1035700091050CF067C010923C029C012F5F3F4FF9
:10358000309301022093000265E00E9493F680FFD1
:1035900003C024E0291B922F4091540450915504FC
:1035A000609156047091570448A359A36AA37BA362
:1035B00019821A821B821C82B4E08B0290011124B2
:1035C000F901EC56F54F4F01208131814281538141
:1035D000F4E09F02C0011124BC016855754F5B01E6
:1035E000DB016D917D918D919C91FE0131966F0172
:1035F000E12CF12C00EA10E40E94B68519821A82AF
:103600001B821C82B601CE0180960E94A486F50121
:1036100080819181A281B38180934C0490934D0469
:10362000A0934E04B0934F04F40180819181A28154
:10363000B3818093500490935104A0935204B093AB
:103640005304C8C080E090E0A0EAB0E48093540442
:1036500090935504A0935604B09357040E945F853D
:103660000E94CF7E8FEF9FEF909301028093000224
:10367000EBE8F2E084918F010F5F1F4F882321F068
:103680000E94679AF801F6CF83E992E09A838983D2
:1036900004E610E019A308A3BE016F5F7F4FCE01BF
:1036A00080960E9430B88AEB92E09A83898319A3AE
:1036B00008A3BE016F5F7F4FCE0180960E9430B895
:1036C00081E00E94C28681E00E94408583C088E537
:1036D0000E9434408823D1F00E94843F1FEF160FD0
:1036E0001530D8F065E070E088E792E00E947EC671
:1036F000E5E7F2E084918F010F5F1F4F882311F4FB
:103700000C94492C0E94679AF801F4CF88E50E9436
:10371000679A0E94C6E80C94492C89E50E943440BF
:103720008823D1F00E94843F0FEF060F0530D8F0B8
:1037300065E070E082E692E00E947EC6EFE5F2E08E
:1037400084918F010F5F1F4F882311F40C94492C33
:103750000E94679AF801F4CF89E50E94679A0E9457
:10376000C6E80C94492C8AE50E943440882399F0DD
:103770000E94B43F25E0129FF0011124E00FF11DDB
:10378000EE0FFF1FEE0FFF1FED55F74E60837183A5
:103790008283938335C08AE50E94679A0E94C6E8B7
:1037A0000C94492C8AE50E9434408823A1F30E949E
:1037B000B43F60939F187093A0188093A1189093C2
:1037C000A2181EC080E00E9440850E94CCD118C083
:1037D0001230B1F4609100027091010269317105FB
:1037E00014F069E170E080E592E00E947EC669E134
:1037F00070E08BE492E00E947EC68AE00E94679AA5
:103800000E94E07E0C94492C80911902882311F4C7
:103810000C94492C89E40E943440E82E882321F03E
:103820000E94843F062F01C000E08AE40E943440D9
:10383000F82E882321F00E94843F162F01C010E04B
:10384000EE2011F0053020F4FF2081F0153070F0EB
:10385000E2E1F3E084918F010F5F1F4F882311F4A1
:103860000C94492C0E94679AF801F4CF0E944040C2
:10387000EE2091F044E00402F0011124E855F54FE8
:1038800080819181A281B381809312119093131151
:10389000A0931411B0931511FF2091F054E015027C
:1038A000F0011124EC56F54F80819181A281B38102
:1038B0008093161190931711A0931811B0931911BA
:1038C00080E50E943440882319F00E94A53F03C080
:1038D00080E50E94EB3F86E40E9434408823D9F0C3
:1038E0000E94B43F6B017C0120E030E0A9010E94FE
:1038F000F1F5181684F420E030E040E752E4C70107
:10390000B6010E94A7F460933D0270933E0280933B
:103910003F02909340020E9492BF0C94492C209346
:1039200035040C94492C27E5222E22E0322E36E76E
:10393000E32E30E1F32E6CE474E079A768A744E24B
:10394000C42E44E0D42E00E010E0D1018D911D0181
:103950000E943440882309F44BC00E94B43F2B01DD
:103960003C01133049F0F6012081318142815381BD
:103970000E94CAF32B013C01A8A5B9A52D913D9148
:103980004D915C91C301B2010E94CAF34B015C01ED
:103990002DEB37E346E855EB0E94F1F587FD0AC0B1
:1039A0002DEB37E346E855E3C501B4010E944EEF25
:1039B0001816F4F4133051F44092580450925904FC
:1039C00060925A0470925B0401E012C0A501940158
:1039D000F70160817181828193810E94CBF3D701CD
:1039E0006D937D938D939C931397812F0E94EE98F6
:1039F0001F5FB4E0EB0EF11CE8A5F9A53496F9A71A
:103A0000E8A7F4E0CF0ED11C143009F09ECF0023BC
:103A100009F4F6CE88E594E00E94D2B6F1CE0E9479
:103A2000CEB90C94492C809146119091471185375D
:103A3000910511F40C94492C0CF0C0C08C34910504
:103A400009F408C50CF058C08931910509F4E8C2A1
:103A50001CF58431910509F4C9C17CF481319105CB
:103A600009F44AC22CF4029708F4C3C10C94F82B51
:103A7000429709F4E0C60C94F82B8631910509F4BD
:103A800089C20CF483C28731910509F489C2489731
:103A900009F49CC20C94F82B8E31910509F47EC375
:103AA00084F48B31910509F4D7C20CF4C7C28C3170
:103AB000910509F469C34D9711F40C94492C0C94A9
:103AC000F82B8A32910509F46CC44CF48F319105BE
:103AD00009F442C4809709F4F3C30C94F82B8133A2
:103AE000910509F492C48B34910511F00C94F82BD4
:103AF0000E94B2C60C94492C8936910509F472C50E
:103B000044F58335910509F492C69CF48E349105F1
:103B100009F4A8C40CF4A2C48135910509F475C652
:103B20008235910511F00C94F82B109234040C940A
:103B3000492C8535910509F4B1C60CF47CC68C3549
:103B4000910509F4C4C68836910509F48FC40C9414
:103B5000F82B8E36910509F4B2C4A4F48B36910586
:103B600009F4BAC50CF49AC58C36910511F40C947D
:103B7000492C8D36910511F00C94F82B0E94AF87DB
:103B80000C94492C8137910509F4FFC45CF48F36FD
:103B9000910509F4A7C48037910511F40C94492CC0
:103BA0000C94F82B8237910509F419C783379105D6
:103BB00011F00C94F82BEFEDF4E050C78E3221E0B9
:103BC000920711F40C94AB290CF082C0893C91054A
:103BD00011F40C942F267CF58D37910509F48EC5D0
:103BE000ACF48737910509F4E1C70CF492C7883724
:103BF000910509F4DEC78937910511F00C94F82B73
:103C00001092E6051092E5050C94492C8B3991052C
:103C100009F403C534F48C38910509F425C50C94D6
:103C2000F82B8E3B910509F435C5883C910509F4C4
:103C3000C6C70C94F82B833D910511F40C943B28D6
:103C400044F58C3C910511F40C9466266CF48B3C85
:103C5000910511F00C94F82BA7E5EA2EA2E0FA2EBC
:103C60000EE917E00C9456268D3C910511F40C9446
:103C7000DB268E3C910511F00C94F82BE7E5CE2E57
:103C8000E2E0DE2EF7EEEF2EF5E0FF2E10E00C94D2
:103C90006227823E910511F40C94B92864F48C3D9E
:103CA000910511F40C943E288D3D910511F40C946E
:103CB0004B280C94F82B8C3251E0950711F40C949E
:103CC000E2288D32914011F40C940B290C94F82BBE
:103CD000863F71E0970711F40C949B2A0CF043C0C7
:103CE0008A39B1E09B0711F40C94492CBCF4803361
:103CF000F1E09F0711F40C94022A14F40C94FF29AC
:103D0000833641E0940709F46DC08039914011F089
:103D10000C94F82B0E94CF7E0C94492C8C3A61E0D5
:103D2000960711F40C9475277CF4843AA1E09A0765
:103D300011F40C94952A853A914011F00C94F82BCB
:103D40000E942E650C94492C843FE1E09E0711F4FB
:103D50000C94982A853F914011F00C94F82B0E9406
:103D60000A900C94492C8B3522E0920711F40C94A4
:103D7000D72AC4F4883F51E0950711F40C94AA2A7D
:103D800014F40C949E2A8C3072E0970711F40C9472
:103D9000CE2A8835924011F00C94F82B0E945C6377
:103DA0000C94492C8B38B3E09B0711F40C94492CEC
:103DB0006CF48A39F2E09F0711F40C94602B84387C
:103DC000934011F40C948D2B0C94F82B803A43E023
:103DD000940709F4B4C2873E934011F40C94E52B88
:103DE0000C94F82BE5E5F4E20C94822AE0E4F3E08D
:103DF0008FC0A0904411B090451180E50E943440DE
:103E0000882359F00E9475996B017C0111E0672BA2
:103E1000682B692B31F410E004C010E0C12CD12CC8
:103E2000760183E50E943440882311F40C94532CCE
:103E30000E94B43F20E030E04AE754E40E94B3EF30
:103E40000E9414F56B017C0111110BC0672B682BCC
:103E5000692B39F4A114B10421F0D5018C918111A1
:103E600002C010E001C011E00E94CF7E1123B9F022
:103E7000EAE6F4E284918F010F5F1F4F882321F05F
:103E80000E94679AF801F6CFF50181915F018823BE
:103E900019F00E94679AF8CF8AE00E94679A83E03F
:103EA0008093C51081E08093C410C114D104E10453
:103EB000F104B1F00E946762C60ED71EE81EF91E1B
:103EC0000E946762DC01CB018C199D09AE09BF0914
:103ED000B7FF0EC08091C41081110C94582C08C0FB
:103EE0008091C410882321F080E00E946EAEF8CF4C
:103EF0001092C4100C94492C5F988A98479880912E
:103F00000801817080930601479812980C94492CFF
:103F100084918F010F5F1F4F882321F00E94679AC1
:103F2000F801F6CF10925A0D8DE09BE00E9416A783
:103F30008BE1EDE0FBE0DE01159601900D928A9594
:103F4000E1F780910B0B90910C0B9C838B838DEE92
:103F500092E09A83898340E050E0BE016F5F7F4F1B
:103F600080E090E00E94F5A1CE0101960E9404AE8F
:103F7000E1E3F3E084918F010F5F1F4F882311F479
:103F80000C94492C0E94679AF801F4CF0E94F99F83
:103F90000C94492C1092DC0A1092DD0A0C94492CE6
:103FA000E0914411F09145118081882329F08032FD
:103FB00009F410823196F8CF40E061E0809144111D
:103FC000909145110E9482DE0C94492C80E090E093
:103FD000A8E4B2E489839A83AB83BC8318A219A2B4
:103FE0001AA21BA21CA21DA21EA21FA280914F08F2
:103FF000882359F020E0AE014F5F5F4FBE01605E45
:104000007F4FCE0184960E9464B88091DD0A882398
:1040100019F081E08093DC0A0E94B2C60C94492C0E
:104020001092DC0A0E94F06181E593E090934B04CA
:1040300080934A040E94CF9A0C94492C8091DD0A07
:10404000882311F40C94492C83E50E94344081119B
:104050000C945D2C0C94492C83E40E94EB3F882344
:1040600009F450C0E3E8F3E084918F010F5F1F4F24
:10407000882321F00E94679AF801F6CF8091A80C5E
:10408000811103C0E6E5F3E012C0BE016F5F7F4F10
:1040900085EA9CE00E94DEA58E010F5F1F4FD801CC
:1040A0008D918D01882349F10E94679AF8CF849100
:1040B0008F010F5F1F4F882301F10E94679AF8015B
:1040C000F6CF9BEDC92E93E0D92EE12CF12C20E008
:1040D0008091BA0790E00E2C02C0959587950A94BE
:1040E000E2F780FD2FC24FEFE41AF40A52E0C50E4A
:1040F000D11C65E0E616F10459F78AE00E94679A40
:104100000C94492C8091DD0A882339F08091DC0AD7
:10411000882319F0E0E6F3E003C0E2E7F3E028C00B
:1041200084918F010F5F1F4F882321F00E94679AAF
:10413000F801F6CF6091560D7091570D8091580D92
:104140009091590D4AE00E94A39D8FE20E94679AC8
:104150006091520D7091530D8091540D9091550DB9
:104160004AE00E94A39D8AE00E94679A0C94492C21
:1041700084918F010F5F1F4F882311F40C94492CF9
:104180000E94679AF801F4CF40E060E0809144110A
:10419000909145110E9482DE0C94492C8091DD0A99
:1041A000882311F40C94492C85EA9CE00E94AFDC32
:1041B00085EA9CE00E94B9A51092DB0A1092DA0A07
:1041C0008091DD0A882311F40C94492C009144114C
:1041D000109145110E94E7A1B801CE0180960E947E
:1041E000FAA38C01892B11F40C94492C68A179A1B4
:1041F0006115710511F06C5F7F4F19821C8222E0FE
:10420000A801CE0101960E9445AB811102C0F12C9C
:1042100014C0CE0101960E9457A18823C1F361E02A
:10422000CE0101960E94C2A5009789F325EEFC01FC
:1042300020831C820E9458DAF82ECE0101960E943B
:10424000619AF11003C0E0EAF3E022C0E2E9F3E092
:1042500084917F012FEFE21AF20A882321F00E9455
:10426000679AF701F5CFD8018D918D01882319F058
:104270000E94679AF8CF8AE00E94679A1092560DC2
:104280001092570D1092580D1092590D0C94492C04
:1042900084917F01BFEFEB1AFB0A882321F00E9473
:1042A000679AF701F5CFF80181918F01882319F002
:1042B0000E94679AF8CF8EE20E94679A0C94492C6C
:1042C0008091DC0A81110E94CF7E8091DD0A8823D3
:1042D00011F40C94492C80E50E943440882319F095
:1042E0000E94A53F03C080E50E94EB3F182F482F96
:1042F00061E080914411909145110E9482DE83E536
:104300000E943440882381F00E94843FAB01BC01AD
:104310004093560D5093570D6093580D7093590D5F
:1043200085EA9CE00E94CFA48091DD0A882319F0E1
:1043300081E08093DC0A11110C94492C6DCE8091A0
:1043400044119091451121E02093DB0A40E060E0A8
:104350000E9482DE0C94492C0E94A26168A379A37A
:104360008AA39BA3BE016F5F7F4FCE0180960E9400
:104370008599EAE6F4E284918F010F5F1F4F88234D
:1043800021F00E94679AF801F6CFBE016F5F7F4F60
:1043900088EB93E00E9497C68AE00E94679A0C948B
:1043A000492C83E50E943440882311F40C94492C55
:1043B0000E94943FE82E80E50E943440882339F023
:1043C0000E94943F182F87FF03C00C94492C1DE0D6
:1043D00089E40E943440882341F00E94A53F811166
:1043E0000C94DA2CEAE2F6E00BC089E40E94EB3F81
:1043F000F6CF319626E0EA35F20711F40C94DA2C68
:1044000084911813F6CF0C94AE2CF090300481E018
:10441000F826F0923004E0EDF3E084918F010F5F15
:104420001F4F882321F00E94679AF801F6CFFF20E2
:1044300019F0E5ECF3E002C0EAECF3E084918F01BF
:104440000F5F1F4F882311F40C94492C0E94679A28
:10445000F801F4CF0E94F0610C94492C0E94F9C637
:104460000C94492C0E947B810C94492C88E690E0A6
:104470000E946E9A81110C94492C8091BA0783FF97
:1044800002C00C94492C83E50E943440882399F0A3
:104490000E94B43F0E940FF5CB010E94FB590E947D
:1044A000B43F20E030E04AEA52E40E944EEF181692
:1044B00014F00E94F9C60E94AAC80C94492C8EE4FC
:1044C0000E943440882311F40C94492C0E94843FAC
:1044D00060932719709328198093291990932A19AA
:1044E0000C94492C83E50E94EB3F882359F083E527
:1044F0000E943440882319F00E94943F01C080E05C
:104500008093BA07EAE6F4E284918F010F5F1F4FB0
:10451000811103C0E9EEF3E004C00E94679AF8013C
:10452000F3CF84918F010F5F1F4F882321F00E94EA
:10453000679AF801F6CF8091BA078111C2CDE5EEF6
:10454000F3E018C0BB24B394B20E222319F08CE21E
:104550000E94679AF60185919491FC0184918F01E4
:104560000F5F1F4F882321F00E94679AF801F6CF52
:104570002B2DB9CD84918F010F5F1F4F882309F434
:10458000BCCD0E94679AF801F5CF83E50E943440C4
:10459000811103C0EAE6F4E20DC00E94943F8D331E
:1045A00020F4809329020C94492C8CE380932902F7
:1045B0000C94492C84918F010F5F1F4F882321F0A9
:1045C0000E94679AF801F6CF4091290250E060E01E
:1045D00070E080EF93E00E9444C68AE00E94679AF0
:1045E0000C94492C89E690E00E946E9A811111C0CA
:1045F000E7EFF3E084918F010F5F1F4F882321F0D5
:104600000E94679AF801F6CF0E94A9588AE00E949A
:10461000679A1092C5100C94EF2C83E50E943440E9
:10462000882311F40C94492C0E94943F182F8D3349
:1046300008F01CE3109375100E9467626B017C0107
:10464000212F30E0A8EEB3E00E94BBF3C60ED71EC8
:10465000E81EF91EC0927110D0927210E092731091
:10466000F09274100C94492C8091BA0783FF02C019
:104670000C94492C83E50E943440882311F40C9457
:10468000492C0E94B43F0E940FF5CB010E94C34108
:104690000C94492C0E94AA7F0C94492C80E50E941E
:1046A0003440811106C083E50E943440882361F0C4
:1046B00006C00E94943F81110C94492CF4CF0E94B3
:1046C000843F6F3F710510F06FEF70E0709341040D
:1046D000609340040C94492C80E50E943440811181
:1046E00006C010924104109240040C94492C0E9480
:1046F000843F672B11F00C94492CF3CF8CE40E947B
:10470000EB3F882381F00E94B43F6B017C0120E0E5
:1047100030E0A9010E94F1F587FF0BC0F7FAF09491
:10472000F7F8F09406C0C12CD12C80E8E82E80E484
:10473000F82EF7FAF094F7F8F094CCA2DDA2EEA2EE
:10474000FFA280E090E0A0EAB0E489839A83AB8383
:10475000BC8380E090E0ADE4B3E48D839E83AF83BF
:10476000B88780E090E0A0EAB1E489879A87AB87B8
:10477000BC8788E50E943440882379F088E50E9450
:104780003440882319F00E94B43F03C060E070E019
:10479000CB0169837A838B839C8389E50E943440B3
:1047A000882379F089E50E943440882319F00E941B
:1047B000B43F03C060E070E0CB016D837E838F83E4
:1047C00098878AE50E943440882379F08AE50E9420
:1047D0003440882319F00E94B43F03C060E070E0C9
:1047E000CB0169877A878B879C8718A219A21AA2A6
:1047F0001BA2AE01405E5F4FBE016F5F7F4FCE01D7
:1048000084960E9446B30C94492C0E940B5A0E9435
:104810001BCB109241041092400468EE73E080E0DC
:1048200090E00E9480610E94092D0C94492C2093F5
:1048300034040C94492C83E50E9434408823A1F071
:104840000E94B43F20E030E04AE754E40E94B3EF16
:104850000E9414F560932A0270932B0280932C021D
:1048600090932D020C94492C88E50E94EB3F811116
:104870000C946E2C89E50E94EB3F81110C946E2CF8
:104880008AE50E94EB3F81110C946E2C85E40E9416
:10489000EB3F81110C946E2C0C94A02C83E50E94AC
:1048A000EB3F882309F4F5C70E94B43F20E030E0D5
:1048B0004AE754E40E94B3EF0E9414F560936D1030
:1048C00070936E1080936F1090937010E2C717E58D
:1048D000C12E12E0D12E06EFE02E00E1F02E10E006
:1048E000D6018D916D010E94EB3F882309F46DC0C4
:1048F000133009F063C00E94B43F4B015C0120E01B
:1049000030E040EA51E40E944EEF87FF4EC0A5011F
:1049100094016091021170910311809104119091A2
:1049200005110E94A7F42B013C019B01AC01609191
:104930008E0770918F0780919007909191070E9448
:10494000B3EF60938E0770938F07809390079093D7
:104950009107A30192016091AA077091AB07809122
:10496000AC079091AD070E94B3EF6093AA077093D4
:10497000AB078093AC079093AD076091F3117091F2
:10498000F4118091F5119091F6110E9452EFA3015C
:1049900092010E94B3EF0E9414F56093F31170939B
:1049A000F4118093F5119093F61180920211909278
:1049B0000311A0920411B092051107C00E94B43FE8
:1049C000F70160837183828393831F5FF4E0EF0EAE
:1049D000F11C143009F084CF0E944BCA5AC70E94C0
:1049E000CF7E83E50E943440882311F40C94001C90
:1049F0000E94843F6230710511F00C94001C0E94EB
:104A00006CC38BE50E94679A6091CB117091CC11B9
:104A10008091CD119091CE1142E00E94289E40914C
:104A2000CF115091D0116091D1117091D2118DEFB1
:104A300093E00E9461C64091D3115091D4116091CE
:104A4000D5117091D6118AEF93E00E9461C68DE571
:104A50000E94679A8AE00E94679A1BC784918F011F
:104A60000F5F1F4F882321F00E94679AF801F6CF4D
:104A700060E08FEC94E00E94726E61E088EC94E05C
:104A80000E94726E61E08DEB94E00E94726E61E0B4
:104A90008DEA94E00E94726E60E084EA94E00E94E5
:104AA000726E61E08AE994E00E94726E60E080E9D3
:104AB00094E00E94726E60E088E894E00E94726E5A
:104AC00061E08AE794E00E94726E60E08CE694E018
:104AD0000E94726E60E08DE594E00E94726E60E06C
:104AE0008FE494E00E94726E60E089E394E00E949B
:104AF000726E61E088E294E00E94726E60E083E191
:104B000094E00E94726E61E080E094E00E94726E18
:104B1000C0C6009144111091451183E0D12C40E0B2
:104B20008150E9F0D8019C91292F2B7F2134C1F7C6
:104B300011962C912133A1F7913421F0953421F471
:104B400041E002C0DD24D39498012E5F3F4F8901DC
:104B50002F5F3F4FF80190819032C9F3E1CF44239A
:104B600069F0EAE6F4E284917F012FEFE21AF20A9B
:104B7000882321F00E94679AF701F5CFDD2069F0C4
:104B8000E8EBF5E084917F014FEFE41AF40A882303
:104B900021F00E94679AF701F5CFD8018D918D0120
:104BA000882309F4AACA0E94679AF7CF0E948BD281
:104BB00070C681E08093E6058093E5056AC688ECBF
:104BC00090E00E946E9A811164C684E40E94EB3FDB
:104BD000882309F441C00E94B43F6B017C0111E0BD
:104BE00020E030E0A9010E944EEF811101C010E0E9
:104BF0001093071920E030E0A901C701B6010E9417
:104C00004EEF882349F10E94B43FE0917805B4E06B
:104C1000EB9FF0011124E45FF64E60837183828381
:104C2000938320E030E0A90160910C1970910D1977
:104C300080910E1990910F190E944EEF81110CC0B6
:104C400080E090E0A0EEBFE380930C1990930D19E3
:104C5000A0930E19B0930F190E945ACB1AC6B7E54C
:104C6000EB2EB2E0FB2E07EF11E1F70181917F01FE
:104C70000E94EB3F882351F00E94B43F0E9414F53C
:104C8000D8016D937D938D939C9313970C5F1F4F69
:104C9000B2E107301B0749F70E94DAC8FAC50C5F7A
:104CA0001F4FB7E00E3A1B0709F4F3C5F7018191D6
:104CB0007F010E94EB3F882391F30E94B43FD8010B
:104CC0006D937D938D939C931397E9CF83E50E9419
:104CD00034408823A1F00E94B43F60939A077093F8
:104CE0009B0780939C0790939D0760939607709312
:104CF0009707809398079093990710E001C011E0FF
:104D000080E50E943440882359F00E94B43F6093AC
:104D10009A0770939B0780939C0790939D0710E0E0
:104D200082E50E943440882359F00E94B43F60938A
:104D3000C0107093C1108093C2109093C31010E004
:104D400084E50E943440882359F00E94B43F609368
:104D5000960770939707809398079093990799C542
:104D6000112309F496C540919A0750919B076091D1
:104D70009C0770919D0782EC95E00E9461C640916E
:104D8000C0105091C1106091C2107091C3108FEB90
:104D900095E00E9461C640919607509197076091F7
:104DA0009807709199078CEB95E00E9461C68AE0A4
:104DB0000E94679A6EC581E50E94EB3F882351F0FF
:104DC0000E9475996093AE077093AF078093B00708
:104DD0009093B10783E50E94EB3F882351F00E9436
:104DE000B43F6093B6077093B7078093B80790936A
:104DF000B90784E50E94EB3F882351F00E94B43F3D
:104E00006093B2077093B3078093B4079093B5078C
:104E100088E50E94EB3F882351F00E94B43F6093E5
:104E2000820770938307809384079093850789E5B1
:104E30000E94EB3F882351F00E94B43F60938607A5
:104E40007093870780938807909389078AE50E946B
:104E5000EB3F8823F1F00E94B43F60938A07709380
:104E60008B0780938C0790938D072DEC3CEC4CECDA
:104E70005DE30E944EEF181664F0E2EDF5E08491D8
:104E80008F010F5F1F4F882321F00E94679AF8015E
:104E9000F6CF85E40E94EB3F882309F4FAC40E9410
:104EA000B43F60938E0770938F0780939007909321
:104EB0009107EFC41F5FB4E0EB0EF11C133011F447
:104EC0000C94001CF60181916F010E94EB3F882336
:104ED00089F30E94B43FD7016D937D938D939C938A
:104EE0001397812F0E94EE98E5CF0E9433B781116E
:104EF000D0C405E515E2ECE4F4E0F9A7E8A7AE01BB
:104F00004F5F5F4F4A017EEAA72E75E2B72E1A0166
:104F1000F8016591759185919491A8A5B9A5CD9059
:104F2000DD90ED90FD90B9A7A8A7A70196010E947A
:104F3000CAF32B013C01F101608371838283938367
:104F400020E030E040EA51EC0E94F1F587FD0AC014
:104F500020E030E040EA51E4C301B2010E944EEF8C
:104F600018162CF4F501849118160CF4ECC4D10138
:104F7000CD90DD90ED90FD901D0120E030E040EA05
:104F800051ECC701B6010E94F1F587FD0AC020E08F
:104F900030E040EA51E4C701B6010E944EEF181616
:104FA0004CF5E5E5F4E284918F010F5F1F4F81110D
:104FB00003C0E4E0F6E004C00E94679AF801F3CF72
:104FC00084918F010F5F1F4F882321F00E94679A01
:104FD000F801F6CF88E290E099A388A388EC90E0EE
:104FE0009DA38CA3BE01605E7F4FCE0184960E947C
:104FF00030B84FC40C5F1F4FBFEFAB1ABB0AE1E6DE
:10500000F5E2E017F10709F083CF67EEE62E65E0E1
:10501000F62E10E0F40181919191A191B1914F018F
:10502000F70181939193A193B1937F01812F0E9406
:10503000EE981F5F133071F70E94E07E83E992E0E3
:105040009DA38CA304E610E019A308A3BE016C5D28
:105050007F4FCE0180960E9430B88AEB92E09DA3EC
:105060008CA319A308A3BE016C5D7F4FCE0180966F
:105070000E9430B80EC40E94946D0BC483E50E9458
:105080003440882309F405C40E94843F70930302CE
:1050900060930202FEC38DED90E00E946E9A811132
:1050A000F8C383E50E943440811103C0EAE6F4E2CC
:1050B0003AC00091780510E00E94843F000F111F54
:1050C000F801EF5AFD4F718360838091780590E07D
:1050D0007C01EE0CFF1CEE0CFF1C87010B5D1D4FCD
:1050E000880F991FFC01EF5AFD4F60817181072ED7
:1050F000000C880B990B0E9454EF2AE037ED43E235
:105100005CE30E94B3EFF701E85FF64E2081318146
:10511000428153810E94B3EFD8016D937D938D93AB
:105120009C931397B6C384918F010F5F1F4F882301
:1051300021F00E94679AF801F6CF85E40E94679AF1
:1051400080917805805D0E94679AE0917805F0E093
:10515000EE0FFF1FEF5AFD4F6081718182E296E0F2
:105160000E947EC685E20E94679A8AE00E94679A42
:1051700090C380E50E94EB3F882309F48AC30E9414
:10518000843F6B017C0183E50E943440882321F039
:105190000E94843F8B0102C00FEF1FEFC8010196F0
:1051A000039708F076C3D7FC74C38C2DEAE2F6E0CF
:1051B0009491891709F4D2C33196B6E0EA35FB071A
:1051C000B9F7CFC383E50E943440882319F00E94C9
:1051D000843F02C064E071E079A368A380E50E9487
:1051E0003440882339F00E94843F6938E3E17E0728
:1051F00030F402C068EE73E07A83698304C088E803
:1052000093E19A838983BE01605E7F4FCE01019650
:105210000E9430B83EC385E40E943440811110C022
:1052200080E50E94EB3F882391F00E94B43F609399
:10523000650570936605809367059093680507C0C0
:105240000E94943F882361F3E5E5F4E271C089E4AC
:105250000E94EB3F882381F00E94B43F2CEA35EC9A
:1052600047E25EE30E94B3EF6093610570936205CD
:10527000809363059093640584E40E94EB3F882348
:1052800081F00E94B43F2CEA35EC47E25EE30E94D5
:10529000A7F46093690570936A0580936B059093FA
:1052A0006C05EAE6F4E284918F010F5F1F4F8823BB
:1052B00021F00E94679AF801F6CF40916505509160
:1052C0006605609167057091680582E696E00E9428
:1052D00061C62CEA35EC47E25EE3609161057091AE
:1052E000620580916305909164050E94A7F4AB016B
:1052F000BC018EE596E00E9461C62CEA35EC47E2DF
:105300005EE36091690570916A0580916B059091EB
:105310006C050E94B3EFAB01BC018AE596E00E94E8
:1053200061C68AE00E94679AB4C20E94679AF80137
:1053300084918F010F5F1F4F8111F7CFE6E6F6E0F2
:1053400084918F010F5F1F4F882309F4A2C20E942E
:10535000679AF801F5CF83E50E94EB3F182F882369
:1053600071F00E94B43F0E940FF570933B0260936E
:105370003A0221E0672B09F020E02093D61080E567
:105380000E94EB3F882359F020913A0230913B0272
:10539000232B11F00E94A53F8093D6107AC21111E1
:1053A00078C2EAE6F4E284918F010F5F1F4F8823F1
:1053B00021F00E94679AF801F6CF8091D6108823D9
:1053C00019F06BE173E002C06EE173E08DE896E0E6
:1053D0000E9497C660913A0270913B028CE796E07A
:1053E0000E947EC6E8E7F6E084918F010F5F1F4FB1
:1053F000882309F44EC20E94679AF801F5CF0E94F3
:105400001D6847C280E50E94EB3F882351F00E944F
:10541000B43F60935D0570935E0580935F05909344
:10542000600589E40E94EB3F882381F00E94B43F2D
:105430002CEA35EC47E25EE30E94B3EF6093590536
:1054400070935A0580935B0590935C0584E40E94F9
:10545000EB3F882381F00E94B43F2CEA35EC47E211
:105460005EE30E94A7F46093550570935605809300
:10547000570590935805EAE6F4E284918F010F5F97
:105480001F4F882321F00E94679AF801F6CF4091C0
:105490005D0550915E0560915F057091600588EA39
:1054A00096E00E9461C62CEA35EC47E25EE360912B
:1054B000590570915A0580915B0590915C050E9499
:1054C000A7F4AB01BC0184EA96E00E9461C62CEA15
:1054D00035EC47E25EE36091550570915605809189
:1054E0005705909158050E94B3EFAB01BC0180EACB
:1054F00096E00E9461C68AE00E94679ACAC10E9433
:10550000679AF80184918F010F5F1F4F8111F7CFC8
:10551000ECEAF6E084918F010F5F1F4F882309F4B6
:10552000B8C10E94679AF801F5CF0E941966B1C10F
:105530000E941690AEC10E94A4D7ABC183E50E9421
:10554000EB3F882321F00E94A53F91E089270E942C
:10555000C1D29FC181E08093CC070E94CF89109275
:10556000CC07882309F495C1EAE6F4E284918F011F
:105570000F5F1F4F811103C0EBEBF6E004C00E94E8
:10558000679AF801F3CF84918F010F5F1F4F882333
:1055900009F47FC10E94679AF801F5CF8091DC0A77
:1055A000882309F476C181E08093DF0A72C18BE51C
:1055B00092E00E946E9A81116CC185E50E94EB3FDA
:1055C0008823D9F10091780510E00E94B43F6B0167
:1055D0007C0120E030E0A9010E94F1F587FF04C0C2
:1055E000F7FAF094F7F8F094000F111F000F111F55
:1055F000F801E75EF64EC082D182E282F38200912A
:105600007805F4E00F9F80011124075E164E20E01C
:1056100030E046E154E4D8016D917D918D919C91EB
:105620000E94F1F518164CF480E090E0A6E1B4E495
:10563000F80180839183A283B3838CE40E94EB3FC3
:10564000882309F426C10091780510E00E94B43F38
:105650006B017C0120E030E0A9010E94F1F587FF99
:1056600004C0F7FAF094F7F8F094000F111F000F40
:10567000111FF801E35EF64EC082D182E282F3820E
:1056800000917805F4E00F9F80011124035E164E0F
:1056900020E030E046E154E4D8016D917D918D9198
:1056A0009C910E94F1F518160CF0F3C080E090E098
:1056B000A6E1B4E4F80180839183A283B383E9C0B7
:1056C0008AE50E943440811103C0E9ECF6E00BC08A
:1056D0000E94B43F6093211970932219809323197B
:1056E00090932419D6C084918F010F5F1F4F882398
:1056F00021F00E94679AF801F6CF4091211950914C
:105700002219609123197091241986EC96E00E9469
:1057100061C68AE00E94679ABCC08BE40E94344054
:10572000811103C0EAE6F4E236C08BE40E94344003
:105730008823C1F00E94B43F6B017C0120E030E07F
:10574000A9010E94F1F587FD0AC020E030E040E2A7
:1057500051E4C701B6010E944EEF181634F4E8EE8A
:10576000F6E00EC0C12CD12C76010E94CF7EC092F3
:105770009207D0929307E0929407F092950789C020
:1057800084918F010F5F1F4F882309F482C00E940C
:10579000679AF801F5CF84918F010F5F1F4F88231F
:1057A00021F00E94679AF801F6CF4091920750913C
:1057B0009307609194077091950787E097E00E94A6
:1057C00061C68AE00E94679A64C081E080931902F2
:1057D00083E50E943440882339F00E94A53F81115F
:1057E00058C00E94A2C355C083E50E94EB3FF7CF8B
:1057F0000E94CEB94EC0F09046110E94CF7E10910B
:10580000E01080E00E944085FF2029F1EAE6F4E202
:1058100084918F010F5F1F4F882321F00E94679AA8
:10582000F801F6CF84E50E94679A6F2D70E080E062
:1058300090E04AE00E94A39D80E20E94679AE4E221
:10584000F7E084918F010F5F1F4F882311F10E94B1
:10585000679AF801F6CF10928E10812F0E94408532
:10586000EAE6F4E284918F010F5F1F4F882321F055
:105870000E94679AF801F6CF60918E1070E082E185
:1058800097E00E947EC68AE00E94679A02C00E944A
:10589000CEB91092C5100E9485C3A1C00E94958305
:1058A0000E9492BFF6CF11110C94311F0C942A1F45
:1058B00080E00E946EAE0C94601F0E94843FAB019A
:1058C000BC014093560D5093570D6093580D709343
:1058D000590D85EA9CE00E94CFA4DBCF0E94CF7EC9
:1058E00088E50E94EB3F882331F05F9A80913F0466
:1058F0008E7F80933F0489E50E94EB3F882339F037
:105900008A9A479A80913F048D7F80933F048AE56D
:105910000E94EB3F882361F080910801809581709F
:1059200080930601479A80913F048B7F80933F04C8
:1059300085E40E94EB3F882309F4ABCF129AA9CFEC
:105940000E941BCBA6CFF7FAF094F7F8F094D101A0
:10595000CD92DD92ED92FC92139709CB0E94ABE8B9
:1059600098CF0E94CF7EBC2C60E08C2D0E9441BA63
:105970000F3FBFEF1B0759F48C2D0E94EBB931E0AC
:1059800020E0892B09F030E0032F122F05C00130F1
:10599000110569F401E010E08B2D0E94EBB980172E
:1059A000910709F476CF80E00E946EAEF5CF00E05B
:1059B00010E0F2CF61E0812F0E9441BA6E2D812F5D
:1059C0000E9413BAF12CB701812F0E947DBA1930C1
:1059D00009F05FCFF0924104E09240045ACFCD5BD2
:1059E000DF4F0FB6F894DEBF0FBECDBFDF91CF9172
:1059F0001F910F91FF90EF90DF90CF90BF90AF90ED
:105A00009F908F907F906F905F904F903F902F90DE
:105A100008952F923F924F925F926F927F928F9252
:105A20009F92AF92BF92CF92DF92EF92FF920F932D
:105A30001F93CF93DF93CDB7DEB76F970FB6F89470
:105A4000DEBF0FBECDBFC0905C04D0905D04E0907F
:105A50005E04F0905F0420E030E040EA50E4C701CB
:105A6000B6010E944EEF87FD43C120E030E041E9DE
:105A700053E4C701B6010E94F1F518160CF438C1C1
:105A80001092F90E1092F80E809109014091F70ED4
:105A9000042E000C550B817021E0822790E04817FE
:105AA000590709F433C08091090181702827209398
:105AB000F70E81111BC00E94F99FEBEFFDE084916E
:105AC0008F01882351F0082E000C990B0E94F49F3F
:105AD0000F5F1F4FF8018491F4CF8DE090E00E949A
:105AE000F49F8AE090E00E94F49F10C0EFEFFDE089
:105AF00084918F01882389F3082E000C990B0E9452
:105B0000F49F0F5F1F4FF8018491F4CF8091EA0E4C
:105B1000833009F44CC02CF4882351F08130D9F043
:105B20009CC0843009F43EC0853009F44DC095C056
:105B30008091DC0A882309F490C081E08093EA0E0A
:105B40000E9467626093EE0E7093EF0E8093F00EEA
:105B50009093F10E82C08091DC0A81117EC0809109
:105B6000A80C882321F082E08093EA0E76C0109280
:105B7000EA0EE7EFFDE084918F01882351F0082EB3
:105B8000000C990B0E94F49F0F5F1F4FF801849146
:105B9000F4CF8DE090E00E94F49F8AE090E00E94B4
:105BA000F49F5BC08091370F8823E9F256C0809143
:105BB000DC0A811152C080915E0A90915F0A891BB4
:105BC0008F7009F4C0C049C08091DC0A811145C0C2
:105BD00080915E0A90915F0A891B8F7009F4CDC095
:105BE0003CC08DE090E00E94F49F8AE090E00E942B
:105BF000F49F1092EA0EC0905404D0905504E090A7
:105C00005604F090570420E030E048E453E4C70124
:105C1000B6010E94F1F587FDC1C08BEE9DE0909327
:105C20004B0480934A040E94CF9A80EE9DE09093AB
:105C30004B0480934A040E94CF9A8CED9DE0909390
:105C40004B0480934A040E94CF9A8DE99DE0909383
:105C50004B0480934A040E94CF9A8091DF0E90916A
:105C6000E00E03974CF571E9272E79E0372EE0E638
:105C70008E2EEAEE9E2EA12CB12C85E490E10E949E
:105C8000883E18161906C4F48091DF0E9091E00E3C
:105C9000049794F485E490E10E944C3E8093E50ED5
:105CA000E091E60EF091E70E8A3019F08D3009F0A0
:105CB000CCC0309709F0D2C08091DF0E9091E00EF9
:105CC000009711F40C94A93D01979093E00E8093F6
:105CD000DF0E8091E10E9091E20E019664E070E09B
:105CE0000E94B4F69093E20E8093E10E0C94A93DCD
:105CF0008091F80E9091F90E8136FAEE9F07E8F048
:105D00001092F90E1092F80EE3E0FEE084918F01FC
:105D1000882351F0082E000C990B0E94F49F0F5F0E
:105D20001F4FF8018491F4CF8DE090E00E94F49F22
:105D30008AE090E00E94F49FA7CE01969093F90E1E
:105D40008093F80EA1CE8091370F882311F082E066
:105D500001C084E08093EA0EE3EFFDE084918F01BF
:105D6000882309F416CF082E000C990B0E94F49F8B
:105D70000F5F1F4FF8018491F3CFEFEEFDE08491A8
:105D80008F01882309F42DCF082E000C990B0E9457
:105D9000F49F0F5F1F4FF8018491F3CF20E030E0B4
:105DA00048E453E4C701B6010E944EEF87FF13C0D9
:105DB00088ED9DE090934B0480934A040E94CF9A13
:105DC0008DEC9DE090934B0480934A040E94CF9AFF
:105DD00089EC9DE034CF20E030E04EE353E4C7018E
:105DE000B6010E944EEF87FF13C085EC9DE09093B3
:105DF0004B0480934A040E94CF9A89EB9DE09093D4
:105E00004B0480934A040E94CF9A85EB9DE017CF04
:105E100020E030E046E153E4C701B6010E944EEFB6
:105E200087FF13CF81EB9DE090934B0480934A044E
:105E30000E94CF9A85EA9DE090934B0480934A0498
:105E40000E94CF9A81EA9DE0FACE8A3309F431CFDD
:105E5000EF35F10514F40C942B3B2BCF8091E30E1E
:105E60009091E40E20E6289F7001299FF00C1124E8
:105E70008701015A124FE00FF11F108261E470E0B8
:105E8000C8010E941BF7009711F40C940F3B9093EC
:105E9000E90E8093E80E801B910B8E0D9F1D60E034
:105EA00070E0805A924F0E944FEB0E940FF5CB0199
:105EB000770FAA0BBB0B8232910510F00C940F3BAD
:105EC000FC018827EE58FF4F8F4F0C94C7F6E8E986
:105ED000FDE084918F01882351F0082E000C990B6E
:105EE0000E94F49F0F5F1F4FF8018491F4CF20E0D0
:105EF00030E040E05FE360915C0470915D0480916C
:105F00005E0490915F041EC0E3E9FDE084918F017F
:105F1000882351F0082E000C990B0E94F49F0F5F0C
:105F20001F4FF8018491F4CF6091480470914904A7
:105F3000072E000C880B990B0E9454EF20E030E0F4
:105F400040E05FE30E94CBF30E940FF5CB010E947B
:105F50008D410E94BEE08DE090E00E94F49F8AE0B7
:105F600090E00E94F49F0C940F3BEEE8FDE08491DA
:105F70008F01882351F0082E000C990B0E94F49F8A
:105F80000F5F1F4FF8018491F4CF20E030E040E034
:105F90005FE36091440470914504809146049091C0
:105FA0004704D0CFE9E8FDE084918F01882351F0C8
:105FB000082E000C990B0E94F49F0F5F1F4FF801F1
:105FC0008491F4CF6091420470914304B1CF209149
:105FD00040043091410444E6429FC001439F900D2C
:105FE00011246FEF70E00E94B4F68B0165367105E5
:105FF00010F004E610E0E4E8FDE084917F018823DE
:1060000059F0082E000C990B0E94F49FFFEFEF1A35
:10601000FF0AF7018491F3CFB80180E090E098C7C0
:10602000E0E8FDE084918F01882351F0082E000CF8
:10603000990B0E94F49F0F5F1F4FF8018491F4CFDA
:1060400080E290E00E94F49FECE7FDE084918F01F4
:10605000882351F0082E000C990B0E94F49F0F5FCB
:106060001F4FF8018491F4CF60914C0470914D045E
:1060700080914E0490914F040E94BFE080E290E036
:106080000E94F49FE8E7FDE084918F01882351F09E
:10609000082E000C990B0E94F49F0F5F1F4FF80110
:1060A0008491F4CF60915004709151048091520416
:1060B000909153040E94BFE080E290E00E94F49F20
:1060C000E4E7FDE084918F01882351F0082E000C55
:1060D000990B0E94F49F0F5F1F4FF8018491F4CF3A
:1060E0006091540470915504809156049091570426
:1060F0000E94BFE080E290E003C68091DC0A882322
:1061000009F450C0EFE6FDE084918F01882351F03F
:10611000082E000C990B0E94F49F0F5F1F4FF8018F
:106120008491F4CF8091DD0A882359F18091A80CE5
:10613000882329F18091520D9091530DA091540D17
:10614000B091550D0097A105B105C1F0BC01CD017D
:106150006D597F4F8F4F9F4F24E630E040E050E075
:106160000E946DF36091560D7091570D8091580DFE
:106170009091590D0E946DF3822F01C080E090E054
:10618000E6CEEBE6FDE084918F01882309F4E3CEAF
:10619000082E000C990B0E94F49F0F5F1F4FF8010F
:1061A0008491F3CFE3E6FDE084918F01882309F425
:1061B000D2CE082E000C990B0E94F49F0F5F1F4F48
:1061C000F8018491F3CFEEE5FDE084918F018823FF
:1061D00051F0082E000C990B0E94F49F0F5F1F4F87
:1061E000F8018491F4CF8091EE0E9091EF0EA09182
:1061F000F00EB091F10E892B8A2B8B2B09F477C00E
:106200000E946762A50194010E946DF369017A0101
:106210006091EE0E7091EF0E8091F00E9091F10E64
:10622000A50194010E946DF38601021B130BC801A6
:106230006CE370E00E94A0F6CB019927EAE0F0E061
:10624000BF010E94B4F6282FCB01BF010E94B4F613
:10625000805D80933704205D2093380410923904C8
:1062600087E394E00E94BEE080E290E00E94F49F09
:10627000ECE5FDE084917F01882359F0082E000CA5
:10628000990B0E94F49FFFEFEF1AFF0AF701849128
:10629000F3CF80E290E00E94F49FC8016CE370E0CD
:1062A0000E94A0F66AE070E00E94B4F6605D609320
:1062B0003704805D809338041092390487E394E0BA
:1062C0000E94BEE080E290E00E94F49FEAE5FDE0DB
:1062D00084918F01882309F43ECE082E000C990B7F
:1062E0000E94F49F0F5F1F4FF8018491F3CF80E26B
:1062F00090E00E94F49FE2E5FDE084918F01882305
:1063000009F429CE082E000C990B0E94F49F0F5F10
:106310001F4FF8018491F3CF1092180F809109015B
:1063200080FF11C0EEE4FDE084918F01882309F421
:1063300012CE082E000C990B0E94F49F0F5F1F4F86
:10634000F8018491F3CF83E50E9454E0882341F063
:106350000E946FE00E9414F57093ED0E6093EC0EB6
:10636000EAE4FDE084918F01882351F0082E000CAF
:10637000990B0E94F49F0F5F1F4FF8018491F4CF97
:106380008DE090E00E94F49F8AE090E00E94F49FEC
:106390008091360F882309F4A1C28091EC0E909170
:1063A000ED0E8430910509F4D2C040F4892B09F038
:1063B0003BC4EEE6FBE084918F010CC08830910570
:1063C00009F47EC10C9709F02FC4E0EFF9E0849145
:1063D0008F012FC2882351F0082E000C990B0E94C8
:1063E000F49F0F5F1F4FF8018491F4CF8DE090E090
:1063F0000E94F49F8AE090E00E94F49FE3E6FBE0B5
:1064000084918F01882351F0082E000C990B0E9473
:10641000F49F0F5F1F4FF8018491F4CF8DE090E05F
:106420000E94F49F8AE090E00E94F49FE7E5FBE081
:1064300084918F01882351F0082E000C990B0E9443
:10644000F49F0F5F1F4FF8018491F4CF8DE090E02F
:106450000E94F49F8AE090E00E94F49FEBE4FBE04E
:1064600084918F01882351F0082E000C990B0E9413
:10647000F49F0F5F1F4FF8018491F4CF8DE090E0FF
:106480000E94F49F8AE090E00E94F49FEDE3FBE01D
:1064900084918F01882351F0082E000C990B0E94E3
:1064A000F49F0F5F1F4FF8018491F4CF8DE090E0CF
:1064B0000E94F49F8AE090E00E94F49FEFE2FBE0EC
:1064C00084918F01882351F0082E000C990B0E94B3
:1064D000F49F0F5F1F4FF8018491F4CF8DE090E09F
:1064E0000E94F49F8AE090E00E94F49FE2E2FBE0C9
:1064F00084918F01882351F0082E000C990B0E9483
:10650000F49F0F5F1F4FF8018491F4CF8DE090E06E
:106510000E94F49F8AE090E00E94F49FE5E1FBE096
:1065200084918F01882351F0082E000C990B0E9452
:10653000F49F0F5F1F4FF8018491F4CF8DE090E03E
:106540000E94F49F8AE090E00E94F49F6DC3E7E010
:10655000FBE084918F01882351F0082E000C990BE9
:106560000E94F49F0F5F1F4FF8018491F4CF8DE0DC
:1065700090E00E94F49F8AE090E00E94F49FE9EF8F
:10658000FAE084918F01882351F0082E000C990BBA
:106590000E94F49F0F5F1F4FF8018491F4CF8DE0AC
:1065A00090E00E94F49F8AE090E00E94F49FE3EE66
:1065B000FAE084918F01882351F0082E000C990B8A
:1065C0000E94F49F0F5F1F4FF8018491F4CF8DE07C
:1065D00090E00E94F49F8AE090E00E94F49FEDEC2E
:1065E000FAE084918F01882351F0082E000C990B5A
:1065F0000E94F49F0F5F1F4FF8018491F4CF8DE04C
:1066000090E00E94F49F8AE090E00E94F49FEBEB00
:10661000FAE084918F01882351F0082E000C990B29
:106620000E94F49F0F5F1F4FF8018491F4CF8DE01B
:1066300090E00E94F49F8AE090E00E94F49FE9EAD3
:10664000FAE084918F01882351F0082E000C990BF9
:106650000E94F49F0F5F1F4FF8018491F4CF8DE0EB
:1066600090E00E94F49F8AE090E00E94F49FEBE9A2
:10667000FAE084918F01882351F0082E000C990BC9
:106680000E94F49F0F5F1F4FF8018491F4CF8DE0BB
:1066900090E00E94F49F8AE090E00E94F49FEDE871
:1066A000FAE084918F01882309F448CF082E000C6A
:1066B000990B0E94F49F0F5F1F4FF8018491F3CF55
:1066C000E6E8FAE084918F01882351F0082E000C4F
:1066D000990B0E94F49F0F5F1F4FF8018491F4CF34
:1066E0008DE090E00E94F49F8AE090E00E94F49F89
:1066F000EFE7FAE084918F01882351F0082E000C17
:10670000990B0E94F49F0F5F1F4FF8018491F4CF03
:106710008DE090E00E94F49F8AE090E00E94F49F58
:10672000E8E6FAE084918F01882351F0082E000CEE
:10673000990B0E94F49F0F5F1F4FF8018491F4CFD3
:106740008DE090E00E94F49F8AE090E00E94F49F28
:10675000E1E5FAE084918F01882351F0082E000CC6
:10676000990B0E94F49F0F5F1F4FF8018491F4CFA3
:106770008DE090E00E94F49F8AE090E00E94F49FF8
:10678000EAE3FAE084918F01882351F0082E000C8F
:10679000990B0E94F49F0F5F1F4FF8018491F4CF73
:1067A0008DE090E00E94F49F8AE090E00E94F49FC8
:1067B000E3E2FAE084918F01882351F0082E000C67
:1067C000990B0E94F49F0F5F1F4FF8018491F4CF43
:1067D0008DE090E00E94F49F8AE090E00E94F49F98
:1067E000E0E1FAE084918F01882351F0082E000C3B
:1067F000990B0E94F49F0F5F1F4FF8018491F4CF13
:106800008DE090E00E94F49F8AE090E00E94F49F67
:10681000EDEFF9E084918F01882309F48FCE082EE3
:10682000000C990B0E94F49F0F5F1F4FF801849199
:10683000F3CF882351F0082E000C990B0E94F49F8F
:106840000F5F1F4FF8018491F4CF8DE090E00E941C
:10685000F49F8AE090E00E94F49FE3EEF9E08491D7
:106860008F01882351F0082E000C990B0E94F49F91
:106870000F5F1F4FF8018491F4CF8DE090E00E94EC
:10688000F49F8AE090E00E94F49FE5EDF9E08491A6
:106890008F01882351F0082E000C990B0E94F49F61
:1068A0000F5F1F4FF8018491F4CF8DE090E00E94BC
:1068B000F49F8AE090E00E94F49FE7ECF9E0849175
:1068C0008F01882309F43ACE082E000C990B0E9400
:1068D000F49F0F5F1F4FF8018491F3CF8091DD0A81
:1068E000882309F478C181E080935A0D10925C0DE1
:1068F00010925B0D8CE29BE00E9416A78BE1ECE20C
:10690000FBE0DE01159601900D928A95E1F78091EA
:106910002A0B90912B0B9C838B838DEE92E09A83B4
:10692000898340E050E0BE016F5F7F4F80E090E0E0
:106930000E94F5A1CE0101960E9404AEC0905B0DAD
:10694000D0905C0D0091EC0E1091ED0EC601801BF5
:10695000910B049720F06801F3E0CF0ED11C58EBA7
:10696000452E59E0552E69EA662E69E0762EC0164E
:10697000D10608F459C10115110509F09DC060EE5A
:106980007AE08CE29BE00E94DEA562E273E080EE9A
:106990009AE00E9426F7892B09F048C0F201849101
:1069A00048EBE42E49E0F42E882359F0082E000C21
:1069B000990B0E94F49FFFEFEF1AFF0AF7018491F1
:1069C000F3CF8DE090E00E94F49F8AE090E00E9477
:1069D000F49FF301849139EAE32E39E0F32E882302
:1069E00059F0082E000C990B0E94F49FFFEFEF1A4C
:1069F000FF0AF7018491F3CF8DE090E00E94F49FAD
:106A00008AE090E00E94F49F80E090E00E94B8E06D
:106A1000E9E9F9E084917F012FEFE21AF20A882375
:106A200009F4D6C00E94679AF701F4CFE5E9F9E0CE
:106A300084917F01882359F0082E000C990B0E9445
:106A4000F49FFFEFEF1AFF0AF7018491F3CF8DE077
:106A500090E00E94F49F8AE090E00E94F49FF10190
:106A6000849121E9E22E29E0F22E882359F0082EA4
:106A7000000C990B0E94F49FFFEFEF1AFF0AF70139
:106A80008491F3CF8DE090E00E94F49F8AE090E043
:106A90000E94F49F80E090E00E94B8E0ECE8F9E00A
:106AA00084917F012FEFE21AF20A882309F490C043
:106AB0000E94679AF701F4CF60E070E0C801019787
:106AC0000E94BAA38091DE0A882309F45AC0EAE83A
:106AD000F9E084917F01882359F0082E000C990B6E
:106AE0000E94F49FFFEFEF1AFF0AF7018491F3CFA2
:106AF00080EE9AE00E94BEE08DE090E00E94F49F5C
:106B00008AE090E00E94F49FE8E8F9E084917F0138
:106B1000882359F0082E000C990B0E94F49FFFEF78
:106B2000EF1AFF0AF7018491F3CF8DEE9AE00E94ED
:106B3000BEE08DE090E00E94F49F8AE090E00E9429
:106B4000F49FC8010E94B8E0E6E8F9E084917F0173
:106B50002FEFE21AF20A882321F00E94679AF701C8
:106B6000F5CF9DEEE92E9AE0F92EF70181917F0194
:106B7000882319F00E94679AF8CF8AE00E94679AEA
:106B800027C080EE9AE00E94BEE08DE090E00E9477
:106B9000F49F8AE090E00E94F49F8DEE9AE00E94BC
:106BA000BEE08DE090E00E94F49F8AE090E00E94B9
:106BB000F49FC8010E94B8E08DEEE82E8AE0F82E1E
:106BC000F70181917F018823C1F20E94679AF8CF73
:106BD0000F5F1F4FCCCEE7E7F9E084918F01882348
:106BE00051F0082E000C990B0E94F49F0F5F1F4F6D
:106BF000F8018491F4CF8DE090E00E94F49F8AE048
:106C000090E00E94F49FE8E6F9E084918F018823E8
:106C100009F494CC082E000C990B0E94F49F0F5F8E
:106C20001F4FF8018491F3CFE6E4FDE084918F01DA
:106C3000882309F490C9082E000C990B0E94F49F38
:106C40000F5F1F4FF8018491F3CF8091DC0A8823F6
:106C500039F00E9428A1E3C48091DC0A882379F1ED
:106C60000E94C9B4DCC48091EA0E823019F08336E8
:106C700009F0D5C40E9467626093EE0E7093EF0E28
:106C80008093F00E9093F10E8091DD0A882319F025
:106C900081E08093DC0A81E08093EA0EE2E4FDE08B
:106CA00084918F01882309F456C9082E000C990B92
:106CB0000E94F49F0F5F1F4FF8018491F3CF8091E2
:106CC000EA0E833609F0ABC4CBCF89E39DE00E9486
:106CD00027AE80915E0A90915F0A891B8F7009F040
:106CE0009EC48091EA0E823009F499C4833609F07B
:106CF000CAC495C48DE090E00E94F49F8AE090E0C1
:106D00000E94F49F28C980915E0A90915F0A891BB6
:106D10008F7009F084C48091EA0E823009F47FC438
:106D2000833609F47CC48091A80C811100C577C416
:106D300083E50E9454E0811126C083E40E9454E060
:106D4000882309F46CC480915E0A90915F0A891BC4
:106D50008F7009F064C420E030E040E251E46091BB
:106D600054047091550480915604909157040E94E8
:106D70004EEF87FF08C086E29DE090934B0480931E
:106D80004A040E94CF9A0E946FE020E030E0A901FF
:106D90000E944EEF87FD10C00E946FE020E030E8B7
:106DA00049E853E40E94F1F518164CF00E946FE098
:106DB0000E9414F5CB0105C080E090E002C083E1A1
:106DC00091E00E94FB592BC483E50E9454E0882384
:106DD00009F425C40E946FE020E030E0A9010E9480
:106DE0004EEF87FD10C00E946FE020E030E046E1EA
:106DF00053E40E94F1F518164CF00E946FE00E94D7
:106E000014F5CB0105C080E090E002C086E990E077
:106E10000E94C34104C483E50E9454E08823D9F052
:106E20000E946FE020E030E04FE753E40E94B3EFB0
:106E300020E030E048EC52E40E94A7F40E9414F5F0
:106E40006F3F710519F010F06FEF70E0709341041F
:106E50006093400480C88FEF90E09093410480934A
:106E6000400479C880915E0A90915F0A891B8F70F7
:106E700009F071C88091DC0A81116DC80E94E06739
:106E80005F9A80913F048E7F80933F048A9A479A4D
:106E900080913F048D7F80933F048091080180950D
:106EA000817080930601479A80913F048B7F809385
:106EB0003F04129A50C883E50E9454E0882319F1D8
:106EC0000E946FE020E030E040E252E40E944EEF8A
:106ED00087FD0FC00E946FE020E030EC49E754E4EA
:106EE0000E94F1F5181644F00E946FE00E940FF521
:106EF00005C068E270E002C067EE73E070930302C1
:106F0000609302028CC3E0E2FDE084918F0188234C
:106F100051F0082E000C990B0E94F49F0F5F1F4F39
:106F2000F8018491F4CFC0900202D09003020D2C9E
:106F3000000CEE08FF08F7FE0DC06DE285E490E15D
:106F40005ED666277727CB016C197D098E099F09CC
:106F50004AE003C04AE0C701B6010E9478E00C9401
:106F6000AB2F80915E0A90915F0A891B8F7009F0A8
:106F700056C38091EA0E823009F451C3833609F07A
:106F80001CC34DC380915E0A90915F0A891B8F706C
:106F900011F00C94AB2F8091EA0E823011F40C9416
:106FA000AB2F833609F0F7C30C94AB2F80915E0AA8
:106FB00090915F0A891B8F7009F031C38091EA0EAE
:106FC000823009F42CC3833609F03BC528C3809175
:106FD0005E0A90915F0A891B8F7009F020C380912F
:106FE000EA0E823009F41BC3833609F060C517C36B
:106FF00080915E0A90915F0A891B8F7009F00FC320
:107000008091EA0E823009F40AC3833609F085C5FF
:1070100006C38091180F811103C00E94F99FF2C12D
:107020008E3271F58091190F8E3209F074C1809102
:107030007D0C882309F4E6C1815080937D0C882360
:1070400061F090E001974FE1489F9001499F300D1A
:107050001124C901895B944F02C089E09BE02BE1B8
:10706000FC013496ACE2BBE001900D922A95E1F769
:10707000FC018281938190932B0B80932A0BC2C1D8
:107080008C3309F048C164E273E088E19FE00E941C
:1070900026F7892B21F481E08093360FB3C163E397
:1070A00073E088E19FE00E9426F7892B79F4E4E4FD
:1070B000F9E084918F010F5F1F4F882321F00E9418
:1070C000679AF801F6CF87E299E012C16AE473E0AB
:1070D00088E19FE00E9426F7892B79F4E3E0F9E04C
:1070E00084918F010F5F1F4F882321F00E94679AC0
:1070F000F801F6CF80EF98E0FBC061E673E088E12D
:107100009FE00E9426F7892B79F4E5EDF8E0849161
:107110008F010F5F1F4F882321F00E94679AF801AB
:10712000F6CF80ED98E0E4C06FE673E088E19FE081
:107130000E9426F7892B79F4E0EBF8E084918F0127
:107140000F5F1F4F882321F00E94679AF801F6CF46
:107150008BEA98E0CDC062E873E088E19FE00E948E
:1071600026F7892B79F4E0E9F8E084918F010F5F2D
:107170001F4F882321F00E94679AF801F6CF87E815
:1071800098E0B6C060E973E088E19FE00E9426F7CE
:10719000892B71F404E618E0F8018491882329F022
:1071A0000F5F1F4F0E94679AF7CF8DE598E0A0C050
:1071B00066EA73E088E19FE00E9426F7892B79F464
:1071C000EEE3F8E084918F010F5F1F4F882321F0D9
:1071D0000E94679AF801F6CF87E398E089C068EBD0
:1071E00073E088E19FE00E9426F7892B79F4EFE1B4
:1071F000F8E084918F010F5F1F4F882321F00E94D8
:10720000679AF801F6CF8EE098E072C063EC73E005
:1072100088E19FE00E9426F7892B79F4E5EFF7E0FB
:1072200084918F010F5F1F4F882321F00E94679A7E
:10723000F801F6CF83EE97E05BC06FEC73E088E176
:107240009FE00E9426F7892B79F4E8ECF7E084911F
:107250008F010F5F1F4F882321F00E94679AF8016A
:10726000F6CF86EB97E044C06DED73E088E19FE0D8
:107270000E9426F7892B79F4ECE9F7E084918F01DD
:107280000F5F1F4F882321F00E94679AF801F6CF05
:107290008BE897E02DC06AEE73E088E19FE00E94E2
:1072A00026F7892B79F4E1E7F7E084918F010F5FEE
:1072B0001F4F882321F00E94679AF801F6CF8CE6D1
:1072C00097E016C067EF73E088E19FE00E9426F721
:1072D000892BA9F4E1E5F7E084918F010F5F1F4F3F
:1072E000882321F00E94679AF801F6CF8CE497E09A
:1072F00090934B0480934A040E94CF9A83C065E028
:1073000074E088E19FE00E9426F7892B09F07AC09B
:107310001092360F77C01D8218861C821B828DEE5C
:1073200092E09A83898380912F0B811103C069E0D9
:107330007BE002C068E27BE06115710519F06C5FCB
:107340007F4F02C060E070E021E048E15FE0CE01E5
:1073500005960E9445AB882361F18BE1FE013596CD
:10736000ACE2BBE001900D928A95E1F72B813C8164
:1073700030932B0B20932A0B80917D0C8A3008F0E0
:107380003DC091E0980F90937D0CFFE18F9FC0016D
:107390001124DC01A55BB44F4BE1ECE2FBE0019072
:1073A0000D924A95E1F7FC01E95BF44F33832283A8
:1073B00025C0EAE6F4E284918F010F5F1F4F882316
:1073C00021F00E94679AF801F6CFE6E3F7E0849196
:1073D0008F010F5F1F4F882321F00E94679AF801E9
:1073E000F6CF08E11FE0F80181918F01882319F0A1
:1073F0000E94679AF8CF8AE00E94679ACE010196B0
:107400000E9404AE1092180F8091090180FF07C1FD
:10741000E4E6FCE084918F01882311F40C94AB2FF7
:10742000082E000C990B0E94F49F0F5F1F4FF8016C
:107430008491F2CF8FE40E9454E081110C94AB2F21
:1074400083E40E9454E00C94AB2F83E50E9454E047
:10745000811159C08FE40E9454E0882319F08CE216
:107460009CE007C084E50E9454E0882349F084E052
:107470009CE090934B0480934A040E94CF9A43C0AF
:1074800083E40E9454E0882319F08BED9BE0F1CF58
:1074900081E50E9454E0882319F083EB9BE0E9CF5B
:1074A00088E40E9454E08823C9F0EFEAFBE084916D
:1074B0008F01882351F0082E000C990B0E94F49F35
:1074C0000F5F1F4FF8018491F4CF8DE090E00E9490
:1074D000F49F8AE090E00E94F49F15C08CE40E9423
:1074E00054E0882381F0EBEAFBE084918F0188234C
:1074F00061F3082E000C990B0E94F49F0F5F1F4F41
:10750000F8018491F4CFE3E7FCE084918F018823B4
:1075100011F40C94AB2F082E000C990B0E94F49FD1
:107520000F5F1F4FF8018491F2CF80915E0A809126
:107530005F0A0C94AB2F83E50E9454E0882309F482
:107540006EC083E89BE090934B0480934A040E94B2
:10755000CF9AE3E7FCE084918F01882311F40C9427
:10756000AB2F082E000C990B0E94F49F0F5F1F4F4A
:10757000F8018491F2CFEEE7FBE084918F0188233C
:1075800051F0082E000C990B0E94F49F0F5F1F4FC3
:10759000F8018491F4CFE9E7FBE084918F0188231F
:1075A00011F40C94AB2F082E000C990B0E94F49F41
:1075B0000F5F1F4FF8018491F2CF88E50E9454E0DD
:1075C000811106C089E50E9454E0882309F4D5C0E2
:1075D00088E50E9454E0882341F08AE19DE0909381
:1075E0004B0480934A040E94CF9A89E50E9454E09C
:1075F000882341F084E19DE090934B0480934A04FA
:107600000E94CF9A8AE50E9454E0882341F08EE0E0
:107610009DE090934B0480934A040E94CF9A8091FE
:10762000E30E9091E40E019664E070E00E94B4F6DF
:107630009093E40E8093E30E8091DF0E9091E00E24
:1076400001969093E00E8093DF0E1092E70E109259
:10765000E60E0C943D2E4091E30E5091E40E9F01F6
:107660002F5F3F4F3093E70E2093E60E90E6949FF6
:107670009001959F300D1124215A324FE20FF31FD4
:1076800080830C943D2E0091E80E1091E90E780154
:1076900024E0E20EF11C6AE270E0C7010E941BF7D1
:1076A000F80124812F3221F4B8016B5F7F4F03C0B2
:1076B0002C3339F4B70188E19FE00E942FF70C9436
:1076C000AB2F1092180F009719F0FC013197108220
:1076D0008091E80E9091E90E40E061E004960E94EE
:1076E00082DE8091A80C882389F0E5E3FDE0849197
:1076F0008F01882309F4FECA082E000C990B0E9402
:10770000F49F0F5F1F4FF8018491F3CFE1E3FDE099
:1077100084918F01882309F4EDCA082E000C990B7F
:107720000E94F49F0F5F1F4FF8018491F3CF0E94D6
:1077300067626093EE0E7093EF0E8093F00E90935D
:10774000F10E8091DD0A882319F081E08093DC0A34
:1077500081E08093EA0EEDE2FDE084918F018823C1
:1077600011F40C94AB2F082E000C990B0E94F49F7F
:107770000F5F1F4FF8018491F2CF8AE50E9454E019
:10778000811126CF83E40E9454E0882309F447CF77
:107790008AE09DE03ECF86E40E9454E0882309F40D
:1077A0004DC10E946FE00E9414F58B0186E09DE0C0
:1077B00090934B0480934A040E94CF9A88E50E94DC
:1077C00054E0882309F451C00E946FE02B013C0172
:1077D0002DEC3CEC4CE45EE30E944EEF9E012F5FEB
:1077E0003F4F7901181674F020E030E0A901C30181
:1077F000B2010E94F1F518162CF41F930F938BEF32
:107800009CE005C12DEC3CEC4CEC5DEBC301B201FE
:107810000E944EEF18167CF020E030E040E85FEB6D
:10782000C301B2010E94F1F518162CF41F930F93B7
:107830008FEE9CE0ECC01F930F93C301B2010E9436
:107840000FF57F936F9385EE9CE09F938F93FF924C
:10785000EF920E9420EF0FB6F894DEBF0FBECDBFAF
:10786000CE0101960E94AA9ADFC089E50E9454E0E9
:10787000882309F441C00E946FE02B013C012DECEC
:107880003CEC4CE45EE30E944EEFFE0131967F013A
:10789000181674F020E030E0A901C301B2010E9483
:1078A000F1F518162CF41F930F938AED9CE0AFC0EE
:1078B0002DEC3CEC4CEC5DEBC301B2010E944EEFB1
:1078C00018167CF020E030E040E85FEBC301B20125
:1078D0000E94F1F518162CF41F930F938EEC9CE088
:1078E00096C01F930F93C301B2010E940FF57F93BF
:1078F0006F9384EC9CE0A9CF8AE50E9454E0882332
:1079000009F441C00E946FE02B013C012DEC3CECDE
:107910004CE45EE30E944EEFFE0131967F011816A3
:1079200074F020E030E0A901C301B2010E94F1F53A
:1079300018162CF41F930F9389EB9CE068C02DEC74
:107940003CEC4CEC5DEBC301B2010E944EEF18160B
:107950007CF020E030E040E85FEBC301B2010E9420
:10796000F1F518162CF41F930F938DEA9CE04FC08D
:107970001F930F93C301B2010E940FF57F936F9382
:1079800083EA9CE062CF85E40E9454E0882309F4F6
:107990004BC00E946FE02B013C012DEC3CEC4CE411
:1079A0005EE30E944EEFFE0131967F01181674F0DF
:1079B00020E030E0A901C301B2010E94F1F51816E0
:1079C0002CF41F930F9388E99CE021C02DEC3CEC34
:1079D0004CEC5DEBC301B2010E944EEF18167CF037
:1079E00020E030E040E85FEBC301B2010E94F1F516
:1079F00018162CF41F930F938CE89CE008C0C30169
:107A0000B2010E940FF57F936F9381E89CE09F93F2
:107A10008F93FF92EF920E9420EF0F900F900F90A4
:107A20000F900F900F901CCF8DE79CE090934B042C
:107A300080934A040E94CF9A0C94AB2F00E010E090
:107A4000B5CE20E030E040E251E460915404709102
:107A5000550480915604909157040E944EEF87FF81
:107A600008C086E79CE090934B0480934A040E94F0
:107A7000CF9A82E390E090934304809342040E9463
:107A8000635988EC90E00E94FB59E3E7FCE08491A5
:107A90008F01882311F40C94AB2F082E000C990B46
:107AA0000E94F49F0F5F1F4FF8018491F2CF20E0F6
:107AB00030E040E251E460915404709155048091AB
:107AC0005604909157040E944EEF87FF08C08CE641
:107AD0009CE090934B0480934A040E94CF9A80E5E7
:107AE00090E090934304809342040E94635980EF96
:107AF00090E00E94FB59E3E7FCE084918F0188232A
:107B000011F40C94AB2F082E000C990B0E94F49FDB
:107B10000F5F1F4FF8018491F2CF80E090E00E9448
:107B2000FB5910924304109242040E946359E8E604
:107B3000FCE084918F01882311F40C94AB2F082E64
:107B4000000C990B0E94F49F0F5F1F4FF801849166
:107B5000F2CF6F960FB6F894DEBF0FBECDBFDF91A8
:107B6000CF911F910F91FF90EF90DF90CF90BF903A
:107B7000AF909F908F907F906F905F904F903F90CD
:107B80002F900895CF92DF92EF92FF92CF93DF93E1
:107B90006B017C01EA0121E338E040EA50EC0E94ED
:107BA000F1F587FD23C022E430E047E553E4C70147
:107BB000B6010E944EEF1816CCF0C880D980EA803A
:107BC000FB802FE632E143E85AEBC701B6010E9481
:107BD000F1F587FD0BC0C1E022E430E047E553E456
:107BE000C701B6010E944EEF18160CF4C0E08C2FAE
:107BF000DF91CF91FF90EF90DF90CF9008950F939A
:107C00001F93CF93DF93FC01A685B7858D010058A4
:107C10001F4FE8018881998101968F779927AD01DF
:107C20004E575F4FEA012881398128173907D1F370
:107C3000E80128813981A20FB31F6C93A685B7850F
:107C4000A058BF4F11969C938E93A689B7892C910B
:107C500081E090E0078C02C0880F991F0A94E2F738
:107C6000822B8C9381E081A30488F589E02D8081AB
:107C70008064808381E090E0DF91CF911F910F912C
:107C80000895FC0181A1882329F0A489B5898C91EC
:107C900086FFFBCF11A20895FC01A485B585FD01E7
:107CA000E058FF4F208131813296808191812817E1
:107CB000390779F080819181A80FB91F8C912081BB
:107CC00031812F5F3F4F2F7733273183208390E01F
:107CD00008958FEF9FEF0895DC011C96ED91FC91C4
:107CE0001D97DF01A058BF4F2D913C91119712961F
:107CF0008D919C9111972817390739F08D919C919E
:107D0000E80FF91F808190E008958FEF9FEF0895AD
:107D1000FC0124853585F901E058FF4F8081918170
:107D200032962081318180589F4F821B930B60E8EF
:107D300070E00C94B4F60895089580E090E0089502
:107D4000CF92DF92EF92FF92C0903D02D0903E0220
:107D5000E0903F02F0904002FC0180819181A2817D
:107D6000B38180933D0290933E02A0933F02B09373
:107D700040020E9492BFC0923D02D0923E02E09229
:107D80003F02F0924002FF90EF90DF90CF90089575
:107D90008091C9119091CA11981759F0E92FF0E01C
:107DA000E75BFE4E80819F5F9F779093CA1190E0C2
:107DB00008958FEF9FEF08951F920F920FB60F92C5
:107DC00011240BB60F920F931F932F933F934F9352
:107DD0005F936F937F938F939F93AF93BF93CF9353
:107DE000DF93EF93FF930091CA11D091C91111E075
:107DF0001D0F1F77C091C6009091E204492F092EF4
:107E0000000C550B660B770B4C30510508F046C043
:107E1000FA018827EC56FF4F8F4F0C94C7F6CD34EC
:107E200041F0CE34B9F481E005C0CA3330F0CD342E
:107E300071F582E08093E20446C0C03308F043C08D
:107E4000C03209F440C0CD3211F53DC0C13329F034
:107E5000C43329F0C032D9F436C083E0EBCF88E0D8
:107E6000E9CFC03321F0C13391F486E0E3CF84E061
:107E7000E1CFC83361F485E0DDCFC23341F487E060
:107E8000D9CFC13321F489E0D5CFC03311F08BE0D5
:107E9000D1CF8AE0CFCFCA30B1F413C0CA3099F441
:107EA000973049F09A3059F0953059F410922402E5
:107EB0001092C41006C081E08093710502C00E9438
:107EC000E0671092E204011731F0ED2FF0E0E75B7C
:107ED000FE4EC083D12FD093C911FF91EF91DF9156
:107EE000CF91BF91AF919F918F917F916F915F9152
:107EF0004F913F912F911F910F910F900BBE0F90BB
:107F00000FBE0F901F9018958091CD079091CE07CE
:107F1000009731F04AE050E060E070E00C94A2EC91
:107F200060E070E0CB010895EFDF97FD0AC0ECDF61
:107F30006F3F71058105910509F02CF4E5DF862F6F
:107F4000089580E008958FEF08958091CD07909176
:107F5000CE07892B31F0E8DF91E0811103C090E07A
:107F600001C091E0892F08950F931F93CF938091C3
:107F7000CD079091CE07009711F1FC018F01C191BF
:107F80002C2F2F7DA9F0C53411F0C536B9F7F801B3
:107F9000108260E070E08091CD079091CE070E9442
:107FA0004FEBF801C083562F472F382F292F0BC0D6
:107FB00060E070E0CF911F910F910C944FEB50E077
:107FC00040E030E020E0652F742F832F922FCF9177
:107FD0001F910F91089581548A3108F042C0E82F13
:107FE000F0E0409140115091411160914211709127
:107FF000431104C076956795579547958A95D2F7B2
:10800000842F817040FF2FC0EA5DFE4E908199233E
:1080100009F1E091BA10F091BB10E90FF11D9081C8
:1080200020ED290F2A3098F09E3211F491810CC076
:108030009D3211F09B3271F4918120ED290F2A308D
:1080400030F09E3239F4928190539A3018F42E2FEA
:108050009F2F02C020E090E02093CD079093CE07A1
:10806000089580E008950895B6DF882341F081E007
:108070002091CD073091CE07232B09F480E008959D
:1080800080E1ECE4F4E0A2E1B1E101900D928A9587
:10809000E1F708952F923F924F925F926F927F92F5
:1080A0008F929F92AF92BF92CF92DF92EF92FF9208
:1080B0000F931F93CF93DF9300D01F921F92CDB7E2
:1080C000DEB77C018B016A01190180904C0490900D
:1080D0004D04A0904E04B0904F04A5019401FC0102
:1080E00060817181828193810E944EEFF1E0FD8376
:1080F000811112C0209150043091510440915204DA
:1081000050915304F80160817181828193810E94B2
:108110004EEF811101C01D82F601408051806280C6
:108120007380209104023091050240910602509123
:108130000702C301B2010E944EEF882309F453C025
:108140004092040250920502609206027092070269
:1081500020E030E040E450E46091A6077091A7076A
:108160008091A8079091A9070E94A7F469837A8358
:108170008B839C838092121190921311A092141100
:10818000B09215118091500490915104A091520425
:10819000B09153048093161190931711A093181166
:1081A000B0931911F60180819181A281B3818093EE
:1081B0001A1190931B11A0931C11B0931D11809163
:1081C000580490915904A0915A04B0915B04809393
:1081D0001E1190931F11A0932011B0932111CE0175
:1081E0000196AEDD4DDFFD81FF2309F16090A2070E
:1081F0007090A3078090A4079090A507A0909E0779
:10820000B0909F07C090A007D090A1079501A6014C
:10821000B301C4010E94F1F5181614F05301640172
:1082200020E030E040E251E4B501C6010CC020E09E
:1082300030E040EC5FE36091AA077091AB0780915A
:10824000AC079091AD070E94A7F469837A838B8372
:108250009C8320913004222349F0AB01BC0187E0CC
:108260009EE00E9461C68AE00E94679AF7018081C1
:108270009181A281B3818093121190931311A093E5
:108280001411B0931511F80180819181A281B381FD
:108290008093161190931711A0931811B093191190
:1082A000F101208131814281538160911E117091D1
:1082B0001F1180912011909121110E94CBF36093A6
:1082C0001E1170931F118093201190932111CE01E4
:1082D000019636DDD5DE0F900F900F900F900F9026
:1082E000DF91CF911F910F91FF90EF90DF90CF9092
:1082F000BF90AF909F908F907F906F905F904F90C6
:108300003F902F90089580E1E2E1F1E1ACE4B4E028
:1083100001900D928A95E1F708959C0197FD0EC09A
:108320008436910584F064E670E00E94B4F6CB01D7
:108330006AE070E00E94B4F6805D06C03195219538
:1083400031098DE201C080E280933B042A3031057F
:1083500064F0EAE0F0E0C901BF010E94B4F6CB018D
:10836000BF010E94B4F6805D01C080E280933C04AE
:10837000C9016AE070E00E94B4F6805D80933D041C
:108380008BE394E00895893691051CF029E680E09E
:1083900002C0282F892F20934204809343040C9419
:1083A00063592F923F924F925F926F927F928F927A
:1083B0009F92AF92BF92CF92DF92EF92FF920F9374
:1083C0001F93CF93DF93CDB7DEB7C455D1090FB656
:1083D000F894DEBF0FBECDBFE6ECF0E184918F01D3
:1083E0000F5F1F4F882321F00E94679AF801F6CF94
:1083F0000E9433B781110C94BE4B80E090E0A0E85E
:10840000BFE380930A1190930B11A0930C11B093CA
:108410000D1180E090E0A0ECB0E480930E119093F9
:108420000F11A0931011B09311118DEC9CECACE4E2
:10843000BEE38093061190930711A0930811B093A7
:10844000091180E090E0A8ECB1E48093DE04909301
:10845000DF04A093E004B093E1048CE390E09093F8
:10846000DD048093DC0488EC90E09093DB0480933F
:10847000DA041092D9048FE4F7DD882311F074DD5B
:1084800004C060E070E080E190E46BAF7CAF8DAF42
:108490009EAF83E4E9DD882311F057DD02C083E459
:1084A0009ADD61968FAF61978BE4DEDD882311F052
:1084B0004CDD02C08BE48FDD60968FAF609782E465
:1084C000D3DD8823E9F050DD0E940FF57093DD04C1
:1084D0006093DC046115710599F068527109653685
:1084E000710570F0E1E9F0E184918F010F5F1F4F9A
:1084F000882311F40C94BE4B0E94679AF801F4CFC4
:108500008CE4B2DD882351F12FDD6B017C01609397
:10851000061170930711809308119093091120E0C0
:1085200030E0A9010E94F1F587FD0AC020E030E0AB
:1085300040E050E4C701B6010E944EEF181674F4F3
:10854000E9E6F0E184918F010F5F1F4F882311F45A
:108550000C94BE4B0E94679AF801F4CF81E53BDD95
:10856000882309F440C08091CD079091CE07892BD4
:1085700019F4EEE3F0E12BC0F7DC6B017C016093B2
:108580000E1170930F1180931011909311112DEC17
:108590003CEC4CE45DE30E94F1F587FD0AC020E06D
:1085A00030E040E751E4C701B6010E944EEF1816D3
:1085B000D4F4EDE0F0E184918F010F5F1F4F882329
:1085C00011F40C94BE4B0E94679AF801F4CF849189
:1085D0008F010F5F1F4F882311F40C94BE4B0E9434
:1085E000679AF801F4CF83E53FDD882319F1BCDCFD
:1085F0004B015C012DEC3CEC4CEC5DE30E94F1F591
:1086000087FD0AC020E030E040E85FE3C501B40127
:108610000E944EEF1816ACF4E6EEFFE084918F0155
:108620000F5F1F4F882311F40C94BE4B0E94679A72
:10863000F801F4CF5DEC852E5CEC952EA92C5EE361
:10864000B52E80E5C8DC882309F443C08091CD07AE
:108650009091CE07892B71F4EEEAFFE084918F01AF
:108660000F5F1F4F882311F40C94BE4B0E94679A32
:10867000F801F4CF8091D9048F5F8093D90474DC22
:108680006B017C016093DE047093DF048093E0044F
:108690009093E10420E030E0A9010E94F1F587FD0C
:1086A0000AC020E030E048EC51E4C701B6010E9466
:1086B0004EEF181674F4E6E8FFE084918F010F5F27
:1086C0001F4F882311F40C94BE4B0E94679AF80147
:1086D000F4CF86E4C9DC882319F146DC6B017C0108
:1086E00020E030E040E85FE30E94F1F587FD0AC03A
:1086F00020E030E040E850E4C701B6010E944EEFB0
:108700001816A4F4EDE5FFE084918F010F5F1F4F71
:10871000882311F40C94BE4B0E94679AF801F4CFA1
:10872000C12CD12C40EEE42E4FE3F42EA70196018C
:10873000C701B6010E94B3EF9B01AC0160E070E09D
:1087400084E490E40E94A7F420910A1130910B1167
:1087500040910C1150910D110E94B3EF2B013C017F
:10876000A5019401C501B4010E94B3EFA7019601D0
:108770000E94B3EF2CEE31E548EB5DE30E94A7F4D5
:108780009B01AC01C301B2010E94B3EF60930A11D7
:1087900070930B1180930C1190930D1188E464DC9D
:1087A0008823C9F0E1DB0E940FF57093DB0460932E
:1087B000DA04655A71096437710568F0EFE2FFE089
:1087C00084918F010F5F1F4F882309F4D7C70E9440
:1087D000679AF801F5CF85E5FEDB8823E9F00E9472
:1087E0006762611571058105910511F00E9446EBE4
:1087F0008091CD079091CE07892B11F0B5DB04C095
:1088000060E070E088E492E46093D5047093D6044D
:108810008093D7049093D80482E5DDDB81110DC0ED
:10882000EBEFFEE084918F010F5F1F4F882309F467
:10883000A5C70E94679AF801F5CF8091CD07909166
:10884000CE07892BA9F060DB2F967FAF6EAF2F97F5
:10885000161617069CF0E7ECFEE084918F010F5F7F
:108860001F4F882309F48AC70E94679AF801F5CF41
:108870008AE190E02F969FAF8EAF2F9788E5F4DBCB
:10888000882361F071DB209124043091250440910C
:108890002604509127040E94CAF308C060914C043A
:1088A00070914D0480914E0490914F046093D104D7
:1088B0007093D2048093D3049093D40489E5D4DBDD
:1088C000882361F051DB20912804309129044091E4
:1088D0002A0450912B040E94CAF308C060915004EE
:1088E0007091510480915204909153046093CD048F
:1088F0007093CE048093CF049093D0046091D10400
:108900007091D2048091D3049091D4044DEC54E042
:1089100039D981110DC0EDE9FEE084918F010F5F1F
:108920001F4F882309F42AC70E94679AF801F5CFE0
:1089300084E451DB91E089270E94408520E030E00B
:1089400040EA50E4609154047091550480915604BB
:10895000909157040E944EEF87FF14C0198A1A8A1B
:108960001B8A1C8A80E090E0A0EAB0E489839A83A5
:10897000AB83BC83BE016F5E7F4FCE0101960E9428
:10898000A486C1DC0E9467626B017C01A8E8CA0E64
:10899000A3E1DA1EE11CF11C8091DC049091DD045E
:1089A000F2DC6091DC047091DD04072E000C880B72
:1089B000990B0E9454EF9B01AC01609144047091AB
:1089C000450480914604909147040E94CAF34B01EC
:1089D0005C0120E030E0A9010E94F1F587FF04C0AE
:1089E000B7FAB094B7F8B09420E030E040E450E437
:1089F000C501B4010E94F1F518160CF50E946762DA
:108A0000DC01CB018C199D09AE09BF09B7FD0FC070
:108A10000E9467626B017C01B8E8CB0EB3E1DB1EFC
:108A2000E11CF11C0E94A9588AE00E94679A80E02C
:108A30000E946EAE8091C9118093CA11B2CF80910D
:108A4000DA049091DB040E94FB596091DA04709182
:108A5000DB04072E000C880B990B0E9454EF9B013E
:108A6000AC0160915C0470915D0480915E04909112
:108A70005F040E94CAF34B015C0120E030E0A901D1
:108A80000E94F1F587FF04C0B7FAB094B7F8B0942C
:108A900020E030E040E450E4C501B4010E94F1F56B
:108AA00018160CF50E946762DC01CB018C199D0938
:108AB000AE09BF09B7FD0FC00E9467626B017C0160
:108AC000E8E8CE0EE3E1DE1EE11CF11C0E94A9588D
:108AD0008AE00E94679A80E00E946EAE8091C91180
:108AE0008093CA11B2CF1092580410925904109278
:108AF0005A0410925B0488E594E00E94D2B68091FB
:108B0000D904882399F1BCDA2091DE043091DF0486
:108B10004091E0045091E10460911E1170911F1189
:108B200080912011909121110E94CBF360931E112E
:108B300070931F11809320119093211120E030E059
:108B400040E751E46091AA077091AB078091AC07B0
:108B50009091AD070E94A7F469837A838B839C83ED
:108B6000CE010196EDD88CDA0E94DFB480E2EDEA06
:108B7000F4E0DF01282F1D922A95E9F7EDE8F4E0F3
:108B8000DF01282F1D922A95E9F7EDE6F4E0DF01D9
:108B90001D928A95E9F774DA809106119091071178
:108BA000A0910811B091091180931A1190931B1193
:108BB000A0931C11B0931D1119821A821B821C8272
:108BC0009E012F5F3F4F4AE151E166E171E182E191
:108BD00091E160DA9E01255C3F4F4AE151E166E197
:108BE00071E182E191E156DA6196BFAD6197BB23F5
:108BF00029F060E574E08CE494E004C06DEC74E06E
:108C000081ED94E00E948AE1298F3A8F4B8F5C8F2F
:108C10006D8F7E8F3FAF2D962FAF2D972D96EFAD99
:108C20002D97E7FD82C4FFADF7FD7FC424E0E2028B
:108C3000F0011124E855F54F408051806280738027
:108C40003FAD84E03802F0011124EC56F54FD0809E
:108C5000C180328023808D2D9C2DA32DB22D8FAB12
:108C600098AFA9AFBAAFAE01495C5F4FB201C30183
:108C70000E94C23D882309F45CC420E030E040EA51
:108C800050E4B201C3010E94CBF3F62E072F182F38
:108C9000E92E862F902FA12FBE2D8BAB9CABADABB9
:108CA000BEAB8D2D9C2DA32DB22D8FA798ABA9AB5C
:108CB000BAAB2D969FAD2D97911152C0AFADA111BA
:108CC00005C05F2D402F312F2E2D04C0542D452D72
:108CD000362D272D852F942FA32FB22F8BAB9CAB36
:108CE000ADABBEABBFADB43034F4F42C052D162DB6
:108CF000E72CBB2369F020E030E040EA50E46D2D22
:108D00007C2D832D922D0E94CAF3362F272F03C06E
:108D10009601832D922D432F522FBC014FA758ABA4
:108D200069AB7AABEFADE4300CF0A7C020E030E0E7
:108D300040EA50E46D2D7C2D832D922D0E94CBF3C3
:108D400021966FAF219723967FAF239725968FAFFC
:108D5000259727969FAF2797FFADF11185C099C042
:108D60002D962FAD2D9724300CF453C03FAD3430E9
:108D70005CF020E030E040EA50E4B201C3010E9420
:108D8000CAF3362F272F03C0342D252DC301432FBF
:108D9000522FBC014BAB5CAB6DAB7EAB8FAD811189
:108DA000E4C420E030E040EA50E4B201C3010E9494
:108DB000CAF3F62E072F182FE92E20E030E040EA04
:108DC00050E46D2D7C2D832D922D0E94CBF36FA747
:108DD00078AB89AB9AAB9FAD992309F44EC020E0E4
:108DE00030E040EA50E46D2D7C2D832D922D0E94C1
:108DF000CAF321966FAF219723967FAF23972596CD
:108E00008FAF259727969FAF2797AFADA43064F11A
:108E100040C0BFADB1110DC020E030E040EA50E4E9
:108E2000B201C3010E94CAF3F62E072F182FE92EB4
:108E30000FC0EFADE430B4F120E030E040EA50E4A0
:108E4000B201C3010E94CAF36BAB7CAB8DAB9EAB8E
:108E50002196DFAE21972396CFAE239725963FAE7E
:108E6000259727962FAE279732ED832E33E5932E45
:108E70003BE7A32E31E4B32E29C02196DFAE219724
:108E80002396CFAE239725963FAE259727962FAEF4
:108E9000279722ED822E23E5922E2BEFA22E20E49F
:108EA000B22E14C02196DFAE21972396CFAE239722
:108EB00025963FAE259727962FAE279792ED892EC0
:108EC00093E5992E9BEFA92E91E4B92E8BA99CA92D
:108ED000ADA9BEA92C968CAF9DAFAEAFBFAF2C97FE
:108EE0009C01AD01B201C3010E94CAF3698B7A8B68
:108EF0008B8B9C8B4FA458A869A87AA8A3019201D8
:108F00006D2D7C2D832D922D0E94CAF36D8B7E8B4F
:108F10008F8B988F2C962CAD3DAD4EAD5FAD2C97C1
:108F200060914C0470914D0480914E0490914F04D7
:108F30000E94CAF32C966CAF7DAF8EAF9FAF2C977B
:108F4000A3019201609150047091510480915204E8
:108F5000909153040E94CAF32B013C018F2D902F56
:108F6000A12FBE2D89839A83AB83BC8321968FADBD
:108F7000219723969FAD23972596AFAD25972796EA
:108F8000BFAD27978D839E83AF83B88780910611ED
:108F900090910711A0910811B091091189879A87C2
:108FA000AB87BC872DEC3CEC4CEC5CE3C501B40119
:108FB0000E94B3EF20910A1130910B1140910C11D6
:108FC00050910D110E94B3EF209158043091590433
:108FD00040915A0450915B040E94CBF36D877E87C9
:108FE0008F87988B2C962CAD3DAD4EAD5FAD2C97F9
:108FF000CA01B9010E94B3EF6B017C01A301920188
:10900000C301B2010E94B3EF9B01AC01C701B601DD
:109010000E94CBF320E030E040E050E40E94F1F504
:1090200018160CF046C00E94DFB41BA21CA21DA2A1
:109030001EA220E030E040E05FE3609154047091B4
:10904000550480915604909157040E94CBF36F8F82
:1090500078A389A39AA39E012D5D3F4FAE01415E87
:109060005F4F60E574E08CE494E014D81BA21CA26E
:109070001DA21EA220E030E040E05FE360910611F7
:109080007091071180910811909109110E94CBF302
:109090006F8F78A389A39AA39E012D5D3F4FAE01E8
:1090A000415E5F4FBE01615D7F4FCE01C3960E945E
:1090B0004A401F8E18A219A21AA29E01215E3F4F9C
:1090C00046E051E1BE01615D7F4FCE01C3960E9433
:1090D0004A400E940BB540903D0250903E02609085
:1090E0003F0270904002E090A207F090A307009129
:1090F000A4071091A507A0909E07B0909F07C0906D
:10910000A007D090A1079501A601B701C8010E9450
:10911000F1F5181614F47501860120E030E040E204
:1091200051E4B701C8010E94A7F460933D02709317
:109130003E0280933F029093400240E0BE016F5E8A
:109140007F4FCE0101960E947EBB40923D0250921D
:109150003E0260923F02709240020E944040A8EAA4
:10916000BAE02496BFAFAEAF249722961FAE1EAED4
:10917000229701E010E021960FAC219702C0000F6A
:10918000111F0A94E2F72296EEADFFAD22973196B9
:109190002296FFAFEEAF229721E030E021960FAC90
:1091A000219702C0220F331F0A94E2F763963FAF64
:1091B0002EAF63978DE6282E84E0382E8DEA94E05A
:1091C0002A969FAF8EAF2A97ADE8B4E02896BFAF3E
:1091D000AEAF2897E4E9FAE02696FFAFEEAF269708
:1091E0002A962EAD3FAD2A9765963FAF2EAF659775
:1091F000D9018D919C919C0120233123232B09F4CB
:10920000ADC06396EEADFFAD63978E239F23892B90
:1092100009F4A4C02896AEADBFAD28978D919C915E
:1092200080239123892B09F099C020E030E040E0B1
:1092300050E42496AEADBFAD24976D917D918D9194
:109240009C910E94CBF36B017C0120E030E040E078
:1092500050E42496EEADFFAD24976481758186813C
:1092600097810E94CAF34B015C0120E030E040E8A6
:1092700050ECC701B6010E944EEF87FD70C120E09F
:1092800030E046E553E4C701B6010E94F1F5181637
:1092900034F4C12CD12CB6E5EB2EB3E4FB2ECBA6D7
:1092A000DCA6EDA6FEA62696AEADBFAD26974D90E8
:1092B0005D906D907C9020E030E040E85FE3C3017A
:1092C000B2010E944EEF87FD51C120E030E046E53B
:1092D00053E4C301B2010E94F1F5181634F4412C95
:1092E000512CF6E56F2EF3E47F2E4F8E58A269A223
:1092F0007AA24FA258A669A67AA620E030E040E8FC
:1093000050ECC501B4010E944EEF87FD36C120E04C
:1093100030E046E553E4C501B4010E94F1F51816AA
:1093200034F4812C912C76E5A72E73E4B72E8BA212
:109330009CA2ADA2BEA2AE01495D5F4FC701B601BE
:109340000E94C23D811120C12896EEADFFAD289745
:1093500080819181802B912B918380832A962EADE1
:109360003FAD2A972E5F3F4F2A963FAF2EAF2A97E9
:109370006596AEADBFAD65978D919C91802391238D
:10938000892B09F4A6C0F901808191818023912362
:10939000892B09F49EC0F101808191818023912362
:1093A000892B09F096C020E030E040E050E426969A
:1093B000AEADBFAD26976D917D918D919C910E9430
:1093C000CBF32B013C0120E030E040E050E4269656
:1093D000EEADFFAD269764817581868197810E94ED
:1093E000CAF34B015C012496AEADBFAD2497CD907E
:1093F000DD90ED90FC9020E030E040E850ECC701BB
:10940000B6010E944EEF87FDFFC020E030E046E548
:1094100053E4C701B6010E94F1F5181634F4C12CCB
:10942000D12C56E5E52E53E4F52ECBA2DCA2EDA21D
:10943000FEA2CBA6DCA6EDA6FEA620E030E040E82A
:109440005FE3C301B2010E944EEF87FDE4C020E05C
:1094500030E046E553E4C301B2010E94F1F518166D
:1094600034F4412C512C36E5632E33E4732E4FA295
:1094700058A669A67AA620E030E040E85FE3C5017F
:10948000B4010E944EEF87FDCDC020E030E046E5FC
:1094900053E4C501B4010E94F1F5181634F4812C8F
:1094A000912C96E5A92E93E4B92E8F8E98A2A9A2AD
:1094B000BAA2AE01495D5F4FC701B6010E94C23D2D
:1094C0008111B7C0F10180819181802B912B918313
:1094D0008083F2E02F0E311C28962EAD3FAD2897E9
:1094E0002E5F3F4F28963FAF2EAF289726968EAD22
:1094F0009FAD2697049626969FAF8EAF269797E747
:10950000291694E0390609F06BCE2496AEADBFADB6
:10951000249714962496BFAFAEAF24972296EEAD53
:10952000FFAD2297359709F024CE8091C911809321
:10953000CA112F962EAD3FAD2F97215031092F968E
:109540003FAF2EAF2F97232B09F4B3C02D963FAD1D
:109550002D9737FDAEC08FAD87FF46CBAAC0C12C7B
:10956000D12CA0E8EA2EA0ECFA2E99CE412C512C59
:10957000E0E86E2EEFE37E2EB8CE812C912C60E8D1
:10958000A62E60ECB62ED3CEAE01415E5F4FC50174
:10959000B4010E94C23D882309F4D6CE80913004E4
:1095A000882321F1B701A60187E79EE00E9461C6EA
:1095B0004FA158A569A57AA581E79EE00E9461C6E2
:1095C0004BA15CA16DA17EA187E69EE00E9461C6D1
:1095D0004F8D58A169A17AA181E69EE00E9461C6E3
:1095E00089E20E94679A8AE00E94679A9E01215E42
:1095F0003F4FAE014D5D5F4FBE01695D7F4FCE01B4
:109600008B960E943BB5A0CEC12CD12C40E8E42E15
:1096100040ECF42E0ACF412C512C20E8622E2FE38F
:10962000722E25CF812C912C80E8A82E8FE3B82EA6
:109630003CCFAE01415E5F4FC701B6010E94C23D03
:10964000882309F43FCF80913004882321F1B701AA
:10965000A6018DE39EE00E9461C64FA158A569A5B1
:109660007AA587E39EE00E9461C64BA15CA16DA133
:109670007EA18DE29EE00E9461C64F8D58A169A136
:109680007AA187E29EE00E9461C689E20E94679A01
:109690008AE00E94679A9E01215E3F4FAE014D5DB8
:1096A0005F4FBE01695D7F4FCE018B960E943BB537
:1096B00009CF0E94DFB480E090E0A0EAB0E480939C
:1096C0001A1190931B11A0931C11B0931D111982B4
:1096D0001A821B821C829E012F5F3F4F4AE151E19B
:1096E00066E171E182E191E10E944A408091D104FA
:1096F0009091D204A091D304B091D404809312111C
:1097000090931311A0931411B09315118091CD046F
:109710009091CE04A091CF04B091D0048093161103
:1097200090931711A0931811B093191119821A82EE
:109730001B821C829E012F5F3F4F4AE151E166E18F
:1097400071E182E191E10E944A406096FFAD60972D
:10975000F11114C010924304109242040E94635904
:1097600080E090E00E94FB5909C02FADF42C052D3C
:10977000162DE72C24300CF032CB1FCBCC5ADF4F08
:109780000FB6F894DEBF0FBECDBFDF91CF911F9112
:109790000F91FF90EF90DF90CF90BF90AF909F9090
:1097A0008F907F906F905F904F903F902F90089593
:1097B0001F920F920FB60F9211240BB60F922F9398
:1097C0003F938F939F93EF93FF932091BD0F309121
:1097D000BE0F8091BF0F9091C00F2817390731F449
:1097E000809131018F7D8093310114C0E091BF0FD2
:1097F000F091C00FE35CF04F20818091BF0F9091FA
:10980000C00F01968F7799279093C00F8093BF0F59
:1098100020933601FF91EF919F918F913F912F916E
:109820000F900BBE0F900FBE0F901F9018951F92B8
:109830000F920FB60F9211240BB60F922F934F93E6
:109840005F938F939F93EF93FF938091300182FDFD
:109850001CC020913601809141109091421040919E
:1098600043105091441001968F7799274817590754
:1098700071F0E0914110F0914210EF53F04F2083CE
:10988000909342108093411002C080913601FF9165
:10989000EF919F918F915F914F912F910F900BBE00
:1098A0000F900FBE0F901F9018952F923F924F92DE
:1098B0005F926F927F928F929F92AF92BF92CF9260
:1098C000DF92EF92FF920F931F93CF93DF93CDB769
:1098D000DEB762970FB6F894DEBF0FBECDBFF89427
:1098E0008FEF9FEF90938900809388002AE02A8B66
:1098F000212C312C78948091350590913605A091DA
:109900003705B0913805892B8A2B8B2B09F016C2AD
:1099100080913B058823E1F010923B058091390549
:1099200090913A05892B09F409C21092ED04109226
:109930003A051092390590915E0A80915F0A981756
:1099400009F4FCC180915F0A8F5F8F7080935F0A7A
:109950008091390590913A05892B09F4EFC1409126
:109960003105509132056091330570913405809135
:109970002D0590912E05A0912F05B09130050091F5
:10998000240510E020E030E0841B950BA60BB70BFC
:10999000081719072A073B0710F4D901C801E82F57
:1099A000840F951FA61FB71F809331059093320532
:1099B000A0933305B0933405209184003091850045
:1099C000225E3F4F4091090550910A0560910B05B9
:1099D00070910C058091F9049091FA04A091FB0418
:1099E000B091FC04840F951FA61FB71F8093090533
:1099F00090930A05A0930B05B0930C05B7FD1CC00E
:109A0000889A8091E6109091E710A091E810B091AB
:109A1000E91040910802042E000C550B660B770BE1
:109A2000840F951FA61FB71F8093E6109093E71031
:109A3000A093E810B093E91040910D0550910E05E8
:109A400060910F05709110058091FD049091FE04C6
:109A5000A091FF04B0910005840F951FA61FB71FAA
:109A600080930D0590930E05A0930F05B0931005FC
:109A7000B7FD1CC08E9A8091EA109091EB10A091D6
:109A8000EC10B091ED1040910902042E000C550B22
:109A9000660B770B840F951FA61FB71F8093EA10E4
:109AA0009093EB10A093EC10B093ED104091110542
:109AB0005091120560911305709114058091010574
:109AC00090910205A0910305B0910405840F951FA4
:109AD000A61FB71F8093110590931205A09313053D
:109AE000B0931405B7FD3FC08091E704F0910A02DE
:109AF0008823C9F08091E50482FF02C0F7FD06C00B
:109B00008091E404882311F40C940A568091E504B2
:109B10009091E60493FF02C0F7FD0CC08091E3042E
:109B2000811108C006C080910B01809588708093D8
:109B30000901419A4091EE105091EF106091F010A0
:109B40007091F1108F2FFF0F990BAA0BBB0B840F95
:109B5000951FA61FB71F8093EE109093EF10A09350
:109B6000F010B093F11040911505509116056091D9
:109B70001705709118058091050590910605A09133
:109B80000705B0910805840F951FA61FB71F809386
:109B9000150590931605A0931705B0931805B7FD0A
:109BA0003AC04091F2105091F3106091F41070910E
:109BB000F510C0900B020C2C000CDD08EE08FF081D
:109BC0004C0D5D1D6E1D7F1D4093F2105093F310E0
:109BD0006093F4107093F5104091F5045091F604E1
:109BE0006091F7047091F804841B950BA60BB70BDA
:109BF0008093150590931605A0931705B09318054B
:109C00009091E8048091220593FF02C0815001C029
:109C10008F5F809322058091840090918500821748
:109C20009307C8F38091090590910A05A0910B054F
:109C3000B0910C05B7FD15C04091F5045091F604A4
:109C40006091F7047091F804841B950BA60BB70B79
:109C50008093090590930A05A0930B05B0930C051A
:109C6000889880910D0590910E05A0910F05B091F7
:109C70001005B7FD15C04091F5045091F6046091B0
:109C8000F7047091F804841B950BA60BB70B809317
:109C90000D0590930E05A0930F05B09310058E98B7
:109CA0008091110590911205A0911305B0911405B2
:109CB000B7FD3AC04091F5045091F6046091F70465
:109CC0007091F804841B950BA60BB70B80931105BC
:109CD00090931205A0931305B09314058091E704A7
:109CE0008823E1F08091E50482FF04C080910A029C
:109CF00087FD05C08091E404882309F493C780910F
:109D0000E5049091E60493FF04C080910A0287FD68
:109D10000BC08091E304811107C005C080910B0145
:109D20008870809309014198E15041F0809184004E
:109D30009091850082179307C8F342CE8091150257
:109D400090911602A0911702B0911802892B8A2BCC
:109D50008B2B09F091C080912305882309F453C00F
:109D60008090310590903205A0903305B090340575
:109D7000C0901E05D0901F05E0902005F0902105B1
:109D800040912205C814D904EA04FB0480F48091B0
:109D9000EE049091EF042091F2043091F30428171F
:109DA000390728F4415040932205019714C08C14C0
:109DB0009D04AE04BF04E0F48091EE049091EF04A2
:109DC0002091F0043091F1048217930788F44F5FDB
:109DD0004093220501969093EF048093EE04409106
:109DE00011025091120260911302709114020EC080
:109DF0008FEF9FEFDC018093110290931202A093EA
:109E00001302B09314024FEF5FEFBA018091220565
:109E100087FD02C0169A01C0169880918400909127
:109E200085004E96209122052223F1F0149A20916C
:109E300084003091850028173907C8F32091220546
:109E400027FF02C02F5F01C02150209322051498E4
:109E500020912205222331F3209184003091850046
:109E600028173907C8F3DDCF409315025093160227
:109E70006093170270931802809135059091360512
:109E8000A0913705B0913805892B8A2B8B2B09F0CF
:109E900046C6A0913905B0913A05109711F40C947B
:109EA000B3578090310590903205A0903305B09063
:109EB000340540912D0550912E0560912F0570912C
:109EC000300584169506A606B706D8F01092ED0464
:109ED00010923A051092390590915E0A80915F0ABE
:109EE000981711F40C94B35780915F0A8F5F8F70AD
:109EF00080935F0A40EDC42E47E0D42EE12CF12C74
:109F00001AC44091290550912A0560912B05709142
:109F10002C05481559056A057B0508F4AAC140912E
:109F20002505509126056091270570912805D69644
:109F30000D911D912D913C91D997401751076207C2
:109F4000730708F077C1411551056105710549F4A2
:109F50008090E9049090EA04A090EB04B090EC04A7
:109F600064C1E12CF980842E952F862F0A811B81F4
:109F7000FD81EE813F8128859C80E0919B18E89DC2
:109F8000912CFF2730919C18389D900CF11D10905A
:109F90009D18189CF00DE99F900CF11D399FF00D54
:109FA000E89FF00D092D1F2F099DE12D3327222752
:109FB0000F9FE00D311D2E1D199DE00D311D2E1D31
:109FC0001F9F300D211D032F122F099DF12C3327C8
:109FD00022270F9FF00C311D2E1D199DF00C311DF5
:109FE0002E1D1F9F300D211D032F122FEE27809055
:109FF000E9049091EA048091EB0400906C040E282F
:10A0000009F483C030916804309FE1198E089E09DD
:10A010008E0920916904209FE01981089E098E090C
:10A02000F0906A04F09E801891098E09319FE01922
:10A0300081089E098E09219F801891098E09F19E41
:10A0400090198109099DF12C332722270F9FF00CCD
:10A05000311D2E1D199DF00C311D2E1D1F9F300D21
:10A06000211D032F122F30916404309FE10D8E1CAF
:10A070009E1D8E1D20916504209FE00D811C9E1D5C
:10A080008E1DF0906604F09E800C911D8E1D319FF8
:10A09000E00D811C9E1D8E1D219F800C911D8E1D2B
:10A0A000F19E900D811D099DF12C332722270F9FD2
:10A0B000F00C311D2E1D199DF00C311D2E1D1F9F02
:10A0C000300D211D032F122F30916004309FE119B4
:10A0D0008E089E098E0920916104209FE019810855
:10A0E0009E098E09F0906204F09E801891098E09F5
:10A0F000319FE01981089E098E09219F80189109DE
:10A100008E09F19E9019810982C030916804309FB8
:10A11000E10D8E1C9E1D8E1D20916904209FE00D77
:10A12000811C9E1D8E1DF0906A04F09E800C911D76
:10A130008E1D319FE00D811C9E1D8E1D219F800C68
:10A14000911D8E1DF19E900D811D099DF12C3327CF
:10A1500022270F9FF00C311D2E1D199DF00C311D73
:10A160002E1D1F9F300D211D032F122F30916404CF
:10A17000309FE1198E089E098E0920916504209F69
:10A18000E01981089E098E09F0906604F09E8018FF
:10A1900091098E09319FE01981089E098E09219F3E
:10A1A000801891098E09F19E90198109099DF12C61
:10A1B000332722270F9FF00C311D2E1D199DF00C07
:10A1C000311D2E1D1F9F300D211D032F122F309189
:10A1D0006004309FE10D8E1C9E1D8E1D2091610438
:10A1E000209FE00D811C9E1D8E1DF0906204F09E4C
:10A1F000800C911D8E1D319FE00D811C9E1D8E1DBA
:10A20000219F800C911D8E1DF19E900D811D1124AA
:10A210009C82F9820A831B83FD83EE833F83288718
:10A22000912C992AA12CB12CA82A83EF98E121E046
:10A23000298B14C0D2968D909D90AD90BC90D597EF
:10A24000F4CFB694A79497948794D988DD0CD98AD3
:10A25000049629E18F30920709F4EAC4FC010591C4
:10A26000159125913491081519052A053B0548F3E8
:10A27000DFC440901E0550901F056090200570902F
:10A280002105481459046A047B0408F0C3C1809175
:10A290001D05811121C0FD01EE5BFF4FE080F180C3
:10A2A0000281138178962081318142815381D29637
:10A2B0006D917D918D919C91D5970E948DC5DD24E6
:10A2C000D394D0921D05E0913905F0913A0582A909
:10A2D00093A9A4A9B5A98EC14091190550911A0559
:10A2E00060911B0570911C05DA960D911D912D91C1
:10A2F0003C91DD97401751076207730708F073C15F
:10A30000411551056105710549F48091E904909169
:10A31000EA04A091EB04B091EC046CC1F0E0E98593
:10A32000842F352F262FAA857B856C855D85BE857C
:10A330004F859889B0919B18B89F612D5527409102
:10A340009C18489F600D511D10909D18189E500D2F
:10A35000B39F600D511D439F500DB29F500DA62F0E
:10A36000752FA69FB12D44279927A59FB00D411D9C
:10A370009F1F769FB00D411D9F1F759F400D911D22
:10A38000A42F792FA69FE12D44279927A59FE00DA3
:10A39000411D9F1F769FE00D411D9F1F759F400D22
:10A3A000911DA42F792FBB278091E9043091EA04F5
:10A3B0002091EB0400906C040F2A09F483C04091B3
:10A3C00068044A9FB1198F0B3F0B2F0B90916904C2
:10A3D0009A9FB01981093F0B2F0BE0916A04EA9F05
:10A3E000801931092F0B479FB01981093F0B2F0BA3
:10A3F000979F801931092F0BE79F30192109A69FDC
:10A40000E12D44279927A59FE00D411D9F1F769FB1
:10A41000E00D411D9F1F759F400D911DA42F792FA9
:10A42000409164044A9FB10D8F1F3F1F2F1F9091D1
:10A4300065049A9FB00D811D3F1F2F1FE091660498
:10A44000EA9F800D311D2F1F479FB00D811D3F1FBB
:10A450002F1F979F800D311D2F1FE79F300D211D4E
:10A46000A69FE12D44279927A59FE00D411D9F1F21
:10A47000769FE00D411D9F1F759F400D911DA42FDC
:10A48000792F409160044A9FB1198F0B3F0B2F0B1E
:10A49000909161049A9FB01981093F0B2F0BE091B5
:10A4A0006204EA9F801931092F0B479FB019810977
:10A4B0003F0B2F0B979F801931092F0BE79F301906
:10A4C000210982C0409168044A9FB10D8F1F3F1F30
:10A4D0002F1F909169049A9FB00D811D3F1F2F1F60
:10A4E000E0916A04EA9F800D311D2F1F479FB00D38
:10A4F000811D3F1F2F1F979F800D311D2F1FE79F2D
:10A50000300D211DA69FE12D44279927A59FE00D21
:10A51000411D9F1F769FE00D411D9F1F759F400DA0
:10A52000911DA42F792F409164044A9FB1198F0B7C
:10A530003F0B2F0B909165049A9FB01981093F0B37
:10A540002F0BE0916604EA9F801931092F0B479F7A
:10A55000B01981093F0B2F0B979F801931092F0BE1
:10A56000E79F30192109A69FE12D44279927A59F30
:10A57000E00D411D9F1F769FE00D411D9F1F759FA0
:10A58000400D911DA42F792F409160044A9FB10D79
:10A590008F1F3F1F2F1F909161049A9FB00D811D47
:10A5A0003F1F2F1FE0916204EA9F800D311D2F1F76
:10A5B000479FB00D811D3F1F2F1F979F800D311D9D
:10A5C0002F1FE79F300D211D1124E987AA877B8764
:10A5D0006C875D87BE874F87988B90E0932BA0E0B8
:10A5E000B0E0A22B07C0A65ABF4F8D919D910D9050
:10A5F000BC91A02D23EF38E141E0498BF901459151
:10A60000559165917491481759076A077B0708F4BB
:10A6100099C3A6C3809122058823E1F0FD01E85B80
:10A62000FF4F4081518160E070E000911102109174
:10A630001202209113023091140240175107620751
:10A64000730741F010921502109216021092170231
:10A650001092180240910D0250910E0260910F026B
:10A660007091100277FF5FC0AE5ABF4FCD90DD9062
:10A67000ED90FC9083EF98E121E0FC01459155912C
:10A68000659174914C155D056E057F0550F4F69447
:10A69000E794D794C794220F049679E18F309707F7
:10A6A00061F72093240580E2C816D104E104F10487
:10A6B00028F470E2C72ED12CE12CF12C90E2C91ABB
:10A6C000D108E108F108C114A8E0DA06E104F104B8
:10A6D00008F402C4B4E0DB9EC00111248D509B4EEF
:10A6E000FC01329625913491EC2D6627E39FA00161
:10A6F000E29F410D561F0694461F561F112460E02D
:10A7000070E0FC0125913491C901A0E0B0E0841B08
:10A71000950BA60BB70B80930D0290930E02A0939E
:10A720000F02B0931002C0900D02D0900E02E09084
:10A730000F02F09010028091390590913A05892B13
:10A7400009F0E5C10E940FC690933A058093390540
:10A75000892B09F4DCC1E0913905F0913A0580813B
:10A7600083FF3EC085899689A789B08D8093E610C6
:10A770009093E710A093E810B093E910818D928D2B
:10A78000A38DB48D8093EA109093EB10A093EC10FE
:10A79000B093ED10858D968DA78DB0A18093EE10AE
:10A7A0009093EF10A093F010B093F11081A192A1BB
:10A7B000A3A1B4A18093F2109093F310A093F4108E
:10A7C000B093F51090915E0A80915F0A981709F492
:10A7D000B9CF80915F0A8F5F8F7080935F0AB2CF8D
:10A7E000C588D688E788F08C81E0C114D104E104E3
:10A7F000F10409F480E0018D128D238D348D011553
:10A8000011052105310509F08260458D568D678D52
:10A8100070A1411551056105710509F084608093AF
:10A82000ED041092190510921A0510921B05109252
:10A830001C051092250510922605109227051092EE
:10A84000280585A196A1A7A1B0A580932D05909379
:10A850002E05A0932F05B093300588249924540128
:10A86000881A990AAA0ABB0A8092150590921605C1
:10A87000A0921705B09218058092110590921205CA
:10A88000A0921305B092140580920D0590920E05CA
:10A89000A0920F05B09210058092090590920A05CA
:10A8A000A0920B05B0920C05CC0CDD1CEE1CFF1C1D
:10A8B000C092F904D092FA04E092FB04F092FC04F6
:10A8C000000F111F221F331F0093FD041093FE047D
:10A8D0002093FF0430930005440F551F661F771F18
:10A8E000409301055093020560930305709304059E
:10A8F00041A152A163A174A1440F551F661F771F88
:10A90000409305055093060560930705709308056D
:10A91000880F991FAA1FBB1F8093F5049093F6041C
:10A92000A093F704B093F804109231051092320509
:10A93000109233051092340582A593A5A4A5B5A560
:10A940008093290590932A05A0932B05B0932C059D
:10A9500086A597A5A0A9B1A980931E0590931F0570
:10A96000A0932005B093210581A58093F404DF0115
:10A97000A95BBF4F9C9190932305992339F11596BC
:10A980002D913C9111973093F3042093F204129788
:10A990002D913C9111973093F1042093F004109283
:10A9A00015021092160210921702109218021297B6
:10A9B0002D913C91A90160E070E040931102509309
:10A9C000120260931302709314020CC088248A94BC
:10A9D000982C54018092110290921202A0921302BC
:10A9E000B0921402EA5BFF4F90812091E804921329
:10A9F0000AC020910C0230E0482F082E000C550BA5
:10AA00004217530731F09093E80480930C020E94A0
:10AA1000DFC50E94DCD12FEF3FEFA90120930D028B
:10AA200030930E0240930F0250931002E0913905CB
:10AA3000F0913A05DF01DE96ED90FD900D911C91AD
:10AA400022A933A944A955A9EA5AFF4F608171810F
:10AA5000828193810E948DC510921D05E091390578
:10AA6000F0913A05EA5AFF4F80809180A280B3802E
:10AA700083EF98E121E0FC01459155916591749136
:10AA8000481559056A057B0558F4B694A794979420
:10AA90008794220F0496AFE0B9E1A817B90759F7D8
:10AAA00020932405B0E28B169104A104B10428F48C
:10AAB000B0E28B2E912CA12CB12C30E2831A91089C
:10AAC000A108B108811448E09406A104B10408F477
:10AAD00027C254E0959EC00111248D509B4EFC016D
:10AAE000329625913491782D6627739FA001729F2D
:10AAF000410D561F0694461F561F1124FC01C59098
:10AB0000D490E12CF12CC41AD50AE108F108C092C6
:10AB10003505D0923605E0923705F0923805009160
:10AB20003505109136052091370530913805409153
:10AB30001502509116026091170270911802F02EC2
:10AB4000198BF22FE32F401751076207730720F488
:10AB5000F42E598BF62FE72F8F2D9989AF2FBE2F0B
:10AB60000097E1E0AE07B10520F08FEF9FEFA0E086
:10AB7000B0E0081B190B2A0B3B0B00933505109313
:10AB8000360520933705309338054F3FFFEF5F07B9
:10AB90006F077F0761F0481B590B6A0B7B0B4093D3
:10ABA0001502509316026093170270931802F894DE
:10ABB0002091840030918500205F3F4F4A894150A9
:10ABC0004A8B442341F0280E391E2216330610F416
:10ABD0000C947A4C01C019013092890020928800AF
:10ABE000789462960FB6F894DEBF0FBECDBFDF91AA
:10ABF000CF911F910F91FF90EF90DF90CF90BF907A
:10AC0000AF909F908F907F906F905F904F903F900C
:10AC10002F90089580910B01809588708093090191
:10AC20000C94864D80910B0188708093090167C850
:10AC300039893093240580E288169104A104B10477
:10AC400028F430E2832E912CA12CB12C30E2831A0F
:10AC50009108A108B108811488E09806A104B10404
:10AC600020F1E4E09E9EC00111248D509B4EFC011A
:10AC7000329625913491F82DEE27F39F7001F29FC3
:10AC8000E10CFE1E0694EE1EFE1E1124FC01C59072
:10AC9000D490860120E030E0480159018E189F08C9
:10ACA000A108B1087501640122C09501840136959F
:10ACB000279517950795F801EC7FCF018D509F4E92
:10ACC000FC01C590D490FC01329625913491E82D79
:10ACD000E770E29FC001E39F900D112423E0969559
:10ACE00087952A95E1F7C81AD90AE12CF12C4C0D69
:10ACF0005D1D6E1D7F1D40932505509326056093B5
:10AD000027057093280590912305809122059923AA
:10AD100009F473C0882309F40ECDA85BBF4F8D9151
:10AD20009C91A0E0B0E0409111025091120260911C
:10AD300013027091140284179507A607B70709F04C
:10AD40005FC0F9CCB695A79597958795D988DD0C06
:10AD5000D98A2C5F3F4F49E12F30340709F04ECCA0
:10AD600059895093240580329105A105B10520F43D
:10AD700080E290E0A0E0B0E08097A109B1098115E0
:10AD800058E09507A105B10508F443C074E0979F0A
:10AD9000900111242D503B4EF9013296459154916A
:10ADA000EE27859FB001849F610D7E1F06946E1F64
:10ADB0007E1F1124F901C590D490E12CF12CC61A04
:10ADC000D70AE108F1088091190590911A05A09120
:10ADD0001B05B0911C058C0D9D1DAE1DBF1D8093E4
:10ADE000190590931A05A0931B05B0931C0580913B
:10ADF0002305811130C080912205882309F49BCC62
:10AE00001092150210921602109217021092180258
:10AE100092CCAC01BD017695679557954795FA019F
:10AE2000EC7F9F012D503F4EF901C590D490F90160
:10AE30003296459154918770849F9001859F300D83
:10AE40001124F3E036952795FA95E1F7C21AD30A53
:10AE5000E12CF12CB8CF8989480E511C611C711C62
:10AE60008091390590913A05481459046A047B048D
:10AE7000D8F420912205222309F45DCCFC01E85B83
:10AE8000FF4F20813181A90160E070E00091110243
:10AE900010911202209113023091140240175107B1
:10AEA0006207730709F447CC10921502109216023C
:10AEB0001092170210921802FC01E85BFF4F80818C
:10AEC0009181A0E0B0E08093110290931202A093D0
:10AED0001302B09314022FCCD701C601B695A795E3
:10AEE00097958795FC01EC7FCF018D509F4EFC011B
:10AEF00025913491FC013296459154916C2D6770E7
:10AF0000649FC001659F900D112463E0969587951D
:10AF10006A95E1F7281B390BC901A0E0B0E0FBCB33
:10AF2000D501C401B695A79597958795FC01EC7F4F
:10AF3000CF018D509F4EFC01C590D490FC013296FC
:10AF400025913491482D4770429FC001439F900D39
:10AF50001124A3E096958795AA95E1F7C81AD90A16
:10AF6000E12CF12CD4CD80EDC82E87E0D82EE12C39
:10AF7000F12CE8CBCF92DF92EF92FF920F931F93C9
:10AF8000CF93DF936C017A018B01C0E0D0E0CE1546
:10AF9000DF0581F0D8016D918D01D601ED91FC9115
:10AFA0000190F081E02DC6011995892B11F02196B1
:10AFB000EECF7E01C701DF91CF911F910F91FF90DE
:10AFC000EF90DF90CF900895FF920F931F93CF9350
:10AFD000DF938C01EB01F42E80E20E94679A8FEFE1
:10AFE000F81611F084E501C082E40E94679A8AE3B2
:10AFF0000E94679AF801608171818281938142E0A9
:10B000000E94289E488159816A817B8187EB9BE160
:10B010000E9461C662E070E080E090E0DF91CF9135
:10B020001F910F91FF900C9444BB8F929F92AF920F
:10B03000BF92CF92DF92EF92FF920F931F93CF9325
:10B04000DF93F0E2FF2EE12CAE2DB0E0BD016F0DDD
:10B05000711D759567956E1511F0F6120BC0E1E93B
:10B06000F9E165917491072E000C880B990B0E94F1
:10B0700054EF62C09B0121503109220F331F220F70
:10B08000331FF901ED5EF64E05911491AB01440FAB
:10B09000551F440F551FFA01ED5EF64EC591D49130
:10B0A0008017910714F4F62ED1CFC817D90714F4DE
:10B0B000E62ECACFF901EB5EF64EE590F490FA0168
:10B0C000EB5EF64EC590D490BC01601B710B072E51
:10B0D000000C880B990B0E9454EF4B015C01B601E8
:10B0E0006E197F09072E000C880B990B0E9454EFF4
:10B0F0009B01AC01C501B4010E94B3EF4B015C019F
:10B10000C01BD10BBE01DD0F880B990B0E9454EFC1
:10B110009B01AC01C501B4010E94A7F44B015C0185
:10B12000B701FF0C880B990B0E9454EF9B01AC01F7
:10B13000C501B4010E94CBF3DF91CF911F910F9114
:10B14000FF90EF90DF90CF90BF90AF909F908F9047
:10B1500008950F931F93CF93DF93CDB7DEB7289752
:10B160000FB6F894DEBF0FBECDBF6091480470915A
:10B170004904072E000C880B990B0E9454EF6D8335
:10B180007E838F83988780915C0490915D04A09169
:10B190005E04B0915F0489839A83AB83BC834DEFD7
:10B1A000BE016B5F7F4FCE0101960EDF60914204BE
:10B1B00070914304072E000C880B990B0E9454EFEA
:10B1C0006D837E838F83988780914404909145049A
:10B1D000A0914604B091470489839A83AB83BC83D2
:10B1E0004FEFBE016B5F7F4FCE010196EDDEEFEBBF
:10B1F000FBE184918F010F5F1F4F882321F00E9494
:10B20000679AF801F6CFE0917805F0E0EA58FA4F36
:10B21000608170E080E090E00E940E9EEAEBFBE12E
:10B2200084918F010F5F1F4F882321F00E94679A3E
:10B23000F801F6CF6091770570E080E090E00E9421
:10B240000E9E28960FB6F894DEBF0FBECDBFDF91DD
:10B25000CF911F910F9108950F930FB70F93009106
:10B260006E000B7F00936E0078940F930BB70F93D3
:10B270000CB70F921F922F933F934F935F936F934F
:10B280007F938F939F93AF93BF93EF93FF9311247B
:10B29000F0D1FF91EF91BF91AF919F918F917F91ED
:10B2A0006F915F914F913F912F911F900F900CBF25
:10B2B0000F910BBF0F910460F89400936E000F91F3
:10B2C0000FBF0F911895CF92DF92EF92FF92C0902F
:10B2D0004404D0904504E0904604F0904704609107
:10B2E00042047091430466507109072E000C880BCC
:10B2F000990B0E9454EF9B01AC01C701B6010E945B
:10B300004EEF87FF1FC020E030E040E050E4C7016F
:10B31000B6010E94CBF30E9414F57093A8056093C8
:10B32000A7050E946762DC01CB01805A9541AF4FAF
:10B33000BF4F8093A3059093A405A093A505B09358
:10B34000A60508C01092A3051092A4051092A505A9
:10B350001092A605FF90EF90DF90CF900895CF92C6
:10B36000DF92EF92FF92C0905C04D0905D04E09079
:10B370005E04F0905F046091480470914904675046
:10B380007109072E000C880B990B0E9454EF9B014A
:10B39000AC01C701B6010E944EEF87FF1FC020E03D
:10B3A00030E040E450E4C701B6010E94CBF30E94B4
:10B3B00014F57093A2056093A1050E946762DC01F9
:10B3C000CB01805A9541AF4FBF4F80939D0590931D
:10B3D0009E05A0939F05B093A00508C010929D05FF
:10B3E00010929E0510929F051092A005FF90EF907D
:10B3F000DF90CF90089520912202309123022F50A8
:10B400003109821793070CF49C013093490420936F
:10B41000480480E0A4CF1092720580E090E0EBDF5A
:10B4200010924304109242044EDF0E94F9C680E05D
:10B4300090E0E1DF109276052C9810924304109270
:10B44000420410927705809102018072809300017E
:10B4500008958F929F92AF92BF92CF92DF92EF9218
:10B46000FF920F931F93CF93DF93F0E4FF2EE12C15
:10B47000AE2DB0E0BD016F0D711D759567956E1510
:10B4800011F0F6120BC0ECE0FBE165917491072E10
:10B49000000C880B990B0E9454EF62C09B01215055
:10B4A0003109220F331F220F331FF901E25FF54EDE
:10B4B00005911491AB01440F551F440F551FFA011C
:10B4C000E25FF54EC591D4918017910714F4F62EE2
:10B4D000D1CFC817D90714F4E62ECACFF901E05F1F
:10B4E000F54EE590F490FA01E05FF54EC590D490EA
:10B4F000BC01601B710B072E000C880B990B0E947E
:10B5000054EF4B015C01B6016E197F09072E000C48
:10B51000880B990B0E9454EF9B01AC01C501B4014B
:10B520000E94B3EF4B015C01C01BD10BBE01DD0FCC
:10B53000880B990B0E9454EF9B01AC01C501B4012B
:10B540000E94A7F44B015C01B701FF0C880B990B1B
:10B550000E9454EF9B01AC01C501B4010E94CBF3E2
:10B56000DF91CF911F910F91FF90EF90DF90CF90DF
:10B57000BF90AF909F908F90089560E08091B40548
:10B580009091B50552DD60935C0470935D048093E7
:10B590005E0490935F048091B2059091B30559DFEA
:10B5A0006093440470934504809346049093470449
:10B5B000A895109273050895DF92EF92FF920F9372
:10B5C0001F93CF93DF93F82ED62EE72E8A0180911A
:10B5D0001902882309F439C0E5E5F4E28491EF010A
:10B5E0002196882321F00E94679AFE01F7CFED2D66
:10B5F000FE2D8491EF012196882321F00E94679A05
:10B60000FE01F7CFE4EAF9E18491EF012196882366
:10B6100021F00E94679AFE01F7CFF7FC0BC06F2D57
:10B62000FF0C770B880B990B0E940E9E8AE00E94FC
:10B63000679A0BC0EFE9F9E18491EF012196882325
:10B6400021F00E94679AFE01F7CF80917905811160
:10B6500008C01092190281E080937905C8010E9408
:10B6600027AEDF91CF911F910F91FF90EF90DF9068
:10B67000D2CE0F931F93CF93DF9380911C028F370D
:10B68000A0F08F57909176059093C505992311F0FE
:10B690002C9A01C02C98209177052093C405909195
:10B6A0000201222369F090950BC09091C50589177E
:10B6B00008F02C989091C405891728F09091020108
:10B6C0009072909300018F5F80931C029091C3054C
:10B6D00081E089278093C30580911B0285301CF48B
:10B6E000C1E0C80F01C0C0E0823009F4B8C054F412
:10B6F000882301F1813009F0E7C088E080937B0066
:10B7000085E4C4C0843009F4C9C00CF4BBC08530E2
:10B7100009F0DAC09091C205911102C08093C20570
:10B720008091C20581508093C205882309F4CCC062
:10B73000C5E0CAC080911A028F5F80311CF48093EB
:10B740001A02C2C010921A0280917305811113C0AF
:10B750008091B8059091B9059093B5058093B40593
:10B760008091B6059091B7059093B3058093B2058B
:10B7700081E0809373058AE0E8EBF5E0DF011D923C
:10B780008A95E9F71092B7051092B6050091B405B5
:10B790001091B5051195019511098091480490917A
:10B7A0004904D1E0181619062CF080917605811114
:10B7B00001C0D0E08091D0059091D10591958195FF
:10B7C00091098017910734F445E45BE166E67BE17B
:10B7D00080E0F2DE80912002909121029195819586
:10B7E00091090817190744F4DD2331F048E75BE1BC
:10B7F00069E97BE180E0E0DE8091420490914304BE
:10B8000011E0181619062CF080917705811101C0FE
:10B8100010E02091B2053091B3058091CE05909152
:10B82000CF058217930734F045E55BE166E67BE1DF
:10B830008FEFC2DE20911E0230911F028091B2056F
:10B840009091B305821793070CF43EC01123E1F1E8
:10B8500048E85BE169E97BE18FEFAEDE35C08091BE
:10B860007A0086FD2EC08091780090917900209119
:10B87000B8053091B905820F931F9093B905809355
:10B88000B80522C088E080937B0086E480937C002A
:10B8900080917A00806480937A0016C080917A004B
:10B8A00086FD11C080917800909179002091B605B5
:10B8B0003091B705820F931F9093B7058093B6051B
:10B8C00003C0C2E001C0C4E0C0931B020E94DCD1EF
:10B8D0008091740590917505009799F00197909368
:10B8E000750580937405892B61F48BEA9BE1909335
:10B8F0004B0480934A04DF91CF911F910F910C94D8
:10B90000CF9ADF91CF911F910F9108952F923F927F
:10B910004F925F926F927F928F929F92AF92BF925F
:10B92000CF92DF92EF92FF920F931F93CF93DF930B
:10B9300000D01F92CDB7DEB75C017A8369831A010C
:10B9400007FD0DC0802F002E000C990B9C838B836C
:10B95000FC01E952FF4E80818823E1F008C080910C
:10B96000B105882399F0E1E0F0E0FC83EB83F50179
:10B970001082EB81FC81EE0FFF1FEE0FFF1FE755DA
:10B98000FA4F108211821282138230C081E090E05F
:10B990009C838B83F90140805180628073808B810E
:10B9A0009C81880F991F880F991F9C0127553A4F3A
:10B9B0004901A3019201F401608171818281938127
:10B9C0000E944EEF882391F0F401408251826282FE
:10B9D000738211E020E030E0A901C301B2010E94AE
:10B9E000F1F518160CF010E0F5011083F5018081D7
:10B9F0008230F1F0833009F464C0813009F082C0F4
:10BA0000EB81FC81EE0FFF1FEE0FFF1FE755FA4F92
:10BA10002081318142815381F10160817181828174
:10BA200093810E944EEF87FD6DC082E0F501808317
:10BA30002B813C81220F331F220F331F27553A4F92
:10BA40003C832B83B60180E090E00E9452EF9B0183
:10BA5000AC01EB81FC8160817181828193810E94C4
:10BA6000CAF39B01AC01F1016081718182819381F4
:10BA70000E94F1F587FD13C02AD54B015C019701A7
:10BA8000A8EEB3E00E94BBF3860E971EA81EB91E57
:10BA9000E981FA8180829182A282B38233C017D574
:10BAA000E981FA81C080D180E280F380DC01CB01A2
:10BAB0008C199D09AE09BF09B7FD24C083E0F501CB
:10BAC00080830F3F19F04EE05BE102C041E25BE191
:10BAD00065E37BE1802F0F900F900F900F90DF9127
:10BAE000CF911F910F91FF90EF90DF90CF90BF907B
:10BAF000AF909F908F907F906F905F904F903F900E
:10BB00002F905ACD0F900F900F900F90DF91CF9103
:10BB10001F910F91FF90EF90DF90CF90BF90AF906B
:10BB20009F908F907F906F905F904F903F902F905D
:10BB300008957F928F929F92AF92BF92CF92DF92A1
:10BB4000EF92FF920F931F93CF93DF9320E030E0AB
:10BB500048E452E460915C0470915D0480915E045D
:10BB600090915F040E94F1F518164CF4E9E9F9E1AF
:10BB7000E491C1E001C0CC0FEA95EAF701C0C0E052
:10BB800083E9E82E89E1F82E09E919E196E0A92E6A
:10BB9000912CD0E0CC24C394D12CF7017490F801FF
:10BBA000849077FC23C0892D90E0082C02C09595E5
:10BBB00087950A94E2F780FD19C0BE01082C02C0E7
:10BBC000759567950A94E2F76170B62EB1946B2D66
:10BBD000872D0E9413BA6B2D70E0872D0E947DBACD
:10BBE000C60101C0880F8A94EAF7982AAA94FFEF49
:10BBF000EF1AFF0A0F5F1F4FA110CFCFDF91CF9138
:10BC00001F910F91FF90EF90DF90CF90BF90AF907A
:10BC10009F908F907F9008954F925F926F927F9246
:10BC20008F929F92AF92BF92CF92DF92EF92FF924C
:10BC30000F931F93CF93DF93CDB7DEB760970FB607
:10BC4000F894DEBF0FBECDBF80917105811138C160
:10BC500080917305811117C060960FB6F894DEBF0E
:10BC60000FBECDBFDF91CF911F910F91FF90EF904D
:10BC7000DF90CF90BF90AF909F908F907F906F900C
:10BC80005F904F90089579DC22D44B015C01809144
:10BC9000D710811117C08091BC109091BD10A09158
:10BCA000BE10B091BF100097A105B10559F0A501D4
:10BCB0009401281B390B4A0B5B0B57FD03C081E035
:10BCC0008093D7106091480470914904072E000CAE
:10BCD000880B990B0E9454EF69837A838B839C8332
:10BCE00044E1C42ED12C5CE3E52EF12C00E09E0152
:10BCF0002F5F3F4F4CE554E069E975E088E995E036
:10BD000005DE40905C0450905D0460905E0470908D
:10BD10005F046091D2057091D305072E000C880B4B
:10BD2000990B0E9454EF9B01AC01C301B2010E9428
:10BD3000F1F518160CF4C8C060E0609376058091A8
:10BD40009D0590919E05A0919F05B091A00500973B
:10BD5000A105B10521F1A5019401281B390B4A0B5E
:10BD60005B0B57FD1CC06091A1057091A20580E09E
:10BD700090E00E9452EF9B01AC0160915C047091D5
:10BD80005D0480915E0490915F040E944EEF87FFF6
:10BD90004BC244EE59E166EF79E180E00DDC809121
:10BDA0006D0590916E05A0916F05B0917005A5018C
:10BDB0009401281B390B4A0B5B0B57FD0FC0B9DEF2
:10BDC000D501C4018C53964FAF4FBF4F80936D0583
:10BDD00090936E05A0936F05B09370058091A305B5
:10BDE0009091A405A091A505B091A6050097A10585
:10BDF000B10511F1881A990AAA0ABB0AB7FC1CC03E
:10BE00006091A7057091A80580E090E00E9452EF34
:10BE10009B01AC01609144047091450480914604FB
:10BE2000909147040E944EEF87FF3BC142EC59E1DD
:10BE300065ED79E18FEFC0DB6091420470914304BE
:10BE4000072E000C880B990B0E9454EF69837A83AC
:10BE50008B839C8395E0C92ED12C24E1E22EF12C1A
:10BE60000FEF9E012F5F3F4F44E454E063E975E01C
:10BE700087E995E04BDD8091B10581110FC1C0903C
:10BE80004404D0904504E0904604F090470420E03C
:10BE900030E040EA50E4C701B6010E94F1F587FDA9
:10BEA0000BC020E030E040EF52E4C701B6010E9431
:10BEB0004EEF18160CF0F7C060E060937705CCCE1B
:10BEC00085E09AE10E9427AE6091220270912302E0
:10BED000072E000C880B990B0E9454EF9B01AC01BC
:10BEE000C301B2010E944EEF87FF26CF00914804A4
:10BEF0001091490420ED3CEC4CE45DE36091690550
:10BF000070916A0580916B0590916C050E94B3EF6A
:10BF10006B017C0120918F05309190054091910536
:10BF200050919205C301B2010E94CAF39B01AC017A
:10BF3000C701B6010E94B3EF6B017C0123E333E339
:10BF400043E75FE360918B0570918C0580918D05CF
:10BF500090918E050E94B3EF9B01AC01C701B60121
:10BF60000E94CBF36B017C0160938B0570938C0571
:10BF700080938D0590938E0540928F055092900589
:10BF800060929105709292058091D71081114FC1F6
:10BF9000B801012E000C880B990B0E9454EFA301ED
:10BFA00092010E94CAF32B013C0120E030E040E204
:10BFB00051E40E94F1F518160CF44AC120E030E07B
:10BFC00040E251ECC301B2010E944EEF87FD2FC148
:10BFD000012B09F42CC180918A05811170C18091D7
:10BFE000860590918705A0918805B09189058D837C
:10BFF0009E83AF83B8872091650530916605409197
:10C00000670550916805C301B2010E94B3EF6987CB
:10C010007A878B879C87A30192016D817E818F81B6
:10C0200098850E94CBF36D837E838F83988760937E
:10C0300086057093870580938805909389052091E4
:10C0400061053091620540916305509164050E943D
:10C05000B3EF29853A854B855C850E94CBF3A70118
:10C0600096010E94CAF36B017C0120E030E04FE7AB
:10C0700053E40E94F1F520E030E0A90118160CF419
:10C0800006C1C701B6010E944EEF87FD1FC1C7015F
:10C09000B6010E940FF5759567954FCE1092770502
:10C0A000DBCD11D9C9CE6091420470914304072EB3
:10C0B000000C880B990B0E9454EFA70196010E9477
:10C0C000CAF34B015C0120915D0530915E05409102
:10C0D0005F05509160050E94B3EF69877A878B876F
:10C0E0009C87209182053091830540918405509171
:10C0F0008505C501B4010E94CBF36D837E838F83D8
:10C10000988760938205709383058093840590934C
:10C1100085052091590530915A0540915B05509154
:10C120005C050E94B3EF6D877E878F87988B20ED2B
:10C130003CEC4CE45DE360915505709156058091AF
:10C140005705909158050E94B3EF2B013C012091B7
:10C150007E0530917F054091800550918105C70192
:10C16000B6010E94CAF39B01AC01C301B2010E9457
:10C17000B3EF2B013C0123E333E343E75FE360913B
:10C180007A0570917B0580917C0590917D050E94D8
:10C19000B3EF9B01AC01C301B2010E94CBF32B01B1
:10C1A0003C0160937A0570937B0580937C059093A6
:10C1B0007D05C0927E05D0927F05E0928005F092C9
:10C1C00081052D853E854F85588969857A858B85C2
:10C1D0009C850E94CBF3A30192010E94CAF36B01DC
:10C1E0007C0120E030E04FE753E40E94F1F520E0CD
:10C1F00030E0A9011816FCF4C501B4010E94F1F564
:10C20000181684F4A50194016D817E818F81988533
:10C210000E94CAF36093820570938305809384051E
:10C22000909385056FE749CE80E099D8B8CD81E03D
:10C2300080938A0581CDC701B6010E944EEF87FD2C
:10C240000CC0C701B6010E940FF57595679535CEF4
:10C2500081E080938A056FE770CD20E030E0A9018E
:10C26000C501B4010E944EEF87FF26CEA5019401BF
:10C270006D817E818F8198850E94CAF360938205CB
:10C2800070938305809384059093850515CEC30133
:10C29000B2010E94F1F51816F4F6A30192016D8126
:10C2A0007E818F8198850E94CAF360938605709382
:10C2B000870580938805909389056FE73ECD10929E
:10C2C0008A051D821E821F82188695CE20E030E0EE
:10C2D000A901C301B2010E944EEF87FF2DCDA3013A
:10C2E00092016D817E818F8198850E94CAF360934F
:10C2F00086057093870580938805909389051CCDEA
:10C30000CF92DF92EF92FF926B017C0183E3C8161C
:10C31000D104E104F10468F082E3C81AD108E1080D
:10C32000F10862E370E080E090E00E9444BB74DCBE
:10C33000EDCFC701B6010E9444BBFF90EF90DF90A4
:10C34000CF906ACC0F931F9380915405813011F4E4
:10C35000BED008C060915005709151058091520582
:10C360009091530500914C0510914D0520914E057B
:10C3700030914F05601B710B820B930B28EE33E05D
:10C3800040E050E00E946DF380914805909149058E
:10C39000A0914A05B0914B05BC01CD01620F731FFE
:10C3A000841F951F1F910F910895109254051092AC
:10C3B0004C0510924D0510924E0510924F051092AB
:10C3C000500510925105109252051092530510928B
:10C3D00048051092490510924A0510924B050895A0
:10C3E00080915405813071F482E0809354056FD0C0
:10C3F00060935005709351058093520590935305B7
:10C4000081E0089580E0089590916F00292F2270B7
:10C4100091FF05C090916F009D7F90936F0034E075
:10C42000839FC0011124FC01EA51FF4E40815181DC
:10C4300062817381FC01E45CFA4F40835183628323
:10C44000738381E080933B05222329F080916F0064
:10C45000826080936F000895BC012091390530916E
:10C460003A054091390550913A052417350711F0E6
:10C470009A01F7CF81E02617370709F080E0089589
:10C480000E94DBF63FB7F89480917E0790917F077A
:10C49000A0918007B091810726B5A89B05C02F3FCA
:10C4A00019F00196A11DB11D3FBFBA2FA92F982FDA
:10C4B0008827820F911DA11DB11DBC01CD0142E055
:10C4C000660F771F881F991F4A95D1F708952FB7D8
:10C4D000F89460917A0770917B0780917C07909126
:10C4E0007D072FBF08951F920F920FB60F92112450
:10C4F0002F933F938F939F93AF93BF9380917A072E
:10C5000090917B07A0917C07B0917D0730917907CE
:10C5100023E0230F2D3720F40196A11DB11D05C086
:10C5200026E8230F0296A11DB11D20937907809361
:10C530007A0790937B07A0937C07B0937D07809147
:10C540007E0790917F07A0918007B09181070196A7
:10C55000A11DB11D80937E0790937F07A093800754
:10C56000B0938107BF91AF919F918F913F912F9190
:10C570000F900FBE0F901F9018951F920F920FB63D
:10C580000F9211240BB60F922F933F934F935F930B
:10C590006F937F938F939F93AF93BF93EF93FF938B
:10C5A0008091C9059091CA05A091CB05B091CC05A9
:10C5B000892B8A2B8B2B59F19091C805E091C605E8
:10C5C000F091C7058081892780838091C90590916A
:10C5D000CA05A091CB05B091CC05181619061A060C
:10C5E0001B060CF056C08091C9059091CA05A09118
:10C5F000CB05B091CC050197A109B1098093C9057C
:10C600009093CA05A093CB05B093CC0542C080910E
:10C610001D02E3ECFBE1E4919FEF90931D02E230F9
:10C62000C9F050F4EE2399F0E13081F590916F005C
:10C630009D7F90936F002AC0E43019F1E0F0E5305F
:10C6400029F5909173009D7F909373001FC0109205
:10C650006E001CC0909170009D7F9093700091E0DF
:10C660009093B0009091B100987F94609093B10046
:10C670001092B3000BC0909171009D7F9093710058
:10C6800005C0909172009D7F9093720060E00E94BF
:10C6900013BAFF91EF91BF91AF919F918F917F91CD
:10C6A0006F915F914F913F912F910F900BBE0F9023
:10C6B0000FBE0F901F901895CF92DF92EF92FF92CE
:10C6C0000F931F93CF93DF93CDB7DEB7A0970FB62D
:10C6D000F894DEBF0FBECDBF80E090E0A0EAB0E4EA
:10C6E00089839A83AB83BC8380E090E0ADE4B3E4BC
:10C6F0008D839E83AF83B88780E090E0A0EAB1E4A9
:10C7000089879A87AB87BC8788E592E00E946E9AFA
:10C71000811195C185E40E94EB3F882381F00E943E
:10C72000B43F6B017C0120E030E0A9010E94F1F5EB
:10C7300087FF0BC0F7FAF094F7F8F09406C0C12C0D
:10C74000D12C80E8E82E80E4F82EF7FAF094F7F880
:10C75000F094C98ADA8AEB8AFC8A8AE50E9434401E
:10C76000882379F08AE50E943440882319F00E94DA
:10C77000B43F03C060E070E0CB0169877A878B87A4
:10C780009C8788E50E943440882379F088E50E94E0
:10C790003440882319F00E94B43F03C060E070E089
:10C7A000CB0169837A838B839C8389E50E94344023
:10C7B000882379F089E50E943440882319F00E948B
:10C7C000B43F03C060E070E0CB016D837E838F8354
:10C7D000988785E50E94EB3F882329F00E94B43FAB
:10C7E0006B017C010CC0E0918E1084E0E89FF001A9
:10C7F0001124E75EF64EC080D180E280F38020E015
:10C8000030E0A901C701B6010E94F1F587FF04C01D
:10C81000F7FAF094F7F8F094F7FAF094F7F8F09448
:10C82000CD8ADE8AEF8AF88E198E1A8E1B8E1C8EA8
:10C830008CE40E94EB3F882329F00E94B43F6B01F7
:10C840007C010CC0E0918E1094E0E99FF00111246E
:10C85000E35EF64EC080D180E280F38020E030E0DD
:10C86000A901C701B6010E94F1F587FF04C0F7FADC
:10C87000F094F7F8F094CD8EDE8EEF8EF8A282E47D
:10C880000E943440882321F00E94843F162F01C06B
:10C890001AE000915405AE014B5E5F4FBE016F5F21
:10C8A0007F4FCE0141960E9446B3882309F4C3C04E
:10C8B000EAE6F4E284917F019FEFE91AF90A8823FE
:10C8C00021F00E94679AF701F5CFE6E2F0E2849149
:10C8D0007F019FEFE91AF90A882321F00E94679AE5
:10C8E000F701F5CF61E0812F0E948A82F0DDDC0143
:10C8F000CB0180529C46AB4FBF4F8093BC109093AE
:10C90000BD10A093BE10B093BF101092D71083E05B
:10C910008093C51081E08093C4108091C410882357
:10C9200009F46FC060E0812F0E948A828091D71045
:10C93000882309F462C0EAE6F4E284917F019FEF64
:10C94000E91AF90A882321F00E94679AF701F5CFC6
:10C95000ECE0F0E284917F019FEFE91AF90A882365
:10C9600039F00E94679AF701F5CF81E00E946EAE20
:10C970008091C4108111F9CF1092BC101092BD109B
:10C980001092BE101092BF101092D7100E94AF5993
:10C990000E94CCB2EAE6F4E284917F019FEFE91AAB
:10C9A000F90A882321F00E94679AF701F5CFEDEE8E
:10C9B000FFE184917F019FEFE91AF90A811119C003
:10C9C00086DDDC01CB0180529C46AB4FBF4F80938C
:10C9D000BC109093BD10A093BE10B093BF101092E6
:10C9E000D71081E08093C41061E0812F0E948A8279
:10C9F00004C00E94679AF701DCCF81E00E946EAE0E
:10CA00008CCF81E08093C51080E090E0A8E4B2E490
:10CA10008D879E87AF87B88B80914F08882359F008
:10CA2000212FAE01435F5F4FBE01635E7F4FCE019A
:10CA300049960E9464B8013011F40E94B2C6A096D3
:10CA40000FB6F894DEBF0FBECDBFDF91CF911F911F
:10CA50000F91FF90EF90DF90CF900895CF92DF92EB
:10CA6000EF92FF920F931F93CF93DF9388E50E947D
:10CA7000EB3FD82E89E40E94EB3FC82E882319F0A3
:10CA80000E94843F1CC0DD20C1F00E94B43F20E022
:10CA900030E040E251E40E94CAF320E030E040EC94
:10CAA00051E40E94CBF32BEA3AEA4AEA5CE30E94A3
:10CAB000B3EF0E940FF5653010F01FEF01C0162F85
:10CAC00089E50E94EB3F082F8AE40E94EB3FC82FC4
:10CAD000882319F00E94843F1CC00023C1F00E94EB
:10CAE000B43F20E030E040E251E40E94CAF320E08D
:10CAF00030E040EC51E40E94CBF32BEA3AEA4AEAF8
:10CB00005CE30E94B3EF0E940FF5653010F0DFEF99
:10CB100001C0D62F8AE50E94EB3FE82E811105C0A7
:10CB200081E50E94EB3FF82E01C0F12CC11001C03D
:10CB3000C0E02C2F30E0D11001C000E0200F311DEB
:10CB40002130310521F4E1101AC0F11018C0E5E5DB
:10CB5000F4E28491EF012196811103C0EDECFFE135
:10CB600004C00E94679AFE01F4CF8491EF012196E0
:10CB7000882309F455C00E94679AFE01F6CF17FD7D
:10CB800002C0D7FF17C0E5E5F4E28491EF012196DA
:10CB9000811103C0EEEAFFE104C00E94679AFE0122
:10CBA000F4CF8491EF0121968823D1F10E94679AF6
:10CBB000FE01F7CF0E94B43F9B01AC01012F110F82
:10CBC000110BAD2FDD0FBB0BFF2099F085E0809F8F
:10CBD000F001819FF00D1124EA0FFB1FEE0FFF1FE4
:10CBE000EE0FFF1FED55F74E6081718182819381B9
:10CBF00003C060E070E0CB01E5E0E09FE001E19F71
:10CC0000D00D1124CA0FDB1FCC0FDD1FCC0FDD1F91
:10CC1000CD55D74E0E94CBF3688379838A839B835B
:10CC2000DF91CF911F910F91FF90EF90DF90CF9008
:10CC300008952F923F924F925F926F927F928F92C0
:10CC40009F92AF92BF92CF92DF92EF92FF920F939B
:10CC50001F93CF93DF93CDB7DEB761970FB6F894EC
:10CC6000DEBF0FBECDBF83E50E94EB3F882349F0B6
:10CC70000E94A53F182F811106C080E00E944085C8
:10CC800002C01091E01080914C0490914D04A0914D
:10CC90004E04B0914F0489839A83AB83BC83809107
:10CCA000500490915104A0915204B09153048D838B
:10CCB0009E83AF83B8878091540490915504A091CE
:10CCC0005604B091570489879A87AB87BC870E9426
:10CCD0001385882309F49AC083E40E94EB3F8823DC
:10CCE00009F494C00E94B43F1B012C0105E0612CA3
:10CCF000712C38EC388B82EC898BA12CB12C98EC00
:10CD00009E87E2E4EF87015080F125E02D87209F88
:10CD1000400111243D8531503D873F3FA1F3F4018F
:10CD2000E30FF11DEE0FFF1FEE0FFF1FED55F74E46
:10CD3000C080D180E280F3809601A701B5018E8585
:10CD40009F850E94F1F518161CF45601EE86FF86A9
:10CD50009601A701B301888999890E944EEF87FF48
:10CD6000D9CF3601E88AF98AD5CF93014889598904
:10CD7000B5018E859F850E94CBF320E030E040E036
:10CD80005FE30E94B3EFA20191010E94CBF32B015C
:10CD90003C012DEB37E346E855EB0E94F1F587FDAA
:10CDA0000AC02DEB37E346E855E3C301B2010E9408
:10CDB0004EEF18165CF580E00E94408535E0D32EDA
:10CDC00045E0C42EDA949FEFD91601F105E0CD9C21
:10CDD000500111240150B0F37501E00EF11CC701A0
:10CDE000880F991F880F991FFC01ED55F74E7F01A1
:10CDF000A301920160817181828193810E94CAF3B3
:10CE0000F7016083718382839383E4CF86E50E9478
:10CE1000EB3F882399F00E941385882379F0E8E995
:10CE2000FFE184917F012FEFE21AF20A882321F0BB
:10CE30000E94679AF701F5CF0E9419D18AE50E94F6
:10CE4000EB3F882321F00E94B43F0E949BB7812FC3
:10CE50000E944085111103C0EAE6F4E21CC08091F3
:10CE6000E0108111F9CFE5E5F4E284918F010F5FC5
:10CE70001F4F882321F00E94679AF801F6CFE9E757
:10CE8000FFE184918F010F5F1F4F882329F30E94D8
:10CE9000679AF801F6CF84918F010F5F1F4F8823A7
:10CEA00021F00E94679AF801F6CF8091E01081117D
:10CEB00003C067E173E002C063E173E08BE69FE1CA
:10CEC0000E9497C68AE00E94679AEAE6F4E284919B
:10CED0008F010F5F1F4F882321F00E94679AF8018E
:10CEE000F6CFEEE5FFE184918F010F5F1F4F88239E
:10CEF00021F00E94679AF801F6CFC090E110D0901F
:10CF0000E210E090E310F090E41020E030E0A9019E
:10CF1000C701B6010E94F1F518164CF442E0C701B2
:10CF2000B6010E94289E8AE00E94679A0CC0E9E53B
:10CF3000FFE184918F010F5F1F4F882321F00E9432
:10CF4000679AF801F6CF4CE050E06CE474E0CE0153
:10CF500001960E94E7F6892BD1F061960FB6F894FE
:10CF6000DEBF0FBECDBFDF91CF911F910F91FF901C
:10CF7000EF90DF90CF90BF90AF909F908F907F9079
:10CF80006F905F904F903F902F900C94E07E619651
:10CF90000FB6F894DEBF0FBECDBFDF91CF911F91CA
:10CFA0000F91FF90EF90DF90CF90BF90AF909F9048
:10CFB0008F907F906F905F904F903F902F9008954B
:10CFC00080916F00982F927081FF05C080916F0053
:10CFD0008D7F80936F0080915F0A80935E0A8093BB
:10CFE0005D0A80935C0A84E680935B0A28EE33E056
:10CFF0003093750520937405992329F080916F0073
:10D00000826080936F0081E080933B050E94CF7E19
:10D010000E946CC38091E010882321F08BEC91E199
:10D020000E9479C78CE0EBECF1E1ACE4B4E0019054
:10D030000D928A95E1F70C942E992F923F924F9280
:10D040005F926F927F928F929F92AF92BF92CF9298
:10D05000DF92EF92FF920F931F93CF93DF93CDB7A1
:10D06000DEB7CD54D1090FB6F894DEBF0FBECDBFE9
:10D0700085E40E943440882321F00E94843F8B0184
:10D0800002C000E010E083E40E943440882321F0D5
:10D090000E94843F6AA302C025E02AA385E50E947E
:10D0A0003440882319F00E94A53F03C085E50E9403
:10D0B000EB3F8CA717FD07C0C12CD12CB6E1EB2E9E
:10D0C000B3E4FB2E06C0C12CD12CACE8EA2EA2E4BE
:10D0D000FA2E83E50E943440882321F00E94B43F59
:10D0E0006B017C010115110511F410927805109265
:10D0F000C510102FECD92B013C01302F331F3327E3
:10D10000331F83E0831B8983D301C2018C53964F65
:10D11000AF4FBF4F80936D0590936E05A0936F0541
:10D12000B09370050F5F023080F0EFE2FFE1849171
:10D13000AF014F5F5F4F5A834983882309F472C35D
:10D140000E94679AE981FA81F2CF17FD12C0E12FA0
:10D15000EE0FFF0BEE5DFD4F608171816F50710925
:10D16000072E000C880B990B0E9454EF4B015C01B9
:10D1700006C0812C912CF2EDAF2EF2E4BF2EC70138
:10D18000B6010E940FF5072E000C880B990B0E9428
:10D1900054EF69877A878B879C87A50194010E9449
:10D1A000F1F518167CF4E0EFFEE18491DF011196B1
:10D1B000BA83A983882309F435C30E94679AE98159
:10D1C000FA81F3CFEBE1FFE184917F01BFEFEB1A2E
:10D1D000FB0A882321F00E94679AF701F5CF0E948D
:10D1E0000B5A17FF04C08FE78093770508C0E12F23
:10D1F000012E000CFF0BEA58FA4F8FE78083E9817C
:10D200008E2F90E0A3019201205A35414F4F5F4F7E
:10D210002EAB3FAB48AF59AF21E0209324021F3F14
:10D2200049F44AE55EE15BAF4AAFA4E2BEE1BDAFBF
:10D23000ACAF08C0E8E4FEE1FBAFEAAF21E13EE1BC
:10D240003DAF2CAF4CA25DA26EA27FA24DA65EA602
:10D250006FA678AA19AA1AAA1BAA1CAA1DAA2A96FE
:10D260001FAE2A9730E4398F4CE14A8F56E45B8F2A
:10D270001C8E1D8E1E8E1F8E1D8A1E8A1F8A188E62
:10D28000198A1A8A1B8A1C8A19821A821B821C829A
:10D290002FE730E040E050E02D833E834F835887F6
:10D2A0007FE7C72ED12CE12CF12C18A619A61AA6BF
:10D2B0001BA631E03D87188A1F8629961FAE299745
:10D2C000212C312C00E0212F012E000C330BA90161
:10D2D0004A585A4F5FAF4EAF220F331F220F331FF2
:10D2E000D901A45ABB4FB9A3A8A39C01092E000CD5
:10D2F000440B550B24962CAF3DAF4EAF5FAF249738
:10D3000004969C01990F440B550B28962CAF3DAF0A
:10D310004EAF5FAF28974AA1042E000C550B5BA3BC
:10D320004AA380912402882309F47AC2D0D84B0101
:10D330005C0180917305882309F4D8C00E94BD5A0E
:10D3400017FD0CC0A8A1B9A1BC912996BFAF299720
:10D35000E8A1F9A12180328003810BC0F09144043F
:10D360002996FFAF299720904504309046040091FC
:10D37000470429962FAD2997322D432D502F6C8DC0
:10D380007D8D8E8D9F8D0E944EEF87FF07C0299661
:10D390002FAD29972C8F2D8E3E8E0F8F2A962FAD75
:10D3A0002A97398D4A8D5B8D29966FAD2997722DFD
:10D3B000832D902F0E944EEF87FF09C029963FAD25
:10D3C00029972A963FAF2A97298E3A8E0B8F809104
:10D3D0006D0590916E05A0916F05B0917005A50146
:10D3E0009401281B390B4A0B5B0B57FD10C00E94A0
:10D3F000995DD501C4018C53964FAF4FBF4F8093B9
:10D400006D0590936E05A0936F05B09370053D85F3
:10D4100029962FAD2997332309F44BC0322D432D84
:10D42000502F69857A858B859C850E944EEF87FFFA
:10D430005DC0D501C40184199509A609B7092E96C6
:10D440008CAF9DAFAEAFBFAF2E9788589341A10967
:10D45000B109B7FD4BC0D701C6012D813E814F8177
:10D460005885821B930BA40BB50BB595A795979583
:10D47000879517FF03C08093770503C0EEADFFAD1E
:10D4800080832E962CAD3DAD4EAD5FAD2E9728A777
:10D4900039A74AA75BA739853C8F4A854D8F5B85A5
:10D4A0005E8F8C858F8F8CA29DA2AEA2BFA21D869F
:10D4B0001DC0322D432D502F69857A858B859C8523
:10D4C0000E94F1F5181694F4D501C4012CA13DA1D8
:10D4D0004EA15FA1821B930BA40BB50BAC01BD0148
:10D4E000485853416109710977FFB9C120E030E024
:10D4F00040EA51E469857A858B859C850E94CBF34F
:10D5000029962FAD2997322D432D502F0E944EEF93
:10D5100087FF0FC0ECE7FEE18491DF011196BA832B
:10D52000A983882309F47CC10E94679AE981FA8162
:10D53000F3CFD501C4012DA53EA54FA558A9821B47
:10D54000930BA40BB50BB7FD89C00E94A9588AE0C4
:10D550000E94679AD501C4018053984FAF4FBF4FC7
:10D560008DA79EA7AFA7B8AB99A991115AC02AA9B8
:10D570003BA94CA95DA929966FAD2997722D832DE2
:10D58000902F0E94F1F51816DCF524966CAD7DAD58
:10D590008EAD9FAD24970E9454EF29962FAD299709
:10D5A000322D432D502F0E94CBF36AAB7BAB8CAB5B
:10D5B0009DABA5019401205A35414F4F5F4F2EABD3
:10D5C0003FAB48AF59AF28966CAD7DAD8EAD9FADEA
:10D5D00028970E9454EF9B01AC0169857A858B8561
:10D5E0009C850E94CAF329962FAD2997322D432D91
:10D5F000502F0E944EEF881F8827881F89AB2EC0AE
:10D60000D501C4012EA93FA948AD59AD821B930B8A
:10D61000A40BB50BB7FD22C04AAD5BAD6DE67EE154
:10D620001AC020E030E040EA51E469857A858B85B4
:10D630009C850E94CAF39B01AC0129966FAD299786
:10D64000722D832D902F0E944EEF87FF07C04CADA7
:10D650005DAD68E37EE1812F0E94DC5AD501C401F3
:10D66000880F991FAA1FBB1F2CA13DA14EA15FA12E
:10D67000821B930BA40BB50B84199509A609B70956
:10D6800081309F49A442B10580F0E3EFFDE1849130
:10D69000AF014F5F5F4F5A834983882309F4C0C0AD
:10D6A0000E94679AE981FA81F2CF8AA19BA1AF8596
:10D6B000B8898A179B070CF034CEE6E9FDE1849126
:10D6C0003F01BFEF6B1A7B0A882321F00E94679A03
:10D6D000F301F5CF17FD05C0E6E1F3E0FE83ED832E
:10D6E00004C02CE034E03E832D836D817E8185E88B
:10D6F0009DE10E9497C649815A816B817C8181E8B6
:10D700009DE10E9461C68AE00E94679A6D817E81D8
:10D7100080E79DE10E9497C649895A896B897C8977
:10D720008CE69DE10E9461C68AE00E94679A6D8145
:10D730007E818BE59DE10E9497C64D895E896F8948
:10D74000788D87E59DE10E9461C68AE00E94679A14
:10D750003CA5332309F466C017FF31C089819A8143
:10D76000AB81BC8180935D0590935E05A0935F05BE
:10D77000B09360052CEA35EC47E25EE369897A896B
:10D780008B899C890E94B3EF6093590570935A0569
:10D7900080935B0590935C052CEA35EC47E25EE3F1
:10D7A0006D897E898F89988D0E94A7F460935505B5
:10D7B00070935605809357059093580533C029817F
:10D7C0003A814B815C8120936505309366054093D7
:10D7D0006705509368052CEA35EC47E25EE36989FA
:10D7E0007A898B899C890E94B3EF6093610570935D
:10D7F000620580936305909364052CEA35EC47E25B
:10D800005EE36D897E898F89988D0E94A7F460936D
:10D81000690570936A0580936B0590936C0502C04F
:10D820000E940B5A81E08093C510C35BDF4F0FB697
:10D83000F894DEBF0FBECDBFDF91CF911F910F9146
:10D84000FF90EF90DF90CF90BF90AF909F908F9020
:10D850007F906F905F904F903F902F9008954F85ED
:10D860005889452B09F437C148A459A46AA47BA45C
:10D87000480E591E6A1E7B1E28A539A54AA55BA520
:10D88000281B390B4A0B5B0B6D817E818F8198853C
:10D890000E945EF3A30192010E948FF3DA01C90195
:10D8A0008C0D9D1DAE1DBF1D84319105A105B105D7
:10D8B000FCF06C017D018C3E9105A105B1052CF0B9
:10D8C0005BEEC52ED12CE12CF12C80E8C816D104DA
:10D8D000E104F104DCF02EEF30E040E050E02C19E0
:10D8E0003D094E095F092D833E834F83588712C03F
:10D8F00044E1C42ED12CE12CF12C84E190E0A0E095
:10D90000B0E08D839E83AF83B88704C0CD82DE8272
:10D91000EF82F886E8EEFEE18491DF011196BE8782
:10D92000AD87882329F00E94679AED85FE85F4CFA4
:10D93000C701B6010E940E9EE3EEFEE184919F01B5
:10D940002F5F3F4F3E872D87882329F00E94679ADB
:10D95000ED85FE85F3CF6D817E818F8198850E9454
:10D960000E9E2A964FAD2A97598D6A8D7B8D8CED30
:10D970009EE10E9461C64C8D5D8D6E8D7F8D85ED23
:10D980009EE10E9461C64F855889433051050CF4D1
:10D99000A2C06D817E818F8198850E9454EF20E026
:10D9A00030E040E850E40E94B3EF69837A838B83D0
:10D9B0009C832A962FAD2A97398D4A8D5B8D6C8D6D
:10D9C0007D8D8E8D9F8D0E94CAF32BED3FE049E443
:10D9D00050E40E94B3EF20E030E040E05FE30E94BB
:10D9E000B3EF9B01AC0169817A818B819C810E949C
:10D9F000A7F469837A838B839C83C301B2010E945D
:10DA000054EF2FE632E143E85AE30E94B3EF2B01D3
:10DA10003C0149815A816B817C818FEC9EE10E949F
:10DA200061C6B301A20189EC9EE10E9461C62AE9A8
:10DA300039E949E15FE369817A818B819C810E94A8
:10DA4000B3EF69837A838B839C839B01AC010E9433
:10DA5000CBF3A30192010E94A7F4698B7A8B8B8B85
:10DA60009C8B29813A814B815C81C301B2010E9468
:10DA7000B3EF20E030E040E05EE30E94B3EF6D8B57
:10DA80007E8B8F8B988FE9EBFEE184913F015FEFF6
:10DA9000651A750A882321F00E94679AF301F5CF71
:10DAA00049815A816B817C8183EB9EE10E9461C632
:10DAB00049895A896B897C898DEA9EE10E9461C6F9
:10DAC0004D895E896F89788D87EA9EE10E9461C6E3
:10DAD0008AE00E94679A8D819E81AF81B8858C0D06
:10DAE0009D1DAE1DBF1DB595A7959795879517FFF1
:10DAF00003C08093770503C0EEADFFAD80832F8513
:10DB000038892F5F3F4F388B2F8739852A963FAF53
:10DB10002A974A85498F5B855A8F8C858B8F240184
:10DB2000350191E09D87E2CCCF93DF93EAE6F4E202
:10DB30008491EF012196882321F00E94679AFE01CB
:10DB4000F7CF83E50E94EB3F882321F00E94A53F99
:10DB500080933C02E7E4FDE18491EF012196882364
:10DB600021F00E94679AFE01F7CF80913C0281115B
:10DB700003C0E3E4FDE102C0EFE3FDE18491EF01C6
:10DB80002196882321F00E94679AFE01F7CFE7E3F0
:10DB9000FDE18491EF012196882321F00E94679A8C
:10DBA000FE01F7CF209124043091250440912604F2
:10DBB000509127046091821070918310809184109D
:10DBC000909185100E94CBF3AB01BC0185E39DE1F0
:10DBD0000E9461C6209128043091290440912A04B2
:10DBE00050912B046091861070918710809188105D
:10DBF000909189100E94CBF3AB01BC0182E39DE1BF
:10DC00000E9461C620912C0430912D0440912E0475
:10DC100050912F0460918A1070918B1080918C101C
:10DC200090918D100E94CBF3AB01BC018FE29DE17E
:10DC30000E9461C6E7E2FDE18491EF01219688230D
:10DC400021F00E94679AFE01F7CF209124043091C1
:10DC50002504409126045091270460912E02709172
:10DC60002F0280913002909131020E94CBF3AB01E0
:10DC7000BC0185E29DE10E9461C62091280430919B
:10DC8000290440912A0450912B0460913202709132
:10DC9000330280913402909135020E94CBF3AB01A4
:10DCA000BC0182E29DE10E9461C620912C0430916A
:10DCB0002D0440912E0450912F04609136027091F2
:10DCC000370280913802909139020E94CBF3AB0168
:10DCD000BC018FE19DE10E9461C68AE0DF91CF9196
:10DCE0000C94679AFF920F931F93CF93DF93F82EB4
:10DCF000092F162FEAE1FDE18491EF012196882397
:10DD000021F00E94679AFE01F7CFEF2DF02F84914A
:10DD1000EF012196882321F00E94679AFE01F7CF38
:10DD2000E8E1FDE18491EF012196882321F00E9432
:10DD3000679AFE01F7CF612F70E080E090E00E94CB
:10DD40000E9E8AE0DF91CF911F910F91FF900C946E
:10DD5000679A2F923F924F925F926F927F928F922B
:10DD60009F92AF92BF92CF92DF92EF92FF920F936A
:10DD70001F93CF93DF93CDB7DEB7C857D1090FB646
:10DD8000F894DEBF0FBECDBFE0917405F09175052C
:10DD9000EF2B11F00C946A772896DFAECEAE289761
:10DDA0006E2C79016A015B01FC0120813181428185
:10DDB00053816C962CAF3DAF4EAF5FAF6C97209107
:10DDC000F6103091F7104091F8105091F9106C96C0
:10DDD0006CAD7DAD8EAD9FAD6C970E94B3EF0E9490
:10DDE000FCF5E0966CAF7DAF8EAF9FAFE097D501AD
:10DDF0008D919D910D90BC91A02DA0968CAF9DAF63
:10DE0000AEAFBFAFA0972091FA103091FB104091B8
:10DE1000FC105091FD10BC01CD010E94B3EF0E9497
:10DE2000FCF5E4966CAF7DAF8EAF9FAFE497D60163
:10DE30002D913D914D915C91A4962CAF3DAF4EAF8D
:10DE40005FAFA4972091FE103091FF104091001118
:10DE500050910111A4966CAD7DAD8EAD9FADA49790
:10DE60000E94B3EF0E94FCF5E8966CAF7DAF8EAFD9
:10DE70009FAFE897D7012D913D914D915C912296EE
:10DE80002CAF3DAF4EAF5FAF229720910211309182
:10DE90000311409104115091051122966CAD7DAD96
:10DEA0008EAD9FAD22970E94B3EF0E94FCF5609665
:10DEB0006CAF7DAF8EAF9FAF60978091BA0783FF45
:10DEC0001CC060962CAD3DAD4EAD5FAD609720930C
:10DED000900A3093910A4093920A5093930A2296A3
:10DEE0008CAD9DADAEADBFAD22978093800A90936F
:10DEF000810AA093820AB093830AD801BC91B9A782
:10DF0000F801F181F9ABD8011296BC91BEABF801D2
:10DF1000F381FAAF80915E0A90915F0A891B8F703E
:10DF20008F3021F480E00E946EAEF4CF00915E0A43
:10DF3000E9960FAFE99780915E0A082F10E01CA3C5
:10DF40000BA38091840A9091850AA091860AB091D2
:10DF5000870AE0968CAC9DACAEACBFACE097881A5B
:10DF6000990AAA0ABB0A8091880A9091890AA0910D
:10DF70008A0AB0918B0AE4962CAC3DAC4EAC5FACF7
:10DF8000E497281A390A4A0A5B0A80918C0A909110
:10DF90008D0AA0918E0AB0918F0AE8962CAD3DAD06
:10DFA0004EAD5FADE897281B390B4A0B5B0B2DA3D9
:10DFB0003EA34FA358A78091900A9091910AA091F7
:10DFC000920AB091930A60960CAD1DAD2EAD3FAD97
:10DFD0006097081B190B2A0B3B0B0DA71EA72FA739
:10DFE00038AB012B022B032B09F4BCC08091D61057
:10DFF00081114BC060915C0470915D0480915E045E
:10E0000090915F040E940FF520913A0230913B02FB
:10E01000621773070CF039C060962CAD3DAD4EAD64
:10E020005FAD60972093900A3093910A4093920AD3
:10E030005093930A22968CAD9DADAEADBFAD2297A5
:10E040008093800A9093810AA093820AB093830AF6
:10E05000EAE6F4E284918F010F5F1F4F811103C044
:10E06000E1E7F0E204C00E94679AF801F3CF8491DF
:10E070008F010F5F1F4F882321F00E94679AF801DC
:10E08000F6CF1DA61EA61FA618AA94E0699E8001C1
:10E0900011240B5D1D4F6DA57EA58FA598A90E942B
:10E0A00054EFD8012D913D914D915C910E94B3EFB9
:10E0B0006B017C0120E030E0A9010E94F1F587FFAF
:10E0C00004C0F7FAF094F7F8F0946091021170919F
:10E0D000031180910411909105110E940FF59B018D
:10E0E000AC01A8E5B2E00E94ABF30E9454EFA70197
:10E0F00096010E944EEF87FF39C060960CAD1DADB2
:10E100002EAD3FAD60970093900A1093910A209333
:10E11000920A3093930A22962CAD3DAD4EAD5FAD81
:10E1200022972093800A3093810A4093820A509369
:10E13000830AEAE6F4E284918F010F5F1F4F811199
:10E1400003C0E2E5F0E204C00E94679AF801F3CF51
:10E1500084918F010F5F1F4F882321F00E94679ADF
:10E16000F801F6CF1DA61EA61FA618AAD501C40148
:10E170008827B7FD83959927AA27BB27782E57FEB6
:10E1800003C0382F3260732E8DA19EA1AFA1B8A518
:10E19000B7FF03C0972D9460792E0DA51EA52FA55E
:10E1A00038A937FF03C0172D1860712E24E0629E36
:10E1B000800111240B5D1D4F6DA57EA58FA598A92B
:10E1C0000E9454EFD8012D913D914D915C910E9498
:10E1D000B3EF6B017C0120E030E0A9010E94F1F572
:10E1E00087FF04C0C701B601905802C0C701B6013D
:10E1F00020E030E040E05FE30E94CBF30E9414F5A2
:10E200006AAB7BAB8CAB9DAB88E60BA11CA1809F5E
:10E21000F001819FF00D1124E55EFD4E1082EA5B56
:10E22000FF4F7082B501A401B7FE07C044275527F0
:10E23000BA01481959096A097B0988E60BA11CA192
:10E24000809FF001819FF00D1124E55EFD4E458B0E
:10E25000568B678B708F2C962CAE3DAE4EAE5FAE5C
:10E260002C9757FE0DC088279927DC018219930946
:10E27000A409B5092C968CAF9DAFAEAFBFAF2C975C
:10E2800028E60BA11CA1209FF001219FF00D112475
:10E29000E55EFD4E2C968CAD9DADAEADBFAD2C9721
:10E2A000818F928FA38FB48F0DA11EA12FA138A5AE
:10E2B00037FF07C030952095109501951F4F2F4FC0
:10E2C0003F4FE8E67E2EABA1BCA17A9EF0017B9E7B
:10E2D000F00D1124E55EFD4E058F168F278F30A3BC
:10E2E0008AA99BA9ACA9BDA981A392A3A3A3B4A306
:10E2F00023964FAF2397752EF62FE72F2C968CADD4
:10E300009DADAEADBFAD2C97481759076A077B0787
:10E3100078F429969FAD299723969FAF23972A9645
:10E320007FAC2A972B96FFAD2B972C96EFAD2C97B1
:10E3300023968FAD2397972DAF2FBE2F8017910770
:10E34000A207B30710F4D901C8010AA91BA92CA977
:10E350003DA980179107A207B30710F4D901C8019E
:10E3600028E60BA11CA1209FF001219FF00D112494
:10E37000E55EFD4E85A396A3A7A3B0A70697A105CA
:10E38000B10508F4A0C5DF01AE59BF4F809140042C
:10E39000909141048D939C9361A6452B462B472B6E
:10E3A00009F05F9888E60BA11CA1809FF001819F76
:10E3B000F00D1124E55EFD4E818D928DA38DB48DFF
:10E3C000892B8A2B8B2B11F08A98479888E60BA112
:10E3D0001CA1809FF001819FF00D1124E55EFD4E90
:10E3E000858D968DA78DB0A1892B8A2B8B2B31F033
:10E3F0008091080181708093060147982AA93BA962
:10E400004CA95DA9232B242B252B09F465C58091EC
:10E41000BF07882319F081508093BF07611004C0A3
:10E42000129880E28093BF076090B6077090B7079C
:10E430000091B8071091B9079301A80169A579A9BE
:10E440008EA99AAD0E944EEF87FF04C069A679AAF3
:10E450000EAB1AAFC501B4010E9454EF2091071210
:10E46000309108124091091250910A120E94B3EFA4
:10E4700026966CAF7DAF8EAF9FAF2697698B7A8B58
:10E480008B8B9C8BC201B1010E9454EF20910B1227
:10E4900030910C1240910D1250910E120E94B3EF68
:10E4A0002B013C016D8B7E8B8F8B988F6DA17EA194
:10E4B0008FA198A50E9454EF20910F123091101255
:10E4C00040911112509112120E94B3EF4B015C0166
:10E4D000698F7A8F8B8F9C8F209113123091141239
:10E4E0004091151250911612C701B6010E94B3EF68
:10E4F0006B017C016D8F7E8F8F8F98A388E60BA1B7
:10E500001CA1809FF001819FF00D1124E55EFD4E5E
:10E51000258936894789508D2DA33EA34FA358A73F
:10E52000263031054105510508F4DFC42896AEAD0B
:10E53000BFAD2897CD90DD90ED90FC9020E030E0CD
:10E54000A901C701B6010E944EEF8111EDC42696C4
:10E550002CAD3DAD4EAD5FAD2697CA01B9010E940D
:10E56000B3EF6B017C01A3019201C301B2010E94D0
:10E57000B3EF9B01AC01C701B6010E94CBF36B0165
:10E580007C01A5019401C501B4010E94B3EF9B0178
:10E59000AC01C701B6010E94CBF30E9436F628E613
:10E5A0000BA11CA1209FF001219FF00D1124E55E1D
:10E5B000FD4E658776878787908B88E60BA11CA127
:10E5C000809FF001819FF00D1124E55EFD4E458492
:10E5D000568467847088A301920160E070E080E84F
:10E5E0009FE30E94A7F464966CAF7DAF8EAF9FAFA0
:10E5F000649729A539A94EA95AAD0E94B3EF4B01E2
:10E600005C0180915E0A90915C0A891B8F7027964D
:10E610008FAF2797A501940160E074E284E799E445
:10E620000E94A7F40E94FCF56B017C0127968FAD38
:10E6300027978250863008F486C4A5019401C3014F
:10E64000B2010E94B3EF9B01AC010E94B3EF689648
:10E650006CAF7DAF8EAF9FAF689788E6ABA1BCA1D2
:10E660008A9F80018B9F100D1124055E1D4E6896B8
:10E670002CAD3DAD4EAD5FAD6897D80111962D9391
:10E680003D934D935C93149795962D913D914D91AB
:10E690005C9198972EAB3FAB48AF59AFCA01B90117
:10E6A0000E9452EF6AAF7BAF8CAF9DAF9B01AC0174
:10E6B000C501B4010E94B3EF0E9491F40E9414F5C9
:10E6C000A8966CAF7DAF8EAF9FAFA897F801EE5ABA
:10E6D000FF4F60837183828393838E010F5E1F4F90
:10E6E0002A961FAF0EAF2A970051110924961FAF2B
:10E6F0000EAF24970EE917E0AC961FAF0EAFAC97A4
:10E700008E010F5D1F4F1AA309A324960EAD1FADF6
:10E710002497AA961FAF0EAFAA97312C212C10E890
:10E7200019A70FE309AB2A96AEADBFAD2A972D917D
:10E730003D914D915D912A96BFAFAEAF2A97C5012D
:10E74000B4010E94B3EF6B017C01AA96EEADFFAD60
:10E75000AA976193719381939193AA96FFAFEEAFBD
:10E76000AA9720E030E0A9010E94F1F587FF04C0DC
:10E77000F7FAF094F7F8F094AC96AEADBFADAC9765
:10E780004D905D906D907D90AC96BFAFAEAFAC9765
:10E79000A7019601C301B2010E944EEF87FD0DC48F
:10E7A00009A11AA12A962EAD3FAD2A970217130789
:10E7B00009F0B9CF20E030E040E85FE3632D722D2F
:10E7C00089A599A90E944EEF87FF58C07E0131E1CB
:10E7D000E30EF11C24960EAD1FAD2497232D322D90
:10E7E00049A559A9D8016D917D918D919C910E9467
:10E7F000B3EFF80161937193819391938F01EE16BA
:10E80000FF0661F728E60BA11CA1209FC001219FF4
:10E81000900D11249C01255E3D4E790189010E5A0F
:10E820001F4FA8966CAD7DAD8EAD9FADA8970E9491
:10E8300052EF232D322D49A559A90E94B3EF0E9412
:10E8400014F5D8016D937D938D939C931397232D8D
:10E85000322D49A559A9632D722D89A599A90E9428
:10E86000B3EF68962CAD3DAD4EAD5FAD68970E949D
:10E87000B3EFF70161837283838394832AAD3BAD49
:10E880004CAD5DAD64966CAD7DAD8EAD9FAD6497C6
:10E890000E94B3EF69A77AA78BA79CA70DA11EA121
:10E8A0002FA138A5012B022B032B09F09EC388E66C
:10E8B0002BA13CA1829F8001839F100D1124055E36
:10E8C0001D4EF801818D928DA38DB48D892B8A2BDD
:10E8D0008B2B09F08AC3858D968DA78DB0A1892BCE
:10E8E0008A2B8B2B09F081C32091C0103091C1106D
:10E8F0004091C2105091C31069A57AA58BA59CA523
:10E900000E94B3EF0E9491F40E9414F52B013C0188
:10E91000F801E95BFF4F108288E62BA13CA1829FA2
:10E920008001839F100D1124055E1D4EF801E25AEF
:10E93000FF4F4082518262827382C301B2010E9402
:10E9400052EF29A53AA54BA55CA50E94A7F46AAF92
:10E950007BAF8CAF9DAFD80151966D937D938D9316
:10E960009C935497F801E95BFF4F8081882381F1E4
:10E970007801B8E4EB0EF11C3796209192073091A4
:10E98000930740919407509195076081718182812E
:10E9900093810E94B3EF2AAD3BAD4CAD5DAD0E94BB
:10E9A000B3EF209102113091031140910411509165
:10E9B00005110E94B3EF9B01AC0160E074E284EFAB
:10E9C00099E40E94A7F40E9414F5F7017183608313
:10E9D00088E60BA11CA1809FF001819FF00D1124FE
:10E9E000E55EFD4E21813281438154812C962CAF0E
:10E9F0003DAF4EAF5FAF2C97CA01B9010E9436F60A
:10EA0000362E272E8C0142E857E062965FAF4EAF5C
:10EA100062973E0151E1650E711C82E897E09FAB61
:10EA20008EAB24964EAC5FAC24973DA62DA209A7D1
:10EA300019AB1AAAD201CD90DD90ED90FD902D0179
:10EA400020E030E0A901C701B6010E94F1F587FF7F
:10EA500004C0F7FAF094F7F8F094EEA9FFA98190BA
:10EA60009190A190B190FFABEEABA7019601C501CB
:10EA7000B4010E944EEF87FDD8C564147504D1F629
:10EA800027965FAD2797552309F448C6C090600AC2
:10EA9000D090610AE090620AF090630A2DEB37E3B0
:10EAA00046E855E3C701B6010E944EEF87FD36C622
:10EAB000C701B6010E9436F66B017C019B01AC01D7
:10EAC000632D722DC8010E944EEF87FD03C03C2CC0
:10EAD0002D2C87019601A701632D722DC8010E947C
:10EAE000A7F468966CAF7DAF8EAF9FAF689784E652
:10EAF0009AE028969FAF8EAF289720E030E040E85C
:10EB00005FE32AAB3BAB4CAB5DAB1EAA2896AEAD28
:10EB1000BFAD28972D913D914D915D912896BFAF46
:10EB2000AEAF289768966CAD7DAD8EAD9FAD689702
:10EB30000E94B3EF4B015C012496EEADFFAD24972C
:10EB4000C190D190E190F1902496FFAFEEAF249761
:10EB5000FEA9FF2391F02AA93BA94CA95DA90E9417
:10EB6000B3EF4B015C012AA93BA94CA95DA9C701E0
:10EB7000B6010E94B3EF6B017C01A7019601C501AC
:10EB8000B4010E94F1F520E030E0A90118160CF064
:10EB900092C5C701B6010E94F1F518160CF486C59E
:10EBA00020E030E0A901C501B4010E944EEF87FDCD
:10EBB0007DC52601370177FA709477F87094A30128
:10EBC0009201C501B4010E94F1F5181614F4240154
:10EBD00035016296AEADBFAD6297CD90DD90ED9000
:10EBE000FD906296BFAFAEAF6297A3019201C701DD
:10EBF000B6010E944EEF87FF15C0A3019201C70125
:10EC0000B6010E94A7F49B01AC016AA97BA98CA95B
:10EC10009DA90E94B3EF6AAB7BAB8CAB9DABBEA949
:10EC2000BF5FBEABE4E7FAE028962EAD3FAD289774
:10EC3000E217F30709F06ACF3EA9332361F02AA94E
:10EC40003BA94CA95DA9632D722DC8010E94B3EFA9
:10EC5000362E272E8C0124EA30E74DE75FE3632D43
:10EC6000722DC8010E94B3EF6B017C012091BB079C
:10EC70003091BC074091BD075091BE070E944EEFF6
:10EC800087FD42C58DA59DA1A9A5B9A98093BB0704
:10EC90009093BC07A093BD07B093BE0728E64BA195
:10ECA0005CA1249FC001259F900D1124DC01A55E6D
:10ECB000BD4E7D01232D322DA801632D722DC8017B
:10ECC0000E94B3EFF70161877287838794876AADEB
:10ECD0007BAD8CAD9DAD90589B01AC010E94CBF3F8
:10ECE000D7011D962D913D914D915C9150970E94B9
:10ECF000B3EF9B01AC016BE077ED83E29BE30E94F5
:10ED0000CAF39B01AC018BE097EDA3E2BBE3F701F3
:10ED100085839683A783B08710812C966CAD7DADDB
:10ED20008EAD9FAD2C970E944EEF18160CF4FBC4CD
:10ED300083E0182B88E62BA13CA1829FF001839FE2
:10ED4000F00D1124E55EFD4E108380E1FE01319649
:10ED5000A4E6BAE001900D928A95E1F72C968CAD6D
:10ED60009DADAEADBFAD2C978093600A9093610AC4
:10ED7000A093620AB093630AE0960CAD1DAD2EAD70
:10ED80003FADE0970093840A1093850A2093860A8A
:10ED90003093870AE4962CAD3DAD4EAD5FADE49760
:10EDA0002093880A3093890A40938A0A50938B0AE9
:10EDB000E8968CAD9DADAEADBFADE89780938C0A63
:10EDC00090938D0AA0938E0AB0938F0A60960CAD33
:10EDD0001DAD2EAD3FAD60970093900A1093910A40
:10EDE0002093920A3093930A6C962CAD3DAD4EADB4
:10EDF0005FAD6C972093740A3093750A4093760A3E
:10EE00005093770AA0968CAD9DADAEADBFADA097E7
:10EE10008093780A9093790AA0937A0AB0937B0A38
:10EE2000A4960CAD1DAD2EAD3FADA49700937C0A0A
:10EE300010937D0A20937E0A30937F0A22962CAD90
:10EE40003DAD4EAD5FAD22972093800A3093810A8D
:10EE50004093820A5093830A90915E0A80915F0AE0
:10EE6000981303C084E680935B0AE9968FADE99717
:10EE70008F5F8F7080935E0A80915E0A90915D0A29
:10EE800081508F70891351C410915F0A1BA30091A8
:10EE90005E0A0DA728E61BA10DA51013D1C4812C75
:10EEA000912CA12CB12C1DA219A619AA1EAE212CA1
:10EEB000312C00E010E02DA53BA12313CEC421147A
:10EEC000310409F07FC580916F00826080936F00EC
:10EED00081E0ECC680E0EAC66090B2077090B307AC
:10EEE0000091B4071091B507A7CA818D928DA38DAB
:10EEF000B48D0697A105B10508F018CB858D968DC8
:10EF0000A78DB0A10697A105B10508F00FCB20E0B1
:10EF100030E0A901C701B6010E94F1F587FF04C0E6
:10EF2000F7FAF094F7F8F09488E60BA11CA1809F03
:10EF3000F001819FF00D1124E55EFD4EC586D68659
:10EF4000E786F08A3ACB8091AE079091AF07A09107
:10EF5000B007B091B107C816D906EA06FB0608F05B
:10EF60006CCB8C199D09AE09BF09BC01CD01660FA0
:10EF7000771F881F991F27964FAD2797042F10E002
:10EF800020E030E0A90198010E946DF3CA01B901A7
:10EF90000E9452EF0E94FCF56C0D7D1D8E1D9F1D81
:10EFA0000E9452EF9B01AC0160E074E284E799E4B7
:10EFB0000E94A7F44B015C0140CBA7019601C3015D
:10EFC000B2010E94A7F47B018C019B01AC01632D6F
:10EFD000722D89A599A90E94F1F518160CF0E0CBC5
:10EFE0003E2C2F2C09A719ABDBCB0AA91BA92CA9F6
:10EFF0003DA9012B022B032B49F020919A07309158
:10F000009B0740919C0750919D0708C0209196074F
:10F0100030919707409198075091990769A57AA573
:10F020008BA59CA50E94B3EF0E9491F40E9414F559
:10F030002B013C012AA93BA94CA95DA9232B242B18
:10F04000252BC9F020E030E0A90160919207709172
:10F05000930780919407909195070E944EEF882323
:10F0600051F081E00DA51EA52FA538A91016110697
:10F07000120613060CF080E098E62BA13CA1929FAB
:10F080008001939F100D1124055E1D4E180137E479
:10F09000230E311CD1018C93882309F4B3C0209135
:10F0A000740A3091750A4091760A5091770A6C96ED
:10F0B0006CAD7DAD8EAD9FAD6C970E94CAF36DA710
:10F0C0007EA78FA798AB2091780A3091790A40915A
:10F0D0007A0A50917B0AA0966CAD7DAD8EAD9FAD46
:10F0E000A0970E94CAF34B015C0120917C0A3091E9
:10F0F0007D0A40917E0A50917F0AA4966CAD7DAD49
:10F100008EAD9FADA4970E94CAF36B017C012DA523
:10F110003EA54FA558A9CA01B9010E94B3EF6DA73A
:10F120007EA78FA798ABA5019401C501B4010E94E9
:10F13000B3EF9B01AC016DA57EA58FA598A90E9498
:10F14000CBF34B015C01A7019601C701B6010E94F8
:10F15000B3EF9B01AC01C501B4010E94CBF30E9447
:10F1600036F66B017C012091800A3091810A409132
:10F17000820A5091830A22966CAD7DAD8EAD9FAD13
:10F1800022970E94CAF3A70196010E94A7F46B017F
:10F190007C01F801E25BFF4F60837183828393837C
:10F1A00020E030E040E450E40E94F1F518161CF431
:10F1B000F101108227C0209192073091930740916E
:10F1C000940750919507C701B6010E94B3EF9B01C8
:10F1D000AC0160918E0770918F078091900790919C
:10F1E00091070E94A7F429A53AA54BA55CA50E940A
:10F1F000B3EF0E9414F5641575058605970510F4A4
:10F200002B013C018091E3119091E411A091E51153
:10F21000B091E6110EA91FA928AD39AD801791074D
:10F22000A207B30708F4DFC02DA13EA14FA158A546
:10F23000232B242B252B41F16091E7117091E811CC
:10F240008091E9119091EA1164157505860597057D
:10F25000D8F42EA93FA948AD59AD0E945EF36B01C9
:10F260007C012DA13EA14FA158A5C301B2010E946E
:10F270005EF3C616D706E806F90630F4C701B601F4
:10F280000E946DF329013A0188E60BA11CA1809F21
:10F29000F001819FF00D1124E55EFD4EC18CD28CF2
:10F2A000E38CF48CC114D104E104F10431F16091D8
:10F2B000EB117091EC118091ED119091EE116415AC
:10F2C000750586059705C8F42EA93FA948AD59AD27
:10F2D0000E945EF34B015C01A7019601C301B201DC
:10F2E0000E945EF386169706A806B90630F4C5019B
:10F2F000B4010E946DF329013A0188E60BA11CA11B
:10F30000809FF001819FF00D1124E55EFD4EC58CBC
:10F31000D68CE78CF0A0C114D104E104F10431F1E2
:10F320006091EF117091F0118091F1119091F211B3
:10F330006415750586059705C8F42EA93FA948AD43
:10F3400059AD0E945EF34B015C01A7019601C30118
:10F35000B2010E945EF386169706A806B90630F43D
:10F36000C501B4010E946DF329013A0188E60BA1A1
:10F370001CA1809FF001819FF00D1124E55EFD4EE0
:10F38000C1A0D2A0E3A0F4A0C114D104E104F1040F
:10F3900009F4C2CA6091F3117091F4118091F511D2
:10F3A0009091F611641575058605970508F0B4CAA5
:10F3B0002EA93FA948AD59AD0E945EF34B015C01F7
:10F3C000A7019601C301B2010E945EF3861697065B
:10F3D000A806B90608F0A0CAC501B4010E946DF3E1
:10F3E00029013A0199CA2DA13EA14FA158A5232B6D
:10F3F000242B252BC9F16091E7117091E8118091C0
:10F40000E9119091EA11641575058605970560F577
:10F410000E9452EF2AAD3BAD4CAD5DAD0E94B3EF03
:10F420006B017C016DA17EA18FA198A50E9452EF76
:10F430004B015C01C301B2010E9452EFA50194018E
:10F440000E94B3EF9B01AC01C701B6010E944EEFD1
:10F4500087FF0AC0A5019401C701B6010E94A7F465
:10F460000E9414F52B013C0188E60BA11CA1809F92
:10F47000F001819FF00D1124E55EFD4E818C928C90
:10F48000A38CB48C81149104A104B104B9F16091EE
:10F49000EB117091EC118091ED119091EE116415CA
:10F4A00075058605970550F50E9452EF2AAD3BADD4
:10F4B0004CAD5DAD0E94B3EF6B017C01C501B401A1
:10F4C0000E9452EF4B015C01C301B2010E9452EF56
:10F4D000A50194010E94B3EF9B01AC01C701B601E5
:10F4E0000E944EEF87FF0AC0A5019401C701B60133
:10F4F0000E94A7F40E9414F52B013C0188E60BA1A1
:10F500001CA1809FF001819FF00D1124E55EFD4E4E
:10F51000858C968CA78CB0A081149104A104B104B1
:10F52000B9F16091EF117091F0118091F11190910A
:10F53000F211641575058605970550F50E9452EF86
:10F540002AAD3BAD4CAD5DAD0E94B3EF6B017C01CC
:10F55000C501B4010E9452EF4B015C01C301B2012D
:10F560000E9452EFA50194010E94B3EF9B01AC01F0
:10F57000C701B6010E944EEF87FF0AC0A5019401A2
:10F58000C701B6010E94A7F40E9414F52B013C01AB
:10F5900088E60BA11CA1809FF001819FF00D112432
:10F5A000E55EFD4EC1A0D2A0E3A0F4A0C114D10439
:10F5B000E104F10409F4B0C96091F3117091F41100
:10F5C0008091F5119091F6116415750586059705E2
:10F5D00008F0A2C90E9452EF2AAD3BAD4CAD5DAD23
:10F5E0000E94B3EF4B015C01C701B6010E9452EFCC
:10F5F0006B017C01C301B2010E9452EFA701960189
:10F600000E94B3EF9B01AC01C501B4010E944EEF13
:10F6100087FF82C9A7019601C501B4010E94A7F422
:10F620000E9414F52B013C0177C9FAA9FF2331F19F
:10F63000A5019401632D722DC8010E94B3EF4B0107
:10F640005C012DA53DA149A559A9C701B6010E949C
:10F65000B3EF9B01AC01C501B4010E944EEF87FFDF
:10F6600022C0A7019601C501B4010E94A7F46DA7AD
:10F670007DA389A799AB21E02AABFFC9A701960119
:10F68000C501B4010E94A7F49B01AC016DA57DA149
:10F6900089A599A90E94B3EF6DA77DA389A799AB0E
:10F6A00031E03AABEAC941E04AABE7C9A7019601AC
:10F6B000C501B40113C0C701B6010E944EEF87FD1A
:10F6C00009C020E030E0A901C501B4010E94F1F5B4
:10F6D00018164CF4A5019401C701B6010E94CAF3A3
:10F6E0002B013C0176CA2401350177FA709477F832
:10F6F0007094A3019201C701B6010E944EEF87FDED
:10F7000068CA2601370165CA2DA53DA149A559A999
:10F71000C701B6010E944EEF87FFB4CA3DA42DA0D9
:10F7200009A519A9AFCA81E004CBF0905E0A8FEF5A
:10F730008F0D8F708BA3B0905D0A80915E0AB81612
:10F7400009F454C0C12CD12C0BA10B1509F44EC0E7
:10F75000602E712C28E6269D8001279D100D112416
:10F76000055E1D4ED8018C9183FD2BC00EAF1AABE8
:10F770000115110541F11996BC91BDA7F801F2855B
:10F78000FDA3D8011B96BC91B9A7F801F485F9AB8C
:10F79000D80115962D903D904D905C901897A20140
:10F7A00091016DA57DA189A59F2F0E944EEF81112A
:10F7B00086C1C114D10439F0F601808180FD7FC17A
:10F7C00002C0CEAEDAAA8BA181508F708BA380913C
:10F7D0005D0A8B1103C0CEACDAA8B6CF0BA10B1516
:10F7E00029F081E08B0D8F70B82EF1CF10915D0A5A
:10F7F0001BA3C12CD12C80915E0A0BA1801709F4A8
:10F8000043CB802E912C28E6289D8001299D100D48
:10F810001124055E1D4ED8018C9183FD0AC058014C
:10F82000C114D10439F0C6010E942C62811102C0BA
:10F83000C5C156018BA18F5F8F708BA36501DBCF94
:10F84000802F81508F70289FF0011124E55EFD4EBE
:10F85000908193FF24CB8DA71ECB48E6439FC00128
:10F860001124DC01A55EBD4E1D018C9183FD19C0E4
:10F8700015966D917D918D919C9118970E9436F609
:10F88000F62EE72ED82EC92E0115110509F48CC0CD
:10F89000F801808180FD0AC0D1018C9180FD06C0F5
:10F8A00083C0FDA0E9A4D9A8CEAC83C0F8018081B3
:10F8B00081608083C8010E942C62811171C0F801AF
:10F8C00061817281838194810E9436F62B013C0113
:10F8D0009B01AC0160E070E080E89FE30E94A7F428
:10F8E0004B015C019B01AC016F2D7E2D8D2D9C2D5C
:10F8F0000E94B3EF69837A838B839C832DA139A502
:10F9000049A95EADC501B4010E94B3EF698B7A8B42
:10F910008B8B9C8BAE014F5F5F4FBE016F5E7F4F45
:10F92000C8010E94BFCBF801E95BFF4F80818823AB
:10F93000B9F120919207309193074091940750912B
:10F940009507379660817181828193810E94B3EF20
:10F950002091021130910311409104115091051131
:10F960000E94B3EF4B015C019B01AC01C301B201EA
:10F970000E94B3EF0E9414F5F801E65BFF4F71831C
:10F980006083A50194016F2D7E2D8D2D9C2D0E94ED
:10F99000B3EF0E9414F5F801E45BFF4F71836083BD
:10F9A000D8018C918E7F8C938F2C9E2CAD2CBC2CEF
:10F9B00081018BA18F5F8F708BA3FDA2E9A6D9AACD
:10F9C000CEAE79CAF101808181608083C8010E9436
:10F9D0002C6281116FC0D10111966D917D918D9135
:10F9E0009C9114970E9436F66B017C019B01AC013F
:10F9F00060E070E080E89FE30E94A7F42B013C01E7
:10FA00002DEC3CEC4CE45DE30E94B3EF69837A8318
:10FA10008B839C839401A501C301B2010E94B3EFC3
:10FA2000698B7A8B8B8B9C8BAE014F5F5F4FBE01D6
:10FA30006F5E7F4FC1010E94BFCBF101E95BFF4FB9
:10FA400080818823B9F120919207309193074091EA
:10FA500094075091950737966081718182819381D7
:10FA60000E94B3EF209102113091031140910411D3
:10FA7000509105110E94B3EF4B015C019B01AC0159
:10FA8000C701B6010E94B3EF0E9414F5F101E65BD5
:10FA9000FF4F718360832DEC3CEC4CE45DE3C501CA
:10FAA000B4010E94B3EF0E9414F5F101E45BFF4F33
:10FAB00071836083F10180818E7F808304CA28E690
:10FAC000269DF001279DF00D1124E55EFD4E8081FD
:10FAD00081FD43C0C114D10441F0D6011596CD90EB
:10FAE000DD90ED90FC90189708C08BE0C82E87ED54
:10FAF000D82E83E2E82E8BE3F82EB8E6B69DF0010F
:10FB0000B79DF00D1124E55EFD4E81899289A38990
:10FB1000B489BC01CD0190589B01AC010E94CBF38C
:10FB2000F80125853685478550890E94B3EF9B01F2
:10FB3000AC01C701B6010E94CAF3E62E872E982EAB
:10FB4000A92E262F372F482F592F6DA57DA189A5C6
:10FB500099A90E944EEF87FF04C0EDA48DA099A43F
:10FB6000A9A82E2D382D492D5A2DC201B1010E9470
:10FB70004EEF882309F427CEF8E6F69DC001F79DE5
:10FB8000900D11249C01255E3D4E6901D9018C9197
:10FB900081608C93C8010E942C62882329F0F601B1
:10FBA00080818E7F80830FCE8E2D982DA92DBA2D2A
:10FBB000F60185839683A783B08705CED6018C9105
:10FBC00081FD52C0D60115962D913D914D915C91CC
:10FBD00018972DA73EA74FA758AB1501B5E02B0EE0
:10FBE000311CF8014580568067807084A301920122
:10FBF0006DA57EA58FA598A90E944EEF87FF34C002
:10FC0000F60181899289A389B489BC01CD019058FC
:10FC10009B01AC010E94CBF3D6011D962D913D9125
:10FC20004D915C9150970E94B3EF9B01AC016DA583
:10FC30007EA58FA598A90E94CAF36B017C019B0148
:10FC4000AC01C301B2010E94F1F518166CF4D801A1
:10FC50008C9181608C93C5010E942C628823E1F015
:10FC6000F80180818E7F808318E6189DF001199D30
:10FC7000F00D1124E55EFD4E2185328543855485C6
:10FC800065817681878190850E944EEF8111D2CD6A
:10FC90000BA100935D0ACECDD101CD92DD92ED9204
:10FCA000FC9213970BA100935D0ADECFC858DF4F7B
:10FCB0000FB6F894DEBF0FBECDBFDF91CF911F917D
:10FCC0000F91FF90EF90DF90CF90BF90AF909F90FB
:10FCD0008F907F906F905F904F903F902F900895FE
:10FCE00080915E0A90915F0A891B8F708F3021F49A
:10FCF00080E00E946EAEF4CF80915E0A8F5F8F70BD
:10FD0000E0915E0A98E69E9FF0011124E55EFD4EAB
:10FD1000DF011D929A95E9F798E090834091840A5B
:10FD20005091850A6091860A7091870A458B568B9F
:10FD3000678B708F4091880A5091890A60918A0A76
:10FD400070918B0A418F528F638F748F40918C0A10
:10FD500050918D0A60918E0A70918F0A458F568F4F
:10FD6000678F70A34091900A5091910A6091920A16
:10FD70007091930A41A352A363A374A320915E0AD6
:10FD800090915F0A291303C094E690935B0A8093D5
:10FD90005E0A80916F00826080936F000895909159
:10FDA0005E0A80915F0A981306C080917405909155
:10FDB0007505892B21F080E00E946EAEF0CF08958A
:10FDC0004F925F926F927F928F929F92AF92BF926B
:10FDD000CF92DF92EF92FF92CF93DF932091240492
:10FDE00030912504409126045091270460914C04E1
:10FDF00070914D0480914E0490914F040E94CBF37A
:10FE0000AB01BC0188E591E20E9461C62091280403
:10FE10003091290440912A0450912B0460915004A0
:10FE20007091510480915204909153040E94CBF33D
:10FE3000AB01BC0184E591E20E9461C620912C04D3
:10FE400030912D0440912E0450912F046091540460
:10FE50007091550480915604909157040E94CBF301
:10FE6000AB01BC0180E591E20E9461C6409158045B
:10FE70005091590460915A0470915B048CE491E2B2
:10FE80000E9461C680916F00982F927081FF05C01B
:10FE900080916F008D7F80936F004090E6105090AE
:10FEA000E7106090E8107090E9108090EA10909050
:10FEB000EB10A090EC10B090ED10C090EE10D09030
:10FEC000EF10E090F010F090F110992329F080915C
:10FED0006F00826080936F00E2E4F1E28491EF01B1
:10FEE0002196882321F00E94679AFE01F7CFC30173
:10FEF000B2010E940E9EEEE3F1E28491EF012196A1
:10FF0000882321F00E94679AFE01F7CFC501B40152
:10FF10000E940E9EEAE3F1E28491EF01219688238C
:10FF200021F00E94679AFE01F7CFC701B6010E9437
:10FF30000E9E8AE0DF91CF91FF90EF90DF90CF90FF
:10FF4000BF90AF909F908F907F906F905F904F90F9
:10FF50000C94679A2F923F924F925F926F927F928A
:10FF60008F929F92AF92BF92CF92DF92EF92FF92C9
:10FF70000F931F93CF93DF93CDB7DEB762970FB682
:10FF8000F894DEBF0FBECDBF8091BA0783FD9AC142
:10FF900083E50E9434408C87811106C082E50E946F
:10FFA0003440882309F48EC10E94B43F0E940FF5AB
:10FFB000CB010E94C3410E94B43F20E030E040EA00
:10FFC00050E40E94F1F5181614F40E94B2C6EEE255
:10FFD000F1E28491FB83EA83882371F0082E000C00
:10FFE000990B0E94F49F4A815B814F5F5F4F5B8357
:10FFF0004A83FA018491F0CF8DE090E00E94F49F53
:020000021000EC
:100000008AE090E00E94F49F81E0809324021092A5
:10001000C51080918E10809378051A821B821C82F5
:100020001D82188619861A861B8619821D86FCE396
:10003000FE872CE12F8736E4388B312C212C40E8C9
:10004000498B5FEB5A8B812C912C540160914204B7
:1000500070914304072E000C880B990B0E9454EFFB
:100060007B018C019B01AC01632D722D89899A89DA
:100070000E944EEF882341F12091440430914504C1
:1000800040914604509147048C85B70181110CC002
:10009000C8010E944EEF881F8827881F89833E2C45
:1000A0002F2C098B1A8B10C0C8010E944EEF87FFBE
:1000B00006C0E2E3F1E28491FB83EA83E8C03E2CD0
:1000C0002F2C098B1A8B19820E9467626B017C01AD
:1000D000DC01CB01288539854A855B85821B930B22
:1000E000A40BB50BB7FD3BC0D701C60188519C4F8F
:1000F000AF4FBF4F88879987AA87BB870E94A958AF
:10010000E6E3F1E284913F019FEF691A790A8823BF
:1001100021F00E94679AF301F5CF81149104A104A4
:10012000B104B9F0D501C401805F984DAF4FBF4F06
:10013000BC01CD016C197D098E099F0928EE33E0C1
:1001400040E050E00E946DF3CA01B9010E940E9E8A
:1001500003C08FE30E94679A8AE00E94679A80E05A
:100160000E946EAE0E9467626093691070936A107D
:1001700080936B1090936C10A0914404AE83B09167
:100180004504BF8300914604109147040E94092D45
:100190002E813F81A801632D722D89899A890E9441
:1001A000CAF32B013C0120E030E0A9010E94F1F5E7
:1001B00087FF04C077FA709477F8709481149104E3
:1001C000A104B10459F420E030E040E85FE3C3014A
:1001D000B2010E944EEF87FF0DC00AC020E030E060
:1001E00040E450E4C301B2010E94F1F5181614F482
:1001F00046015701E981EE2391F12A813B814C812F
:100200005D81211531054105510541F0D701C60138
:10021000821B930BA40BB50BB7FD21C02E813F8130
:10022000A8016D857E858F8598890E94CAF320E09C
:1002300030E040EC5FE30E944EEF87FD3ACFD701FC
:10024000C601805A9541AF4FBF4F8A839B83AC83D1
:10025000BD839E819D87AF81AE870F87188B80916C
:100260002402882309F425CF81149104A104B10448
:1002700009F4ECCEB0E1CB1AB7E2DB0AE108F108F1
:10028000C818D908EA08FB08F7FE13CFDFCE882389
:1002900061F0082E000C990B0E94F49FEA81FB810B
:1002A0003196FB83EA838491F2CF8DE090E00E9447
:1002B000F49F8AE090E00E94F49F8091240281E004
:1002C0008093C51062960FB6F894DEBF0FBECDBF07
:1002D000DF91CF911F910F91FF90EF90DF90CF9022
:1002E000BF90AF909F908F907F906F905F904F9056
:1002F0003F902F900895EF92FF920F931F93CF930B
:10030000DF93CDB7DEB769970FB6F894DEBF0FBEA7
:10031000CDBF83E50E943440811103C0E6E1F1E2E4
:1003200008C00E94843F6E347105C1F70E9469C7FE
:10033000E4C084918F010F5F1F4F882321F00E943A
:10034000679AF801F6CFEDE0F1E284918F010F5F3B
:100350001F4F882321F00E94679AF801F6CF809101
:10036000D5059091D6050E94B8E0E0E0F1E28491D5
:100370008F010F5F1F4F882321F00E94679AF801B9
:10038000F6CF8091D7059091D8050E94B8E0E5EFAF
:10039000F0E284918F010F5F1F4F882321F00E94AC
:1003A000679AF801F6CF8091D5059091D6052091F6
:1003B000D7053091D805821B930B2091540521500D
:1003C00041E050E0223010F040E050E0841B950BFB
:1003D0000E94B8E08AE00E94679AEDEEF0E2849114
:1003E0008F010F5F1F4F882321F00E94679AF80149
:1003F000F6CF8091D9059091DA05A091DB05B091F7
:10040000DC058E8B9F8BA88FB98FBE016F5F7F4FEE
:10041000CE0146960E948599E0EEF0E284918F012C
:100420000F5F1F4F882321F00E94679AF801F6CFD3
:10043000CE0101967C018C01F80181918F01882306
:1004400019F00E94679AF8CF8091DD059091DE0542
:10045000A091DF05B091E0058E8B9F8BA88FB98F9F
:10046000BE016F5F7F4FCE0146960E948599E0EDF9
:10047000F0E284918F010F5F1F4F882321F00E94CB
:10048000679AF801F6CFF70181917F01882319F06F
:100490000E94679AF8CF8AE00E94679AE8ECF0E23F
:1004A00084918F010F5F1F4F882321F00E94679A6C
:1004B000F801F6CFE8EBF0E284918F010F5F1F4F58
:1004C000882321F00E94679AF801F6CF20E030E0FF
:1004D0004AE754E46091E1057091E2058091E305FB
:1004E0009091E4050E94A7F442E00E94289E8DE6C8
:1004F0000E94679A8AE00E94679A69960FB6F894FC
:10050000DEBF0FBECDBFDF91CF911F910F91FF9046
:10051000EF9008958F929F92AF92BF92CF92DF9209
:10052000EF92FF920F931F93CF93DF9300D01F9210
:10053000CDB7DEB7F82E662351F01092CA0710929D
:10054000C6071092C7071092C8071092C9070E94E9
:1005500067628090C6079090C707A090C807B090C8
:10056000C9079B01AC01281939094A095B0957FDE4
:100570004CC02091CA07F7FC16C04F2D0F2C000C61
:10058000550B4C5F5F4FE22F022E000CFF0B4E17F6
:100590005F07DCF12F153CF044EFC42EDD24D3942B
:1005A000E12CF12C06C038EEC32E33E0D32EE12C23
:1005B000F12CDC01CB018C0D9D1DAE1DBF1D809368
:1005C000C6079093C707A093C807B093C907022F27
:1005D000017010E024E2209FC001219F900D901B2C
:1005E000112480599C4F9C838B8382E390E09A83F3
:1005F0008983BE016D5F7F4FCE0101960E9430B8A6
:100600008091CA078F5F8093CA070F900F900F9059
:100610000F90DF91CF911F910F91FF90EF90DF909E
:10062000CF90BF90AF909F908F900895AF92BF9260
:10063000CF92DF92EF920F931F93CF93DF93CDB7BB
:10064000DEB760970FB6F894DEBF0FBECDBF5C017A
:100650008B010E944040E0908E1082E1C82E81E123
:10066000D82E84E0E89EF0011124EB5DFD4F20813F
:10067000318142815381F501608171818281938151
:100680000E94A7F4F60124853585468557850E948A
:10069000CBF3F60164877587868797871D861E864C
:1006A0001F86188A80819181A281B38189839A8370
:1006B000AB83BC8384819581A681B7818D839E8322
:1006C000AF83B88780859185A285B38589879A870E
:1006D000AB87BC87AE01475F5F4FBE016B5F7F4F4B
:1006E000CE0101960E9438D0CE010D966C012EE10C
:1006F00031E1AE01475F5F4FBE016B5F7F4F0C97EB
:100700000E94A96E0E9483414ADB60960FB6F8945E
:10071000DEBF0FBECDBFDF91CF911F910F91EF9044
:10072000DF90CF90BF90AF9008959F92AF92BF920D
:10073000CF92DF92EF92FF920F931F93CF93DF93AD
:1007400087E5A82E82E0B82E02E111E1CCE4D4E0E6
:1007500094E2C92E94E0D92E21E3E22E24E0F22E79
:10076000912CF50181915F010E94EB3F882309F1F3
:100770000E94B43FF7012081211104C0209135046B
:10078000222339F0288139814A815B810E94CBF391
:100790000AC0F3E09F1639F0F601208131814281D1
:1007A00053810E94CAF3F80160837183828393832B
:1007B00009C088819981AA81BB81F80180839183D6
:1007C000A283B38393940C5F1F4F2496F4E0CF0E63
:1007D000D11C2FEFE21AF20A84E09812C2CF86E40D
:1007E0000E9434408823C9F00E94B43F20E030E0EA
:1007F000A9010E94F1F5181684F40E94B43F20E08C
:1008000030E040E752E40E94A7F460933D02709309
:100810003E0280933F02909340028091BA0783FD8D
:1008200028C08091D405882321F12091580430916B
:10083000590440915A0450915B0460911E117091CB
:100840001F1180912011909121110E94CAF32091D3
:10085000E1053091E2054091E3055091E4050E94E5
:10086000CBF36093E1057093E2058093E3059093E9
:10087000E405DF91CF911F910F91FF90EF90DF90F2
:10088000CF90BF90AF909F9008952F923F924F923C
:100890005F926F927F929F92AF92BF92CF92DF92C0
:1008A000EF92FF920F931F93CF93DF93CDB7DEB7F5
:1008B00064970FB6F894DEBF0FBECDBF1A012B01AF
:1008C000922EF32EC82ED12CF601E255FA4DE4916A
:1008D000AA24A3941E160CF4A12CBB24B39420E0EC
:1008E00030E0A901C201B1010E94F1F518160CF027
:1008F000B12CCC0CDD1CCC0CDD1CC601845B9B4FE9
:100900003C01FC0110821182128213820E942E99F6
:10091000F3012082318242825382E0908E1020E0E7
:1009200030E0A901B801892D9F2D0E944EEF811161
:100930000AC0F601EF59FA4D85919591A591B491B0
:100940008C019A2EFB2EC801A92DBF2D898B9A8B65
:10095000AB8BBC8B8091540490915504A0915604AC
:10096000B091570440915004509151046091520449
:100970007091530400914C0410914D0420914E0449
:1009800030914F0409831A832B833C834D835E830C
:100990006F83788789879A87AB87BC871D861E8679
:1009A0001F86188AAE01475F5F4FBE016B5F7F4FA6
:1009B000CE0101960E9438D0CE010D966C018E01B9
:1009C0000F5E1F4F28E534E0AE01475F5F4FBE0169
:1009D0006B5F7F4F0C970E94A96EE1D9AB1459F061
:1009E0008091F705882319F01092F70504C08CE870
:1009F00090E20E9427AE64960FB6F894DEBF0FBE59
:100A0000CDBFDF91CF911F910F91FF90EF90DF90BD
:100A1000CF90BF90AF909F907F906F905F904F90DE
:100A20003F902F900895EF92FF921F93CF93DF9303
:100A300083EAE82E88E1F82E15E0C0E0D0E020E05F
:100A400030E0A901F701EC0FFD1F60817181828107
:100A500093810E944EEF81110CC02496C431D105C0
:100A600071F7115084E1E80EF11C1111E6CF80E01E
:100A700001C081E0DF91CF911F91FF90EF90089529
:100A8000CF939091E0109817C1F0C82F88D9C11169
:100A900012C044E554E060E574E08CE494E00E9408
:100AA00038D080E08093E010882339F08CE494E023
:100AB000CF910C9479C7B7DFF5CFCF910895CF923E
:100AC000DF92EF920F931F93CF93DF93CDB7DEB7F3
:100AD00060970FB6F894DEBF0FBECDBFE0908E10CA
:100AE000ECE4F4E080859185A285B385448155814D
:100AF00066817781008111812281338109831A8384
:100B00002B833C834D835E836F83788789879A87A5
:100B1000AB87BC871D861E861F86188AAE01475F7D
:100B20005F4FBE016B5F7F4FCE0101960E9438D0B0
:100B3000CE010D966C010DE312E028E534E0AE0124
:100B4000475F5F4FBE016B5F7F4F0C970E94A96E9E
:100B500060960FB6F894DEBF0FBECDBFDF91CF9188
:100B60001F910F91EF90DF90CF9008952F923F92B9
:100B70004F925F926F927F928F929F92AF92BF92AD
:100B8000CF92DF92EF92FF920F931F93CF93DF9359
:100B9000CDB7DEB72A970FB6F894DEBF0FBECDBF34
:100BA0002B013C012D833E834F8358874701580119
:100BB000DA86C98680913D0290913E02A0913F0263
:100BC000B091400289839A83AB83BC83D6011C9188
:100BD00011960C91119712963C90129713962C90A7
:100BE00020E030E0A901612F702F832D922D0E940B
:100BF0004EEF81110AC0E9E6F5E285919591A59144
:100C0000B491182F092F3A2E2B2EA5019401609133
:100C100054047091550480915604909157040E9499
:100C20004EEF87FF15C0812F902FA32DB22D8093FB
:100C30003D0290933E02A0933F02B0934002809207
:100C4000540490925504A0925604B092570437DF92
:100C5000E985FA85C080D180E280F38020E030E031
:100C6000A901C701B6010E944EEF811107C085E5B9
:100C7000C82EDC2C85E0E82E83E4F82EC0923D02DD
:100C8000D0923E02E0923F02F092400240924C0429
:100C900050924D0460924E0470924F048D819E815B
:100CA000AF81B8858093500490935104A09352046F
:100CB000B093530404DF20915404309155044091C3
:100CC000560450915704C501B4010E944EEF87FFAE
:100CD00015C0812F902FA32DB22D80933D029093AC
:100CE0003E02A0933F02B09340028092540490923F
:100CF0005504A0925604B0925704E1DE50D8898181
:100D00009A81AB81BC8180933D0290933E02A09377
:100D10003F02B09340022A960FB6F894DEBF0FBE92
:100D2000CDBFDF91CF911F910F91FF90EF90DF909A
:100D3000CF90BF90AF909F908F907F906F905F907B
:100D40004F903F902F900895CF92DF92EF92FF92B5
:100D50000F931F936B01FC01E080F18002811381EE
:100D6000ECE4F4E024813581468157816081718112
:100D700082819381FBDE1F910F91FF90EF90DF90B6
:100D8000CF9008958F929F92AF92BF92EF92FF9271
:100D90000F931F93CF93DF9300D01F92CDB7DEB791
:100DA000182F80913F048770873069F48FE40E9488
:100DB0003440882319F00E94A53F03C08FE40E94AD
:100DC000EB3F8111BDC00E94CF7E80E059DE809153
:100DD0003D0290913E02A0913F02B091400280936B
:100DE000C2079093C307A093C407B093C50780912F
:100DF0000202909103029093C1078093C00784E69A
:100E000090E0909303028093020281E08093E605D4
:100E100011111BC088E50E94EB3FF82E89E50E9466
:100E2000EB3F082F8AE50E94EB3FE82EF11006C049
:100E3000011109C0811107C0F02E0CC0002319F068
:100E4000F02E182F08C010E006C0FF24F39401E034
:100E5000EE24E39411E00E94404082E50E94344079
:100E6000882361F00E94B43F4B015C0120E030E038
:100E7000A9010E944EEF882369F106C0812C912CB4
:100E800080EAA82E80E4B82E111104C0F11002C02F
:100E9000002389F180921A1190921B11A0921C11CB
:100EA000B0921D11A50194016091540470915504F4
:100EB00080915604909157040E944EEF87FF0AC01C
:100EC00019821A821B821C82BE016F5F7F4F8AE1EA
:100ED00091E13ADF111105C0F11003C0011106C004
:100EE0000AC080E00E94CBAC1123C1F381E00E94D4
:100EF000CBAC111102C0EE2019F082E00E94CBAC05
:100F00000E942E998091E5058093E6058091C207A5
:100F10009091C307A091C407B091C50780933D028B
:100F200090933E02A0933F02B09340028091C0078D
:100F30009091C10790930302809302020E94E07E89
:100F40000F900F900F900F90DF91CF911F910F9105
:100F5000FF90EF90BF90AF909F908F9008952F9249
:100F60003F924F925F926F927F928F929F92AF9239
:100F7000BF92CF92DF92EF92FF920F931F93CF9386
:100F8000DF93CDB7DEB762970FB6F894DEBF0FBE22
:100F9000CDBF8DE690E00E946E9A8111C6C180910E
:100FA000BA0783FDC2C183E50E9434408C8781115A
:100FB00006C082E50E94344089838823B1F00E94F4
:100FC000B43F0E940FF5CB010E94FB590E94B43F31
:100FD00020E030E04AEA52E40E944EEF18160CF48A
:100FE0009FC10E94F9C621E02983EEE1F1E28491DC
:100FF0008F01882351F0082E000C990B0E94F49F5A
:101000000F5F1F4FF8018491F4CF8DE090E00E94B4
:10101000F49F8AE090E00E94F49F0E94AAC8F981A0
:10102000FF2309F482C181E0809324021092C5104D
:101030001A821B821C821D82188619861A861B86BC
:1010400019821D862CE32E873CE13F8746E4488BBE
:10105000312C212C50E8598B8FEB8A8B812C912CD1
:1010600054016091480470914904072E000C880BCC
:10107000990B0E9454EF7B018C019B01AC01632D05
:10108000722D89899A890E944EEF882359F1209107
:101090005C0430915D0440915E0450915F049C8536
:1010A000B701802F91110CC0912F0E944EEF881F25
:1010B0008827881F89833E2C2F2C098B1A8B12C0FE
:1010C000912F0E944EEF87FF08C080912402E6E234
:1010D000F1E28491FB83EA83E8C03E2C2F2C098B3C
:1010E0001A8B19820E9467626B017C01DC01CB01C3
:1010F000288539854A855B85821B930BA40BB50B2C
:10110000B7FD3BC0D701C60188519C4FAF4FBF4FC1
:1011100088879987AA87BB870E94A958EAE2F1E2EB
:1011200084913F019FEF691A790A882321F00E9478
:10113000679AF301F5CF81149104A104B104B9F0C9
:10114000D501C401805F984DAF4FBF4FBC01CD01A9
:101150006C197D098E099F0928EE33E040E050E0CC
:101160000E946DF3CA01B9010E940E9E03C08FE375
:101170000E94679A8AE00E94679A80E00E946EAEA1
:101180000E9467626093691070936A1080936B107D
:1011900090936C10A0915C04AE83B0915D04BF830A
:1011A00000915E0410915F040E94092D2E813F8101
:1011B000A801632D722D89899A890E94CAF32B0197
:1011C0003C0120E030E0A9010E94F1F587FF04C056
:1011D00077FA709477F8709481149104A104B104A3
:1011E00059F420E030E040E85FE3C301B2010E941F
:1011F0004EEF87FF0DC00AC020E030E040E450E42D
:10120000C301B2010E94F1F5181614F4460157010A
:10121000E981EE2391F12A813B814C815D81211589
:1012200031054105510541F0D701C601821B930BE1
:10123000A40BB50BB7FD21C02E813F81A8016D85A0
:101240007E858F8598890E94CAF320E030E040ECCB
:101250005FE30E944EEF87FD38CFD701C601805A69
:101260009541AF4FBF4F8A839B83AC83BD839E81E3
:101270009D87AF81AE870F87188B809124028823CA
:1012800009F423CF81149104A104B10409F4E9CE37
:10129000B0E1CB1AB7E2DB0AE108F108C818D908B7
:1012A000EA08FB08F7FE11CFDCCE882361F0082E98
:1012B000000C990B0E94F49FEA81FB813196FB831D
:1012C000EA838491F2CF8DE090E00E94F49F8AE05F
:1012D00090E00E94F49F8091EA0E8130E9F4E2E20E
:1012E000F1E28491FB83EA83882371F0082E000CDD
:1012F000990B0E94F49F4A815B814F5F5F4F5B8334
:101300004A83FA018491F0CF8DE090E00E94F49F2F
:101310008AE090E00E94F49F81E08093C51005C0B0
:101320000E94B2C631E0398360CE62960FB6F8945F
:10133000DEBF0FBECDBFDF91CF911F910F91FF9008
:10134000EF90DF90CF90BF90AF909F908F907F9065
:101350006F905F904F903F902F900895CF93DF93C1
:101360008B3D9240B1F0E5E5F4E28491EF012196E6
:10137000882321F00E94679AFE01F7CFEBE5F1E2A6
:101380008491EF012196882331F00E94679AFE0133
:10139000F7CF80E001C081E0DF91CF9108952F92D7
:1013A0003F924F925F926F927F928F929F92AF92F5
:1013B000BF92CF92DF92EF92FF920F931F93CF9342
:1013C000DF93CDB7DEB7C757D1090FB6F894DEBFAC
:1013D0000FBECDBF2DB63EB6A7961FAE1EAEA797C9
:1013E00084E690E0A9969FAF8EAFA99701E09E0199
:1013F0002B593F4F44E050E0BE01655A7F4FCE016C
:1014000089599F4F0E94EED89E012B593F4F42E0D1
:1014100050E0BE0167597F4FCE0189599F4F0E940E
:10142000EED843E050E0BE01655A7F4F8FED92E069
:101430000E9436F7892B09F43FC06F968FAD6F97E6
:10144000882339F08FE36C968FAF6C976D961FAE43
:101450006D97EAE6F4E284917F012FEFE21AF20A37
:10146000811103C0EEE1F2E204C00E94679AF70125
:10147000F2CF84917F013FEFE31AF30A882321F032
:101480000E94679AF701F5CFBE01655A7F4F85E14B
:1014900092E20E9497C6E7E0F2E284917F019FEF1B
:1014A000E91AF90A882321F00E94679AF701F5CF1B
:1014B00081E08093CB0785C5EDB7FEB7E696FFAF19
:1014C000EEAFE6976B961CAE1DAE1EAE1FAE6B97D1
:1014D000A7961FAE1EAEA79701E09E012B593F4F66
:1014E00041E050E0BE0160597F4FCE0189599F4FC6
:1014F0000E94EED880E1EBE5F2E0DE0191960190EA
:101500000D928A95E1F780E1EBE6F2E0DE0151967B
:1015100001900D928A95E1F780E1EBE7F2E0DE01C0
:10152000119601900D928A95E1F7E1964FADE19702
:1015300050E04D5F5F4F440F551F440F551F2DB7AF
:101540003EB7241B350B0FB6F8943EBF0FBE2DBF20
:101550008DB79EB701967C0100E09E012B593F4F4D
:10156000BC01CE0189599F4F0E94EED89E012B5994
:101570003F4F44E050E06EEA77E0CE0189599F4F3B
:101580000E94EED8E1968FACE197912C93E0890E02
:10159000911C880C991C880C991CEDB7FEB7E819B2
:1015A000F9090FB6F894FEBF0FBEEDBF2DB73EB7D9
:1015B0002F5F3F4F69018DB79EB7881999090FB604
:1015C000F8949EBF0FBE8DBFEDB7FEB731965F0199
:1015D0009E012B593F4FA401B601CE0189599F4F5F
:1015E0000E94EED89E012B593F4FA401B501CE01B8
:1015F00089599F4F0E94EED81091CC07112309F40E
:10160000A7C000E09E012B593F4F44E050E06AE93B
:1016100077E0CE0189599F4F0E94EED89E012B5949
:101620003F4F44E050E060EC70E1CE0189599F4F9C
:101630000E94EED89E012B593F4F44E050E066E9EE
:1016400077E0CE0189599F4F0E94EED89E012B5919
:101650003F4F44E050E066EB77E0CE0189599F4F61
:101660000E94EED89E012B593F4F44E050E062EBC0
:1016700077E0CE0189599F4F0E94EED89E012B59E9
:101680003F4F40E150E062E877E0CE0189599F4F3B
:101690000E94EED89E012B593F4F44E050E0BE011E
:1016A000695A7F4FCE0189599F4F0E94EED89E0103
:1016B0002B593F4F4CE050E067EE75E0CE01895961
:1016C0009F4F0E94EED89E012B593F4F44E050E0BF
:1016D00065E179E1CE0189599F4F0E94EED89E01C4
:1016E0002B593F4F44E050E0BE01695A7F4FCE0175
:1016F00089599F4F0E94EED801E09E012B593F4F20
:1017000041E050E0BE0161597F4FCE0189599F4FA2
:101710000E94EED89E012B593F4F41E050E0BE01A0
:1017200062597F4FCE0189599F4F0E94EED8111107
:101730008AC06B968CAD9DADAEADBFAD6B978093FF
:101740009F189093A018A093A118B093A2187BC0E3
:10175000E1968FADE19790E002962EE937E0E496AE
:101760003FAF2EAFE497B501DE01119656EF852EFF
:1017700050E1952EAE014F5E5F4FE7EFAE2EE1E1F7
:10178000BE2EE896FFAEEEAEE8977E0131E2E30EA4
:10179000F11C20E030E0821793072CF0E896EEADC4
:1017A000FFADE89701C0F7014080518062807380EF
:1017B000F50141925192619271925F0182179307F4
:1017C00014F0F60101C0FA014080518062807380FC
:1017D000F40141925192619271924F0182179307E5
:1017E00034F0FB01408051806280738005C04D90D1
:1017F0005D906D907C901397E496EEADFFADE4970D
:101800004192519261927192E496FFAFEEAFE497EC
:101810002F5F3F4F6C5F7F4F1496F4E0CF0ED11CCB
:101820004C5F5F4FE896EEADFFADE8973496E896D3
:10183000FFAFEEAFE897F4E0EF0EF11C2430310576
:1018400009F0A9CFDECEE0968FADE097853099F410
:10185000AF968FADAF97853071F400E09E012B59A4
:101860003F4F44E650E063EA78E1CE0189599F4F4B
:101870000E94EED824C0111102C00E94CCD1E09683
:101880008FADE097AF96CFACAF978C9D60011124E0
:10189000E12CF12CEC14FD0491F000E09E012B5999
:1018A0003F4F44E050E0BE01695A7F4FCE01895955
:1018B0009F4F0E94EED82FEFE21AF20AEBCF00E022
:1018C0009E012B593F4F44E050E0BE016D5A7F4FBF
:1018D000CE0189599F4F0E94EED81AE0115079F03D
:1018E00000E09E012B593F4F44E050E0BE01695A91
:1018F0007F4FCE0189599F4F0E94EED8EFCF01E074
:101900009E012B593F4F41E050E0BE0163597F4F8C
:10191000CE0189599F4F0E94EED89E012B593F4F0F
:1019200041E050E0BE0164597F4FCE0189599F4F7D
:101930000E94EED800E09E012B593F4F44E050E05A
:10194000BE01635C7F4FCE0189599F4F0E94EED844
:101950009E012B593F4F44E050E0BE016F5C7F4F2A
:10196000CE0189599F4F0E94EED8AE968FADAE97AB
:10197000AD96CFACAD978C9D60011124E12CF12C7C
:1019800000E09E012B593F4FCE14DF0471F044E07C
:1019900050E0BE01695A7F4FCE0189599F4F0E9486
:1019A000EED83FEFE31AF30AEBCF41E050E0BE017F
:1019B0006F587F4FCE0189599F4F0E94EED89E01EC
:1019C0002B593F4F41E050E0BE0165597F4FCE019A
:1019D00089599F4F0E94EED89E012B593F4F44E0FA
:1019E00050E0BE01695A7F4FCE0189599F4F0E9436
:1019F000EED89E012B593F4F44E050E0BE01695A9A
:101A00007F4FCE0189599F4F0E94EED89E012B59DE
:101A10003F4F44E050E061E279E1CE0189599F4FA8
:101A20000E94EED89E012B593F4F44E050E0BE018A
:101A3000615B7F4FCE0189599F4F0E94EED89E0176
:101A40002B593F4F44E050E0BE01655B7F4FCE0114
:101A500089599F4F0E94EED89E012B593F4F44E079
:101A600050E0BE01695B7F4FCE0189599F4F0E94B4
:101A7000EED810E000E09E012B593F4F44E050E0CB
:101A8000BE01695A7F4FCE0189599F4F0E94EED8FF
:101A9000111110C06B96CCACDDACEEACFFAC6B970B
:101AA00020E030E84BE355E4C701B6010E944EEF59
:101AB000811103C044E0F42E33C08091CC07811122
:101AC00008C0C0926505D0926605E0926705F09265
:101AD000680500E09E012B593F4F44E050E061E66D
:101AE00075E0CE0189599F4F0E94EED89E012B5977
:101AF0003F4F44E050E069E675E0CE0189599F4FC1
:101B00000E94EED89E012B593F4F44E050E0BE01A9
:101B1000695A7F4FCE0189599F4F0E94EED812C05B
:101B2000FA94FF2079F000E09E012B593F4F44E0EA
:101B300050E0BE01695A7F4FCE0189599F4F0E94E4
:101B4000EED8EECF1F5F153009F094CF00E09E0174
:101B50002B593F4F42E050E0BE016D597F4FCE01FF
:101B600089599F4F0E94EED89E012B593F4F44E068
:101B700050E0BE01695A7F4FCE0189599F4F0E94A4
:101B8000EED86B96CCACDDACEEACFFAC6B9720E046
:101B900030E84BE355E4C701B6010E944EEF8823BD
:101BA00029F18091CC07811108C0C0925D05D092C7
:101BB0005E05E0925F05F092600500E09E012B5902
:101BC0003F4F44E050E069E575E0CE0189599F4FF1
:101BD0000E94EED89E012B593F4F44E050E065E54E
:101BE00075E0CE0189599F4F0E94EED800E09E011A
:101BF0002B593F4F42E050E0BE016F597F4FCE015D
:101C000089599F4F0E94EED89E012B593F4F41E0CA
